:0200000480007A
:10000000970500009385450A732510FC6B10B50019
:10001000EF004009130510006B0005001775010083
:100020001305459B177601001306469E3306A6402E
:1000300093050000EF00804A170500001305451DD9
:10004000EF004045EF00C012EF0080006F00C04598
:1000500037550180130101FF130585F22326110096
:10006000EF0080598320C100130500001301010136
:100070006780000093070000638807003705008051
:100080001305C5206F00004167800000630605006E
:100090009301050073000000EF00801E13050000AF
:1000A0006B000500732500FC6B00050097610100E3
:1000B0009381C1751701007F1301C1F493050040BE
:1000C000732610CCB385C5023301B140F32630CC82
:1000D00063860600130500006B00050067800000C2
:1000E0001305F0FF678000001305F0FF6780000034
:1000F0001305000067800000130500006780000002
:100100001305F0FF67800000130500006780000002
:10011000130101FF23202101232611002324810044
:100120002322910013090600635EC00013840500BA
:10013000B384C5000345040013041400EF00C0128B
:10014000E31A94FE8320C10003248100832441002C
:100150001305090003290100130101016780000054
:100160001305F0FF67800000732540F167800000F1
:10017000130101FF23248100232021013764018022
:100180003769018093070400130909003309F94016
:1001900023261100232291001359294063000902EC
:1001A00013040400930400008327040093841400C4
:1001B00013044400E7800700E31899FE37640180C8
:1001C0003769018093070400130949003309F94096
:1001D000135929406300090213040400930400002A
:1001E000832704009384140013044400E78007006D
:1001F000E31899FE8320C100032481008324410079
:10020000032901001301010167800000130101FFB0
:1002100023248100B7670180376401801304440000
:1002200093874700B387874023229100232611003C
:1002300093D42740638004029387C7FF33848700E9
:10024000832704009384F4FF1304C4FFE7800700AE
:10025000E39804FE8320C10003248100832441002D
:100260001301010167800000F32220CC93F2F20316
:10027000130300FCB38262002380A20067800000A9
:10028000F32750CC3707FF00B387E7009397870029
:10029000732700B023A0E700732710B023A2E70064
:1002A000732720B023A4E700732730B023A6E7000C
:1002B000732740B023A8E700732750B023AAE700B4
:1002C000732760B023ACE700732770B023AEE7005C
:1002D000732780B023A0E702732790B023A2E70220
:1002E0007327A0B023A4E7027327B0B023A6E702C8
:1002F0007327C0B023A8E7027327D0B023AAE70270
:100300007327E0B023ACE7027327F0B023AEE70217
:10031000732700B123A0E704732710B123A2E704D9
:10032000732720B123A4E704732730B123A6E70481
:10033000732740B123A8E704732750B123AAE70429
:10034000732760B123ACE704732770B123AEE704D1
:10035000732780B123A0E706732790B123A2E70695
:100360007327A0B123A4E7067327B0B123A6E7063D
:100370007327C0B123A8E7067327D0B123AAE706E5
:100380007327E0B123ACE7067327F0B123AEE7068D
:10039000732700B823A0E708732710B823A2E70843
:1003A000732720B823A4E708732730B823A6E708EB
:1003B000732740B823A8E708732750B823AAE70893
:1003C000732760B823ACE708732770B823AEE7083B
:1003D000732780B823A0E70A732790B823A2E70AFF
:1003E0007327A0B823A4E70A7327B0B823A6E70AA7
:1003F0007327C0B823A8E70A7327D0B823AAE70A4F
:100400007327E0B823ACE70A7327F0B823AEE70AF6
:10041000732700B923A0E70C732710B923A2E70CB8
:10042000732720B923A4E70C732730B923A6E70C60
:10043000732740B923A8E70C732750B923AAE70C08
:10044000732760B923ACE70C732770B923AEE70CB0
:10045000732780B923A0E70E732790B923A2E70E74
:100460007327A0B923A4E70E7327B0B923A6E70E1C
:100470007327C0B923A8E70E7327D0B923AAE70EC4
:100480007327E0B923ACE70E7327F0B923AEE70E6C
:100490006780000093050500930600001306000026
:1004A000130500006F20D071130101FF93050000B8
:1004B000232481002326110013040500EF20107A65
:1004C000B777018003A5079C8327C50363840700D2
:1004D000E780070013050400EFF05FBB1303F00093
:1004E00013070500637EC3029377F7006390070A42
:1004F00063920508937606FF1376F600B386E6004E
:100500002320B7002322B7002324B7002326B700F7
:1005100013070701E366D7FE631406006780000037
:10052000B306C3409396260097020000B386560098
:100530006780C6002307B700A306B7002306B700ED
:10054000A305B7002305B700A304B7002304B70031
:10055000A303B7002303B700A302B7002302B70029
:10056000A301B7002301B700A300B7002300B70021
:100570006780000093F5F50F93968500B3E5D500ED
:1005800093960501B3E5D5006FF0DFF6939627004B
:1005900097020000B386560093820000E78006FAB7
:1005A00093800200938707FF3307F7403306F60076
:1005B000E378C3F66FF0DFF3130101FC2324C102DB
:1005C0002326D1022328E102232AF102232C01034E
:1005D000232E1103138605008325850093068102CF
:1005E000232E11002326D100EF0000068320C10135
:1005F0001301010467800000377301800323439CCB
:10060000130101FC2324C1022326D1022322B102BB
:100610002328E102232AF102232C0103232E1103B4
:10062000832583009306410213060500130503008A
:10063000232E11002326D100EF0000018320C101E9
:100640001301010467800000130101E12326111E3C
:10065000232A511D2328611D2320A11D938A0500F3
:10066000130D06002326D1002324811E2322911E70
:100670002320211F232E311D232C411D2326711DD4
:100680002324811D2322911D232EB11B130B050052
:10069000EF60406983270500138507002320F104DC
:1006A000EF804067232EA1022328010E232A010E8A
:1006B000232C010E232E010E63060B0083278B03D0
:1006C000E38A072A8396CA009397060113972601A7
:1006D00093D70701634A0702B727000003A64A061B
:1006E000B3E7F60093970701B7E6FFFF93D70741FB
:1006F0009386F6FFB376D6002396FA009397070108
:1007000023A2DA0693D7070193F687006380062EAB
:1007100083A60A01638C062C93F7A7019306A00019
:100720006388D72EB75701809387C7F7232AF10034
:1007300083470D00930BC110B75901802322710F1D
:100740002326010E2324010E23280100232C01005F
:1007500023220104232C0102232401042326010463
:100760002322010093880B009389890F638207225B
:1007700013040D00930650026388D740834714008A
:1007800013041400E39A07FEB304A4416302A421F6
:100790008326C10E8327810E23A0A801B38696006D
:1007A0009387170023A298002326D10E2324F10E4D
:1007B000930670009388880063C0F63E03274100CB
:1007C00083470400330797002322E1006382071C5C
:1007D00083441400A303010C130414001303F0FF5B
:1007E000130A000013090000130CA005930C9000DD
:1007F000930DA00213041400938704FE6364FC04A9
:100800000327410193972700B387E70083A70700D9
:1008100067800700130A0000938704FD83440400E7
:1008200093162A00338A4601131A1A00338A4701A5
:10083000938704FD13041400E3F2FCFE938704FE87
:10084000E370FCFC6386041423069114A303010CDB
:10085000130C1000930C1000130DC114930D000025
:100860001303000023260102232A01022328010288
:10087000937F290063840F00130C2C00137F490819
:100880008327C10E63180F0033088A4163540001A7
:100890006F00D07C8346710C638A06028326810E2A
:1008A0001306710C23A0C8009387170013061000CD
:1008B0009386160023A2C8002326F10E2324D10E0E
:1008C00013067000938888006342D662638C0F021F
:1008D0008326810E1306810C23A0C800938727006E
:1008E000130620009386160023A2C8002326F10ECB
:1008F0002324D10E13067000938888006354D60019
:100900006F10C00593060008E30ADF4633039341E6
:10091000E340605493760910E39606320327810E74
:10092000B387970123A0A8011307170023A29801FA
:100930002326F10E2324E10E9306700063C4E666BD
:10094000938888001379490063060900B3048A413B
:10095000634A906663548A01130A0C00032741001E
:10096000330747012322E100E392075A2324010EB3
:1009700063880D0093850D0013050B00EF3040399F
:1009800093880B00130D040083470D00E39207DEEC
:100990008327C10E638407006F10D03883D7CA0045
:1009A00093F70704638407006F2040298320C11E4A
:1009B0000324811E032541008324411E0329011EB7
:1009C0008329C11D032A811D832A411D032B011D7B
:1009D000832BC11C032C811C832C411C032D011C67
:1009E000832DC11B1301011F6780000093850A003E
:1009F00013050B00EF20D006630405006F200024D0
:100A000083D7CA009306A00093F7A701E39CD7D031
:100A10008397EA00E3C807D08326C10013060D00C0
:100A200093850A0013050B00EF2080772322A10095
:100A30006FF0DFF713050B00232E11012324610053
:100A4000EF60402E83274500138507002326F1041D
:100A5000EF80402C9307050013050B0093840700DB
:100A60002324F104EF60002C8327850003238100F9
:100A70008328C101232CF102638404006F10001845
:100A8000834404006FF01FD78344040013690902F4
:100A90006FF05FD6136909019377090263880760D5
:100AA0008327C1009387770093F787FF03A7470049
:100AB00083AD0700938787002326F100930C07007E
:100AC000634007621307F0FF130C09006300E3762D
:100AD00033E79D01137CF9F7631A0774631E0374EF
:100AE00013090C0013030000930C0000130D011BED
:100AF000138C0C0063D46C00130C03008347710C3F
:100B000023260102232A010223280102930D00005B
:100B1000E38007D6130C1C006FF09FD51369090101
:100B200093770902638C07548327C10013877700EA
:100B3000137787FF832D0700832C470093078700D7
:100B40002326F100137CF9BF13070000A303010C57
:100B50009306F0FF630AD35AB3E69D011379FCF7BD
:100B6000E39A064EE3120308E31E07F6937C1C008B
:100B7000130D011BE38E0CF693070003A307F11A74
:100B8000130DF11A6FF0DFF6B304A441E312A4C110
:100B9000834704006FF09FC31306410E93850A003C
:100BA00013050B00EFA0D065E31A05DE93880B0058
:100BB0006FF0DFC093778900639407006F10C0085F
:100BC0000327C10083270700130747002326E100FE
:100BD00083A5070003A6470083A6870083A7C70055
:100BE0002328B10E232AC10E232CD10E232EF10E61
:100BF0001305010F232E110123246100EF60C00BA8
:100C00002326A10C93072000032381008328C10120
:100C10006314F5006F100048930710006314F5008B
:100C20006F10C05C930710066394F4006F204018A7
:100C3000930710046394F4006F10101093FCF4FDFC
:100C40009307F0FF232891076314F3006F204017E8
:100C5000930770046394FC006F200017032EC10FEC
:100C600023242107832E010F032F410F832F810F90
:100C70009367091063540E006F204039232E01063C
:100C800013890700930D0000930760046394FC0030
:100C90006F10906293075004232411036384FC00B7
:100CA0006F101059930C1300130C010B1308C10D96
:100CB00093860C009307010D1307C10C1306200047
:100CC00093050C0013050B00232261022328D10B8E
:100CD0002320D103232AE10B232EE101232CF10B46
:100CE0002328F101232EC10B2324C101EF40905092
:100CF000032E8100832F0101032FC101832E0102E6
:100D0000032341028328810233089501130D050056
:100D1000930C010A93850C0013050C00232E01018E
:100D200023281101232461002328D10B232AE10B5E
:100D3000232CF10B232EC10B2320010A2322010AAD
:100D40002324010A2326010AEF00C1620328C101FE
:100D50000323810083280101930708006302050231
:100D60008327C10D63FE0701130600039386170056
:100D7000232ED10C2380C7008327C10DE3E807FF92
:100D80000327C10CB387A7412328F1002328E102E0
:100D900003270107930770046314F7006F10903A5C
:100DA00003270107930760046314F7006F10D063F3
:100DB0008327010303270107930510049387F7FF97
:100DC0002326F10C93F6F40F130600006318B70006
:100DD0009386F60093F6F60F13061000230AD10C43
:100DE0009306B00263DA070003270103930710009C
:100DF0009306D002B387E740A30AD10C9306900074
:100E000063C4F6006F2040211308310E130508005B
:100E10001306A000130E3006B3E6C70293050500C3
:100E2000138307001305F5FF93860603A38FD5FEF2
:100E3000B3C7C702E3426EFE9387070313F6F70FAB
:100E4000A30FC5FE9387E5FF63E407016F20C0325F
:100E50009306610D6F00800003C607002380C60063
:100E60009387170093861600E39807FF9307510EA8
:100E7000B387B7401307610DB307F7009306410D21
:100E8000B387D7402322F1040327010183264104BD
:100E900093071000B30CD70063C4E7006F208025D0
:100EA0008327C103B38CFC008327810613CCFCFF8E
:100EB000135CFC4113F9F7BF1369091033FC8C0173
:100EC00023260102232A0102232801028327C107C6
:100ED000639407006F10502E9307D002A303F10C08
:100EE00013030000130C1C006FF09F981306410EB3
:100EF00093850A0013050B0023206102232EE101D4
:100F00002324F101EFA0D02FE31C05008327C10E9D
:100F100003230102032FC101832F810093880B005B
:100F20006FF0DF9A832601040327C10313067000C4
:100F300023A0D8008326810EB307F70023A2E80080
:100F4000938616002326F10E2324D10E9388880061
:100F50006354D6021306410E93850A0013050B0055
:100F6000EFA0102A631E057A8325C10C8327C10ECA
:100F70008326810E93880B0063D405006F10904D7B
:100F8000032701019386160023A0A801B307F700E9
:100F900023A2E8002326F10E2324D10E13077000AC
:100FA000E350D79A1306410E93850A0013050B00F0
:100FB000EFA01025631605768327C10E93880B00DA
:100FC0006FF05F98930600010327810E63C49600BB
:100FD0006F109047B7560180938E860E130900015B
:100FE000930C70006F00C000938404FF635A99044F
:100FF000938707011307170023A0D80123A2280114
:101000002326F10E2324E10E93888800E3DEECFC16
:101010001306410E93850A0013050B002324D1010A
:10102000EFA0101E631E056E938404FF8327C10E7C
:101030000327810E832E810093880B00E34A99FADF
:10104000B38797001307170023A0D80123A29800A5
:101050002326F10E2324E10E93067000E3DCE68ED6
:101060001306410E93850A0013050B00EFA05019DB
:101070006318056A8327C10E6FF0DF8D8326C100D8
:101080009377090113874600E39C0740937709048F
:10109000639407006F1000108327C100930C0000B9
:1010A0002326E10083DD07006FF0DFA98326C1005E
:1010B0009377090113874600E39E07369377090467
:1010C000639407006F1080108327C1002326E1007E
:1010D000839D070093DCFD4113870C00E354079EBA
:1010E0003337B001B3079041B38CE7401307D00208
:1010F000A303E10C9306F0FFB30DB041130C0900FC
:1011000013071000E31AD3A4930610006300D7124C
:10111000930620006306D72E130D011B1396DC01E6
:1011200093F67D0093DD3D0093860603B36DB60113
:1011300093DC3C00A30FDDFE33E69D0193050D001B
:10114000130DFDFFE31C06FC93771C006384072E40
:10115000930700036380F62E9385E5FFA30FFDFE42
:101160009307011BB38CB74013090C00138D0500C6
:101170006FF01F9813050B00EF2010216FF08FD434
:101180000327C100A303010C130C100083270700E1
:10119000130747002326E1002306F114930C1000E7
:1011A000130DC1146FF08FEB8327C100A303010C53
:1011B00003AD070093864700E3040D409307F0FF5B
:1011C000E306F376130603009305000013050D00F4
:1011D000232ED1002326110123246100EF608050CB
:1011E000032381008328C1008326C101930D0500DC
:1011F000631405006F109018B30CA5418347710C60
:1012000013CCFCFF135CFC412326D10023260102F2
:10121000232A01022328010233FC8C01930D0000D4
:1012200013030000E398078E6FF08FE4E3920C48FD
:1012300013079000E36EB747938D0D03A307B11B0F
:1012400013090C00930C1000130DF11A6FF05F8A54
:1012500083440400136949006FF0CFD99307B002AB
:1012600083440400A303F10C6FF0CFD8834404003F
:10127000136909086FF00FD8834404009306140023
:101280006394B4016F10106C938704FD13840600FF
:101290001303000063E2FCD683440400931623008A
:1012A00033836600131313003303F300938704FDA5
:1012B00013041400E3F2FCFE6FF00FD48327C10087
:1012C0008344040003AA0700938747002326F10004
:1012D00063520AD2330A4041136949006FF08FD13B
:1012E00083440400136919006FF0CFD08347710C59
:1012F00083440400639007D093070002A303F10C1A
:101300006FF04FCF136C090193770C02E38C070841
:101310008327C10013877700137787FF9307870020
:10132000832D0700832C47002326F10013071000AC
:101330006FF0DF8183440400136989006FF08FCB65
:101340008327C1003787FFFF1347078383AD07005B
:101350002314E10C93874700375701802326F100BF
:10136000930787F4930C0000136C2900232CF100E1
:1013700013072000930480076FF04FFD8326C10000
:101380009377090203A70600938646002326D1001F
:10139000E39A070493770901E392075893770904C6
:1013A000638407006F10C01013790920E308095601
:1013B00083274100130D04002300F7006FF0CFDCFA
:1013C000834404009307C006E38CF41A13690901EF
:1013D0006FF04FC28344040093078006E38AF41839
:1013E000136909046FF00FC1930610006314D7004E
:1013F0006F10901193062000130C0900E31ED7D044
:10140000130D011B8327810193F6FD0093DD4D0031
:10141000B386D70003C606009396CC01B3EDB601A0
:1014200093DC4C00A30FCDFEB3E69D01130DFDFF31
:10143000E39A06FC9307011BB38CA74113090C0028
:101440006FF00FEB9306500663D6962E8326010F9E
:101450009305010A1305010B2328D10A8326410FA6
:10146000232EF10023241101232AD10A8326810F80
:101470002320010A2322010A232CD10A8326C10F2B
:101480002324010A2326010A232ED10AEFF0906EAD
:10149000832881008327C101631A054E0327810E2B
:1014A000B7560180938686F723A0D800938717004C
:1014B000930610001307170023A2D8002326F10E6D
:1014C0002324E10E9306700093888800E3C0E63879
:1014D0000327C10C83260101635ED76E0327010435
:1014E0008326C1039388880023ACE8FE0327810E7E
:1014F000B387D70023AED8FE130717002326F10EBB
:101500002324E10E93067000E3CCE60803270101D3
:101510009304F7FF635890C2930600010327810EDE
:10152000E3D69634930C0001130D70006F00C000D9
:10153000938404FFE3DC9C329387070113071700B1
:1015400023A0380123A298012326F10E2324E10EC3
:1015500093888800E35EEDFC1306410E93850A0034
:1015600013050B00EFA0C049631C051A8327C10EA9
:101570000327810E93880B006FF09FFB33088A418D
:10158000635600B9130600018326810E635C0607CB
:10159000130E0001930E70006F00C000130808FFC7
:1015A00063520E07938707019386160023A0380124
:1015B00023A2C8012326F10E2324D10E938888008C
:1015C000E3DEDEFC1306410E93850A0013050B00D3
:1015D000232E010123246100EFA080426312051431
:1015E0000328C101130E00018327C10E130808FF51
:1015F0008326810E0323810093880B00930E7000D5
:10160000E3420EFBB38707019386160023A038013F
:1016100023A208012326F10E2324D10E1306700005
:10162000938888006354D6AE1306410E93850A0052
:1016300013050B0023246100EFA0803C6312050E0C
:101640008327C10E0323810093880B006FF00FAC3A
:10165000130600018326810E6358660613080001F5
:10166000130E70006F00C000130303FF635E680475
:10167000938707019386160023A0380123A208014F
:101680002326F10E2324D10E93888800E35EDEFC2E
:101690001306410E93850A0013050B0023246100F5
:1016A000EFA00036631E0506032381001308000126
:1016B0008327C10E130303FF8326810E93880B003B
:1016C000130E7000E34668FAB3876700938616002E
:1016D00023A0380123A268002326F10E2324D10E73
:1016E00013067000938888006356D6A21306410E35
:1016F00093850A0013050B00EFA0803063120502EA
:101700008327C10E93880B006FF0CFA01306410E04
:1017100093850A0013050B00EFA0802E630805A433
:10172000638E0DA693850D0013050B00EF20405E20
:101730006FF0CFA60326810E032701019306100048
:1017400023A0A8019387170093041600938C8800A8
:1017500063DCE63A9306100023A2D8002326F10E9C
:101760002324910E9306700063C096700327C10373
:101770008326010493841400B387E70023A0DC00D0
:1017800023A2EC002326F10E2324910E9306700071
:10179000938C8C0063CC966E8326010F1388140003
:1017A0009305010A2328D10A8326410F1305010B53
:1017B000232EF100232AD10A8326810F232401013D
:1017C0002320010A232CD10A8326C10F2322010AD8
:1017D0002324010A232ED10A2326010AEFF090398F
:1017E000832701010328810093888C009386F7FFEB
:1017F000130608008327C101630C053213071D007F
:10180000B387D70023A0EC0023A2DC002326F10E2F
:101810002324010F130770006344074D13870C0145
:1018200013862400938C0800930807008326410444
:101830001307410D23A0EC00B387F60023A2DC00C0
:101840002326F10E2324C10E13077000635CC78E9C
:101850006FF04FF5130C09006FF01F8B37570180A5
:10186000130600018326810E930E870E130E0001CE
:1018700093027000634806016F004008130808FFD8
:10188000635E0E07938707019386160023A0D80195
:1018900023A2C8012326F10E2324D10E93888800A9
:1018A000E3DED2FC1306410E93850A0013050B00FC
:1018B0002324D1032322010323206102232EE101EB
:1018C0002324F101EFA0C013E31C05E40328410227
:1018D000130E00018327C10E130808FF8326810E13
:1018E000832E810203230102032FC101832F810074
:1018F00093880B0093027000E3460EF9B38707014B
:101900009386160023A0D80123A208012326F10EF6
:101910002324D10E13067000938888006344D600F8
:101920006FE05FF71306410E93850A0013050B0065
:1019300023206102232EE1012324F101EFA0400CBA
:10194000E31005DE8327C10E03230102032FC1012B
:10195000832F810093880B006FE0DFF31306410EA5
:1019600093850A0013050B00232E61002324E10157
:10197000EFA00009E31605DA8327C10E0323C10196
:10198000032F810093880B006FE0DFF78325C10CE4
:10199000635CB06003270103832601019304070001
:1019A00063C8E630635690028326810EB3879700A2
:1019B00023A0A8019386160023A298002326F10EE7
:1019C0002324D10E1306700093888800E34ED62896
:1019D00093C6F4FF0327010393D6F641B3F4D40072
:1019E000B3049740634E903E03270103937609406A
:1019F000B304ED00E39E06048325C10C0327010117
:101A000063C6E50093761900E38406288326010463
:101A10000327C1031306700023A0D8008326810E7C
:101A2000B387E70023A2E800938616002326F10E71
:101A30002324D10E938888006354D6006F10C01001
:101A4000832601013307DD003386B6403307974014
:101A5000930C06006354C700930C0700635890036F
:101A60000327810EB387970123A09800130717005F
:101A700023A298012326F10E2324E10E9306700081
:101A80009388880063D4E6006F10401813C7FCFFEA
:101A90001357F74133F7EC00B304E640634490007A
:101AA0006FE05FEA930600010327810E63D0965C26
:101AB000930C0001130D70006F00C000938404FFAD
:101AC00063D69C5A938707011307170023A0380198
:101AD00023A298012326F10E2324E10E9388880087
:101AE000E35EEDFC1306410E93850A0013050B001F
:101AF000EF901071E31605C28327C10E0327810EF4
:101B000093880B006FF09FFB93751900E39405C455
:101B100023A2D8002326F10E2324910E1307700070
:101B20006340971C13062600938808016FF01FD0AE
:101B3000E35ED0CE130700016344D7006F10C05C92
:101B4000130D70006F000001938606FF6358D716CF
:101B5000138814009387070123A03C0123A2EC0003
:101B60002326F10E2324010F93040800938C8C008C
:101B7000E35C0DFD1306410E93850A0013050B006F
:101B80002324D100EF90D067E31C05B88327C10E52
:101B90008324810E83268100938C0B0013070001A0
:101BA0006FF09FFA8326C10093770C0113874600DC
:101BB0006398070693770C04638E075A8327C10046
:101BC000930C00002326E10083DD070013071000BB
:101BD0006FE0DFF713771900631407006FE09FD6FB
:101BE0006FF0DF8F83264100130D040093D7F64179
:101BF0002320D7002322F7006FE01FD9832781031A
:101C000083440400639407006FE0DFBE83C70700CE
:101C1000639407006FE01FBE136909406FE09FBD2A
:101C20002326E10083AD0600930C0000130710008B
:101C30006FE0DFF183AD06002326E10093DCFD4178
:101C400013870C006FE0DFE78327C1001305010B4A
:101C5000232E11019387770093F787FF83A5070051
:101C600003A6470093878700232461002326F10001
:101C7000EF2051368327010B8328C1010323810004
:101C80002328F10E8327410B232AF10E8327810B92
:101C9000232CF10E8327C10B232EF10E6FE05FF58D
:101CA00083AD0600930C00002326E1006FE09FE95E
:101CB00093840600E34A90CE6FF09FD11386140000
:101CC00013878C00B387D70023A2DC0023A03C013C
:101CD0002326F10E2324C10E9306700063D6C6742A
:101CE0001306410E93850A0013050B00EF90505127
:101CF000E31805A20326810E8327C10E9308411124
:101D000013061600938C0B006FF05FB2130C0900E2
:101D10006FF08FDFB7570180938787F4232CF10092
:101D200093770902638207128327C1001387770024
:101D3000137787FF832D0700832C470093078700C5
:101D40002326F10013771900630E070033E79D0186
:101D5000630A0700130700032304E10CA304910C9A
:101D600013692900137CF9BF130720006FE01FDE01
:101D70008344140013690920130414006FE09FA723
:101D80008344140013690902130414006FE09FA632
:101D9000B75701809387C7F5232CF1006FF05FF8E8
:101DA0001306410E93850A0013050B00EF90504572
:101DB000E31805968327C10E93880B006FF00FF58B
:101DC00093076000930C030063E0676C3757018052
:101DD000138C0C002326D100130D07F76FE01FA80A
:101DE000130600018326810E63529642930C000174
:101DF000130870006F00C000938404FF63D89C40F8
:101E0000938707019386160023A0380123A2980127
:101E10002326F10E2324D10E93888800E35ED8FC9C
:101E20001306410E93850A0013050B00EF90503DF9
:101E3000E318058E8327C10E8326810E93880B003D
:101E4000130870006FF05FFB8326C10093770901D0
:101E500013874600638E071C83AD0600930C0000B9
:101E60002326E1006FF01FEE1306410E93850A0052
:101E700013050B00EF90D038E314058A8327C10EB9
:101E80008324810E938C0B006FF05F8E1306410E3E
:101E900093850A0013050B00EF909036E312058836
:101EA0008327C10E8324810E938C0B006FF0DF8E8D
:101EB00013790C4023280100130D011B6F00400310
:101EC0001306A0009306000013850D0093850C00F7
:101ED000232E110123246100EFD0103F0323810042
:101EE0008328C101E3840C2E930D0500938C05001B
:101EF0001306A0009306000013850D0093850C00C7
:101F0000232E110123246100EFD0507F832701018C
:101F100013050503A30FADFE938717002328F100D7
:101F2000032381008328C101130DFDFFE30A09F893
:101F30000327810383460700E394D7F81307F00FC4
:101F4000E380E7F863960C009307900063F4B7CF43
:101F5000832781048325C104232E1101330DFD4005
:101F60001386070013050D0023246100EF60506302
:101F7000832781031306A0009306000003CE1700F9
:101F800013850D0093850C00333EC001B387C70154
:101F9000232CF102EFD05033032381008328C101A9
:101FA000232801006FF05FF48326810E37560180ED
:101FB000130686F723A0C8009387170013061000A6
:101FC0009386160023A2C8002326F10E2324D10EE7
:101FD00013067000938888006340D646638405002A
:101FE0006FE05FF40327010193761900B3E6E60082
:101FF000639406006FE01F95832601040327C10345
:102000001306700023A0D8008326810EB307F700C3
:1020100023A2E800938616002326F10E2324D10E76
:102020006354D6006FE01FF3938888006FE05FF57C
:1020300093770904638E07168327C100930C000071
:102040002326E10083DD07006FF0DFCF1306410E8A
:1020500093850A0013050B00EF90901A631205ECAC
:102060008327C10E93880B006FF08FC623A0380121
:1020700023A29800B3879700130717002326F10EB9
:102080002324E10E9306700063C4E6006FE05F8BCB
:102090006FE05FF18327010F9305010A1305010B20
:1020A0002328F10A8327410F232411012320010A49
:1020B000232AF10A8327810F2322010A2324010AFC
:1020C000232CF10A8327C10F2326010A232EF10AAC
:1020D000EFF0C05183288100E34C05288347710C41
:1020E00013077004635C973637570180130DC7F3ED
:1020F00023260102232A0102232801021379F9F77A
:10210000130C3000930D0000930C300013030000FB
:10211000638407006FE01FA06FE08FF58327410005
:10212000130D04002320F7006FE01F8613050D0038
:10213000232411012326D100EF60D03D8347710C89
:10214000134CF5FF135CFC4123260102232A0102F4
:102150002328010283288100930C0500337C85012C
:10216000930D000013030000638407006FE09F9A43
:102170006FE00FF093770C20638407388327C1004A
:10218000930C00002326E10083CD07001307100005
:102190006FE0DF9B93770920638A07348327C100B0
:1021A000930C00002326E10083CD07006FE09F9988
:1021B00093770920638207328327C100930C0000C4
:1021C0002326E10083CD07006FF0DFB79377092066
:1021D0006388072E8327C1002326E100838D070033
:1021E00093DCFD4113870C006FE09F8D8327C10FA7
:1021F00063C407328347710C13077004E356971AC0
:1022000037570180130D47F46FF09FEEB3879700A7
:102210009386160023A0380123A298002326F10EEE
:102220002324D10E1306700093888800635ED6FACB
:102230001306410E93850A0013050B00EF90407CB6
:10224000631005CE8327C10E93880B006FF0CFF982
:1022500003270101130E7000130800013307ED007E
:102260002324E10003274103630E070A0327C10269
:10227000631E070A032781031307F7FF232CE102DC
:10228000032741031307F7FF232AE1028326C10432
:10229000032781049388880023ACD8FE8326810E0F
:1022A000B387E70023AEE8FE938616002326F10EDF
:1022B0002324D10E634EDE100327810383460700DB
:1022C00003278100938C0600330697406354D600A1
:1022D000930C0600635890038326810EB387970101
:1022E00023A098009386160023A298012326F10EBE
:1022F0002324D10E6342DE100327810393888800D4
:102300008346070013C6FCFF1356F641B3FCCC000E
:10231000B38C964163449003B384D40003274103F4
:10232000E31607F40327C102630407600327C10211
:102330001307F7FF2326E1026FF05FF58326810E76
:10234000634898016F00C005938C0CFF635A980591
:10235000938707019386160023A0380123A2080162
:102360002326F10E2324D10E93888800E35EDEFC41
:102370001306410E93850A0013050B00EF90406889
:10238000631005BA13080001938C0CFF8327C10E5C
:102390008326810E93880B00130E7000E34A98FB8E
:1023A000B38797019386160023A0380123A29801D2
:1023B0002326F10E2324D10E6340DE64032781031C
:1023C0009388880083460700B384D4006FF01FF51C
:1023D0001306410E93850A0013050B00EF9040622F
:1023E000631005B48327C10E93880B001308000106
:1023F000130E70006FF05FEC1306410E93850A0018
:1024000013050B00EF90C05F631C05B083278103A9
:1024100093880B001308000183C60700130E700099
:102420008327C10E6FF01FEE130616009308870076
:10243000930C07006FF08FBF1306410E93850A00BF
:1024400013050B00EF90C05B631C05AC8325C10C2A
:102450008327C10E93880B006FF05FB83757018058
:10246000130D87F36FF0DFC81306410E93850A0042
:1024700013050B00EF90C058631405AA8327C10E03
:1024800093880B006FF0CFD4930C60006FF01F9413
:10249000832601013307DD003386B64033039740BE
:1024A000930C06006354C3DE930C03006FF00FDE41
:1024B00083274100130D04002310F7006FE0CFCCF9
:1024C0008327C1002326E10083AD070093DCFD4193
:1024D00013870C006FE0CFDE8327C100930C000050
:1024E0002326E10083AD07006FF0DF858327C1005D
:1024F000930C00002326E10083AD07006FE08FE41A
:102500008327C100930C00002326E10083AD070060
:10251000130710006FE08FE39307D002A303F10CC1
:102520006FF09FCD1306410E93850A0013050B0033
:10253000EF90004D6FE08FC6930700032304F10C6A
:102540009307800513672900A304F10C2324E106F7
:1025500093073006930D0000130DC114E3C4670206
:10256000032EC10F93FCF4FD23289107232E0106AF
:10257000832E010F032F410F832F810F1369291021
:1025800063420E4693071006E38AF416930710047D
:102590006384F4006FE04FEF130C010B13050C0084
:1025A00023261103232461022328D10B232AE10BC4
:1025B000232CF10B232EC10BEF2041441306C10C39
:1025C000EF604035138605009305050013050C00E8
:1025D000EF20412093070109938507002324F10090
:1025E0008327010B930C010A130601082328F10825
:1025F0008327410B13850C002326C106232AF108EB
:102600008327810B2320010823220108232CF108B2
:102610008327C10B23240108232EF108B707FC3FB1
:102620002326F108EFF040110328010A032E410A86
:10263000832E810A032FC10A93850C0013050C0019
:102640002328010B23220103232AC10B2320C103CA
:10265000232CD10B232ED101232EE10B2328E101C2
:102660002320010A2322010A2324010A2326010A26
:10267000EFE05050032F0101832EC101032E010210
:1026800003284102032381028328C1026316050047
:10269000930710002326F10CB75701809387C7F5E5
:1026A0002322F1069306F3FF93070D006F00C00885
:1026B00093850C0013050C002320C106232EF10581
:1026C000232C5104232A71042328F1042328710A9E
:1026D00023267102232A510A23245102232CF10BB1
:1026E0002322F103232EC10A2320C1022320010A41
:1026F0002322010A2324010A2326010AEFE090473E
:102700008326C101032F0102832E4102032E810281
:102710000328C10203230103832841038327010502
:102720008323410583228105832FC10503260106EA
:102730009386F6FF630E05100326810093850C0037
:102740002328F10413050C00B7070340232A1103C3
:10275000232861022326D102232EF1082326E10B30
:102760002320010B2322C10B2324D10B2328010892
:10277000232A0108232C0108EFE0107C832E010B93
:10278000032E410B0328810B0326C10B13050C00FC
:102790002324D1032322C10323200103232EC100BC
:1027A000EF109153930505002328A10013050C0099
:1027B000EF10516D0326C101832E8102032E4102C9
:1027C000232EC1080326010B032801028325810063
:1027D0002320C1080326410B13850C002328D109AF
:1027E0002322C1080326810B232AC109232C0109B6
:1027F0002324C1080326C10B2326C1080326C106D2
:10280000EF00012103274106832701018326C1022E
:102810008323010A3306F700834506008327010559
:102820008322410A832F810A0326C10A232CF10641
:102830002380B700232AD1061307F0FF232ED100EF
:10284000032301038328410393871700E392E6E6FD
:10285000B706FE3F93850C0013050C002320F10200
:10286000232E1101232461002328710A23287102D9
:10287000232A510A23265102232CF10B2324F1038E
:10288000232EC10A2322C1022320010A2322010A86
:102890002324010A2326D10AEFE09040032381007C
:1028A0008328C101832701026344A04683230103D7
:1028B0008322C102832F810203264102B706FE3F15
:1028C00093850C0013050C002328710A232A510A52
:1028D000232CF10B232EC10A2320010A2322010AF3
:1028E0002324010A2326D10AEFE0D0280323810004
:1028F0008328C10183270102631805000327010112
:1029000093761700639606400327410713060003DA
:1029100093061700B386D700635407006FE04FC6D5
:1029200093871700A38FC7FEE39CF6FE6FE04FC5A9
:1029300003270101B306ED0063F0968C9384060033
:102940006FF08F8B032701039307D0FF6344F700D9
:10295000635AE3009384E4FF93F7F4FD2328F10620
:102960006FE00FC583270101032701036344F724A8
:1029700083278106930C070093F7170063860700EF
:102980008327C103B30CF7008327810693F7074021
:102990006386070083270103634AF04C13CCFCFFD6
:1029A000135CFC4133FC8C01930470062326010266
:1029B000232A01026FE08FD18347710C13030000BB
:1029C000638407006FE00F956FD09FEA9307900034
:1029D00063ECB7D16FE01FA623242107930D0000FD
:1029E00013890200B707008033CEC7019307D002D6
:1029F000232EF1066FF01FB91306410E93850A00CE
:102A000013050B00EF80D07F630405006FE05FD1FA
:102A10008327810393880B001308000183C60700F6
:102A2000130E70008327C10EB384D4006FF01F8F84
:102A3000130C010B9307010D930603001308C10D3E
:102A40001307C10C1306200093050C0013050B009F
:102A5000232261022328D10B2320D103232AE10B57
:102A6000232EE101232CF10B2328F101232EC10B8E
:102A70002324C101EF20107893077004032E8100F6
:102A8000832F0101032FC101832E01020323410281
:102A900083288102130D05006394FC0883278106B7
:102AA00093F717006396072C130770048327C10D53
:102AB0002328E1066FE0CFAC130C010B9306030053
:102AC0001308C10D9307010D1307C10C1306300045
:102AD00093050C0013050B0023241103232261022C
:102AE0002328D10B2320D103232AE10B232EE1013C
:102AF000232CF10B2328F101232EC10B2324C10128
:102B0000EF20506F032E8100832F0101032FC1019D
:102B1000832E01020323410283288102130D050045
:102B20009307600433086D00639AFC2483460D000C
:102B3000930700036380F654930C010A8327C10CAA
:102B40003308F8006FE00F9D1306410E93850A00CD
:102B500013050B00EF80D06A630405006FE05FBCD3
:102B60008325C10C8327C10E93880B006FE05FEDB6
:102B70009307D002A303F10C6FF08FD68347710C3B
:102B80002326D10023260102232A01022328010241
:102B9000130C0300930C030013030000638407006D
:102BA0006FD05FF76FD0DFCC37570180130D07F47C
:102BB0006FF00FD4832701010327C103930470062C
:102BC000B38CE70083270103635AF048832781060B
:102BD00093F70740639E072813CCFCFF135CFC416E
:102BE00033FC8C016FF09FDC8327810603270103F0
:102BF00093F71700B3E76700635CE0506396074400
:102C0000832C0103930460066FF05FFC1306410EF2
:102C100093850A0013050B00EF80905E63040500A6
:102C20006FE01FB08324C10C032701018327C10E6D
:102C300093880B00330697406FE05FE59307F0FF42
:102C40002322F1006FD09FD6B7560180938E860E57
:102C50006FE00FBF130600FFB304B04063D2C50698
:102C6000930C0001130870006F00C000938404FFF0
:102C700063D89C04938707019386160023A038012C
:102C800023A298012326F10E2324D10E93888800D5
:102C9000E35ED8FC1306410E93850A0013050B0072
:102CA000EF801056630405006FE09FA78327C10ED5
:102CB0008326810E93880B00130870006FF01FFBB2
:102CC000B38797009386160023A0380123A29800AB
:102CD0002326F10E2324D10E130670006356D6B4BA
:102CE0001306410E93850A0013050B00EF80505127
:102CF000630405006FE0DFA28327C10E8326810EE7
:102D000093880B006FE0CFA7130C09006FE0CFD2C0
:102D10000327810793860700232EE10C0327410632
:102D200003C6F7FF8345F7006310B60213050003DF
:102D3000A38FA6FE8326C10D1386F6FF232EC10C9A
:102D400003C6F6FFE386C5FE930516001305900340
:102D500093F5F50F6306A600A38FB6FE6FE04F82D2
:102D6000032741068345A700A38FB6FE6FE04F817E
:102D70009307700433086D002328F106930C010AB1
:102D80006FD05FF99305130013050B002328110181
:102D900023246100EF40801903238100832801016F
:102DA000130D05006302053C930D05006FF04FFB0A
:102DB000930700032304F10C930780076FF08FF84B
:102DC000130360006FD09FE9631403001303100026
:102DD000032EC10F832E010F032F410F832F810F6D
:102DE00093620910E34A0EBE130C010B9306030015
:102DF0001308C10D9307010D1307C10C1306200022
:102E000093050C0013050B00232651022324110304
:102E1000232261022328D10B2320D103232AE10B93
:102E2000232EE101232CF10B2328F101232EC10BCA
:102E30002324C101EF20103C8322C1022324210757
:102E4000032E8100832F0101032FC101832E010274
:102E50000323410283288102130D05001389020018
:102E6000232E0106930D00006FF05FC393047006DC
:102E7000832781039306F00F2326010283C70700EF
:102E8000232A01026388D7040327010363D4E704DC
:102E9000B307F740032781032328F1028347170074
:102EA000638E07000326410313071700232CE1025A
:102EB00013061600232AC1026FF0DFFC0327C102AC
:102EC000832781031307170083C707002326E10226
:102ED0006FF05FFB0327C10283274103B387E7003D
:102EE00003278104B387E702B38C970113CCFCFF5F
:102EF000135CFC4133FC8C016FD05FFD130C010BA4
:102F000013050C0023261103232461022328D10B6F
:102F1000232AE10B232CF10B232EC10BEF10112ED2
:102F20001306C10CEF50101F138605009305050012
:102F300013050C00EF10110A930701099385070090
:102F40002324F1008327010B930C010A13060108C7
:102F50002328F1088327410B13850C002326C10683
:102F6000232AF1088327810B23200108232201084B
:102F7000232CF1088327C10B23240108232EF108F9
:102F8000B707FC3F2326F108EFE0007B0328010A86
:102F9000032E410A832E810A032FC10A93850C0058
:102FA00013050C002328010B23220103232AC10B44
:102FB0002320C103232CD10B232ED101232EE10B7F
:102FC0002328E1012320010A2322010A2324010AE4
:102FD0002326010AEFE0003A032F0101832EC101ED
:102FE000032E010203284102032381028328C10228
:102FF00063160500930710002326F10CB7570180D4
:10300000938787F42322F1066FF0CFE9930D000038
:10301000138907006FF01F9D9306610D631806006A
:1030200093060003230BD10C9306710D1307011BAC
:10303000938707033386E6402380F6009307D60D77
:103040002322F1046FD05FE48327C1039304600659
:10305000B30CF700B38C6C006FF05FB7B38CFC401F
:10306000938C1C0013CCFCFF135CFC4133FC8C01E3
:103070006FF0DF93930C010A93850C0013050C008D
:103080002326010323241103232261022328D10BC9
:103090002320D103232AE10B232EE101232CF10B62
:1030A0002328F101232EC10B2324C1012320010A6F
:1030B0002322010A2324010A2326010AEFE0802BA0
:1030C000032E8100832F0101032FC101832E0102F2
:1030D00003234102832881020328C102E30005A6DD
:1030E00093071000B38767402326F10C3308F800DC
:1030F0006FD05FC28327810693F7170063940700A0
:103100006FD09FDA6FD0DFD9138708006FE09FBBC5
:10311000639A0700130C100093046006930C1000D0
:103120006FF0DF888327C10393046006938C170038
:10313000B38C6C0013CCFCFF135CFC4133FC8C01A2
:103140006FF0DF868327C10003A307009387470042
:10315000635403001303F0FF834414002326F1009B
:10316000138406006FD00FE983D7CA0093E70704E2
:103170002396FA006FD09F82930720002322F10448
:103180006FD09FD037770180930705000325479CB8
:103190009306060013860500938507006FD0CFCAFB
:1031A00083D7C50003AE450603D3E50083A8C50158
:1031B00003A84502130101B893F7D7FF1307004096
:1031C000232C8146231AF10013840500930701077D
:1031D00093058100232A914623282147232E114657
:1031E000130905002326C107231B610023221103B5
:1031F000232601032324F100232CF1002328E100DE
:10320000232EE10023200102EFD00FC49304050018
:10321000635C05028357410193F707046388070045
:103220008357C40093E707042316F4008320C147A3
:103230000324814703290147138504008324414760
:103240001301014867800000930581001305090000
:10325000EF00C058E30005FC9304F0FF6FF09FFB04
:10326000B777018083A7479C130101FF23248100C6
:1032700023229100232611009304050013840500E6
:103280006386070003A787036300070E0317C400C4
:10329000931707019376870093D70701638006048D
:1032A000832604016380060613F6170063040608EC
:1032B0000326440123240400130500003306C04004
:1032C000232CC400638606088320C10003248100E8
:1032D00083244100130101016780000093F6070178
:1032E0006384060C93F7470063960708832604015E
:1032F00013678700931707012316E40093D707018C
:10330000E39406FA13F6072893050020E30EB6F8B7
:103310009305040013850400EF30502F0317C400F9
:10332000832604019317070193D7070113F61700AB
:10333000E31006F813F62700930500006314060057
:10334000832544012324B40013050000E39E06F600
:1033500093F70708E38A07F6136707042316E400C8
:103360001305F0FF6FF05FF613850700EF00D00143
:103370006FF0DFF183250403638E050093070404D7
:103380006388F50013850400EF0090180317C4004C
:1033900023280402832604011377B7FD23220400A7
:1033A0002320D4006FF0DFF49307900023A0F400F3
:1033B000136707042316E4001305F0FF6FF0DFF036
:1033C000B777018003A7079C83278714638C0704C2
:1033D00003A747001308F001634EE80613182700FF
:1033E00063060502338307012324C30883A88718D3
:1033F000130610003316E600B3E8C80023A417191B
:103400002324D310930620006304D502130717006A
:1034100023A2E700B387070123A4B7001305000028
:10342000678000009307C7142324F7146FF05FFA36
:1034300083A6C7181307170023A2E70033E6C600C8
:1034400023A6C718B387070123A4B70013050000FC
:10345000678000001305F0FF67800000130101FD85
:10346000B7770180232C410103AA079C2320210365
:103470002326110203298A14232481022322910284
:10348000232E3101232A51012328610123267101B2
:103490002324810163000904130B0500938B0500AD
:1034A000930A10009309F0FF832449001384F4FF6A
:1034B0006342040293942400B304990063840B04D0
:1034C00083A74410638077051304F4FF9384C4FF3B
:1034D000E31634FF8320C1020324810283244102C6
:1034E000032901028329C101032A8101832A4101A1
:1034F000032B0101832BC100032C81001301010365
:10350000678000008327490083A644009387F7FF64
:10351000638E870423A20400E38806FA83278918B0
:1035200033978A00032C4900B377F70063920702B0
:10353000E78006000327490083278A146314870164
:10354000E304F9F8E38807F8138907006FF0DFF563
:103550008327C91883A544083377F700631C070045
:1035600013050B00E78006006FF0DFFC23228900C3
:103570006FF09FFA13850500E78006006FF09FFB50
:103580008397C500130101FE232C810023263101FE
:10359000232E1100232A91002328210193F687006E
:1035A0001384050093090500639A0610371700007D
:1035B0001307078083A64500B3E7E7002396F500CD
:1035C0006354D01803278402630A070C83A40900FC
:1035D0009396070123A00900139637018325C401A0
:1035E00093D60601634806169306100013060000E2
:1035F00013850900E70007009307F0FF630CF51837
:103600008356C400032784028325C40193F6460031
:10361000638E060083264400832704033305D540C8
:10362000638607008327C4033305F54013060500AE
:103630009306000013850900E70007009307F0FFD9
:10364000631EF51003A709008317C400630807165B
:103650009306D0016306D700930660016314D70C6C
:103660008326040137F7FFFF1307F77FB3F7E7005F
:103670002316F400232204002320D400832504030E
:1036800023A09900638C0500930704046386F5006A
:1036900013850900EF00C06723280402130500000A
:1036A0008320C101032481018324410103290101F5
:1036B0008329C100130101026780000003A90501ED
:1036C000E30E09FC83A405001397070113570701B4
:1036D0001377370023A02501B3842441930700000A
:1036E0006314070083A745012324F4006348900076
:1036F0006FF0DFFA3309A900E35290FA83274402FE
:103700008325C4019386040013060900138509006C
:10371000E7800700B384A440E34EA0FC8357C400B5
:103720001305F0FF93E707048320C1012316F4007B
:103730000324810183244101032901018329C1005C
:10374000130101026780000003A7C503E34CE0E614
:103750006FF0DFF4032504056FF05FEB8357C400BF
:1037600037F7FFFF1307F77FB3F7E700832604015E
:103770009397070193D707412316F40023220400EF
:103780002320D40013973701E35A07EE2328A4041B
:103790006FF0DFEE83A70900E38407E61307D0018B
:1037A0006388E702130760016384E7028357C4005C
:1037B00093E707042316F4006FF09FEE37F7FFFF3F
:1037C0001307F77F83260401B3F7E7006FF0DFFAF2
:1037D00023A09900130500006FF09FEC130101FE78
:1037E000232C8100232E110013040500630605001D
:1037F00083278503638007028397C50063960702CA
:103800008320C1010324810113050000130101027B
:10381000678000002326B100EF0000378325C10038
:103820008397C500E38E07FC130504000324810180
:103830008320C101130101026FF09FD4930505009D
:1038400063080500B777018003A5479C6FF01FF957
:10385000B777018003A5079CB73500809385C57DA8
:103860006F0090061305000067800000B7D5008048
:103870009385C5ED6F005005130101FEB747008029
:10388000232E1100232C8100232A910023282101BB
:1038900023263101232441012322510123206101E8
:1038A000032445009387C786232EF5021307C52EF0
:1038B000930730002324E52E2322F52E2320052E06
:1038C00093074000130905002326F4001306800027
:1038D0009305000023220406232004002322040071
:1038E0002324040023280400232A0400232C04009A
:1038F0001305C405EFC09FBE379B00808324890059
:10390000B79A0080379A0080B7990080130B8BB06C
:10391000938ACAB6130A4ABF9389C9C5B70701007B
:103920002320640323225403232444032326340343
:10393000232E84009387970023A6F40013068000AB
:103940009305000023A2040623A0040023A2040080
:1039500023A4040023A8040023AA040023AC040029
:103960001385C405EFC09FB70324C900B707020041
:1039700023A0640323A2540323A4440323A63403F3
:1039800023AE9400938727012326F4002322040604
:1039900023200400232204002324040023280400FD
:1039A000232A0400232C04001305C40513068000F9
:1039B00093050000EFC09FB28320C1012320640360
:1039C000232254032324440323263403232E840078
:1039D0000324810193071000232CF9028324410161
:1039E000032901018329C100032A8100832A4100A0
:1039F000032B010013010102678000001305000082
:103A000067800000130101FF232291001306800646
:103A10009384F5FFB384C402232021011389050098
:103A2000232481002326110093854407EF300050A2
:103A300013040500630005021305C50023200400DC
:103A4000232224012324A400138684069305000066
:103A5000EFC0DFA88320C100130504000324810008
:103A60008324410003290100130101016780000044
:103A7000130101FEB77701802328210103A9079CC8
:103A800023263101232E110083278903232C810053
:103A9000232A9100930905006386070A1309092E5A
:103AA0009304F0FF83274900032489009387F7FFDD
:103AB00063D807006F00000813048406638C970620
:103AC0000317C4009387F7FFE31807FEB707FFFF4C
:103AD00093871700232204062320040023220400D6
:103AE000232404002326F40023280400232A0400AE
:103AF000232C040013068000930500001305C40561
:103B0000EFC0DF9D23280402232A04022322040499
:103B1000232404048320C10113050400032481012C
:103B200083244101032901018329C10013010102FA
:103B30006780000003240900630C040013090400DB
:103B40006FF05FF613050900EFF01FD36FF01FF55C
:103B50009305400013850900EFF0DFEA2320A90058
:103B600013040500E31C05FC9307C00023A0F90023
:103B70006FF05FFAB777018003A5079CB7D5008087
:103B80009385C5ED6F004054832785036384070048
:103B9000678000006FF05FCE6780000067800000E4
:103BA0006780000067800000B777018003A5479C0D
:103BB000B7450080938545866F00C046B777018082
:103BC00003A5479CB74500809385C59F6F0080453E
:103BD000130101FE23263101B7690180232C8100E6
:103BE000232A91002328210123244101232E11009F
:103BF000138A05001309050093890943EF30D03B70
:103C000003A78900B71700001384F7FE8324470039
:103C10003304444193F4C4FF330494001354C400A8
:103C20001304F4FF1314C400634EF4009305000062
:103C300013050900EF40D05883A78900B387970088
:103C40006308F50213050900EF3050378320C101E6
:103C50000324810183244101032901018329C10037
:103C6000032A810013050000130101026780000090
:103C7000B305804013050900EF4090549307F0FF0F
:103C8000630AF504B77701809387C79D03A70700F0
:103C900083A68900B384844093E4140033048740EE
:103CA0001305090023A2960023A08700EF301031EE
:103CB0008320C101032481018324410103290101DF
:103CC0008329C100032A810013051000130101029A
:103CD000678000009305000013050900EF40504E77
:103CE00003A789009306F000B307E540E3DCF6F490
:103CF000B776018083A6869C93E717002322F700FE
:103D00003305D540B776018023AEA69C6FF09FF3B4
:103D1000638A0512130101FF2324810023229100ED
:103D2000138405009304050023261100EF30D028EA
:103D30000328C4FF130784FFB76501809377E8FF6A
:103D40003306F700938505438326460003A58500C7
:103D500093F6C6FF630AC51A2322D600137818000B
:103D60003305D6006310080A032384FF03284500A7
:103D70003765018033076740832887001305854333
:103D8000B3876700137818006380A8140323C70063
:103D900023A66800232413016304081E93E617007A
:103DA0002322D7002320F6009306F01F63E8F60ACB
:103DB00093F687FF9386860003A54500B386D5005A
:103DC00003A6060013D8570093071000B397070106
:103DD000B3E7A700138586FF2326A7002324C70087
:103DE00023A2F50023A0E6002326E6000324810099
:103DF0008320C100138504008324410013010101C5
:103E00006F30D01B0325450013751500631E050296
:103E100037650180B387D700130585438326860065
:103E200093E817003308F7006388A6160326C60038
:103E300023A6C6002324D600232217012320F8003E
:103E40006FF09FF66780000093E61700232ED4FEE4
:103E50002320F6009306F01FE3FCF6F493D69700B8
:103E600013064000636CD60E93D667001388960342
:103E7000138686031318380033880501832608004B
:103E8000130888FF6308D81203A646001376C6FFFE
:103E900063F6C70083A68600E318D8FE03A8C60011
:103EA000232607012324D700032481008320C10097
:103EB0002324E800138504008324410023A6E600A0
:103EC000130101016F30900F631608148325C6009B
:103ED00003268600B387F600032481002326B6005C
:103EE00023A4C50093E617008320C1002322D70036
:103EF000138504003307F700832441002320F700D3
:103F0000130101016F30900B13781800B387D700AD
:103F100063100802032584FF3307A7408326C700E8
:103F200003268700B387A7002326D60023A4C60054
:103F3000B776018013E6170083A6C69C2322C7002C
:103F400023A4E500E3E4D7EAB777018083A5879D42
:103F500013850400EFF0DFC76FF05FE9130640013F
:103F60006374D602130640056364D60693D6C70071
:103F70001388F6061386E606131838006FF0DFEF95
:103F8000B387D7006FF09FE91388C6051386B6057F
:103F9000131838006FF05FEE23AAE50023A8E500B0
:103FA0002326A7002324A700232217012320F8009B
:103FB0006FF0DFE303A5450013562640930710007A
:103FC0003396C7003366A60023A2C5006FF05FEDED
:103FD00013064015636CD60093D6F7001388860746
:103FE00013867607131838006FF01FE91306405543
:103FF000636CD60093D627011388D6071386C607AD
:10400000131838006FF05FE71308803F1306E007CE
:104010006FF09FE693E617002322D7002320F600D7
:104020006FF0DFDC130101FE23282101232631017B
:10403000232441012322510123206101232E110059
:10404000232C8100232A9100138B0500930A052E4F
:10405000130A0000930910001309F0FF83A44A001B
:1040600003A48A009384F4FF63C604028357C40048
:104070009384F4FF63FCF9008317E4001305040044
:1040800063862701E7000B00336AAA001304840645
:10409000E39E24FD83AA0A00E3920AFC8320C10167
:1040A0000324810183244101032901018329C100E3
:1040B000832A4100032B010013050A00032A810013
:1040C0001301010267800000130101FD2320210379
:1040D000232E3101232C4101232A51012328610180
:1040E0002326710123261102232481022322910217
:1040F000930A0500938B0500130B052E130A00008D
:10410000930910001309F0FF83244B0003248B0054
:104110009384F4FF63C804028357C4009384F4FFBC
:1041200063FEF9008317E4009305040013850A0079
:1041300063862701E7800B00336AAA001304840614
:10414000E39C24FD032B0B00E3100BFC8320C10236
:104150000324810283244102032901028329C1012E
:10416000832A4101032B0101832BC10013050A009F
:10417000032A8101130101036780000093064500B3
:10418000930700001305A5013788FFFF6F00C001EA
:10419000939717002390E6009397070193862600D4
:1041A00093D70701630ED50203D7060013761700D5
:1041B0006304060093E717001357170013F6270050
:1041C000B3650701E30606FC939717002390B6003A
:1041D000939707019386260093D70701E316D5FC32
:1041E0006780000093068501130700001305250072
:1041F0006F00C001131717002390F6001317070173
:104200009386E6FF135707016304D50483D706009E
:10421000139607011356064193971700635406003F
:10422000136717009397070193D7070113762700A9
:1042300093E51700E30006FC131717002390B60060
:10424000131707019386E6FF13570701E310D5FC08
:1042500067800000130101FE370E0100231D0100DD
:10426000231E0100938585019307C1011308810076
:10427000130EFEFF03D705009387E7FF9385E5FF45
:1042800063180702239F07FEE39607FF1306460005
:104290009306E10103D70700938727001306260042
:1042A000231FE6FEE398D7FE13010102678000009A
:1042B0003307A70283D8270003D30700B376C701CB
:1042C000B38616011357070193D806013307670019
:1042D00033071701935807012391D7002390E70074
:1042E000239F17FFE39807F96FF05FFA1307250183
:1042F000835705001305250063980700E31AE5FEC0
:10430000130500006780000013051000678000009F
:10431000130101FF232291008354250123248100EE
:104320002326110093C7F4FF139717011304050008
:1043300063160700EFF09FFB63180500B787FFFFC8
:10434000B3C4F400231994008320C1000324810026
:10435000832441001301010167800000130101FF64
:104360002324810003542501232611009347F4FFE1
:1043700013971701631A0700EFF05FF79307050023
:1043800013050000639407001355F4008320C10057
:104390000324810013010101678000008357250178
:1043A000130101FD2324810293D7F70023229102F8
:1043B0002326110223202103232E3101B307F040CD
:1043C0002390F50083572501378700001307F7FF77
:1043D000B377F7002391F50093040500130405015A
:1043E0006382E70493876500239205001305E5FFC8
:1043F000035704001304E4FF93872700239FE7FE7D
:10440000E31885FE239C05008320C102032481025A
:1044100083244102032901028329C10113010103FD
:1044200067800000035725011389450033F7E70033
:10443000631CF7022326B100EFF05FEB8325C10078
:104440006304050293876500239205001385C4FF6A
:10445000035704001304E4FF93872700239FE7FE1C
:10446000E31885FE6FF05FFA9389A501130929000F
:10447000231F09FEE39C29FF8320C102032481023C
:1044800083244102032901028329C101130101038D
:104490006780000083572501130101FB2324810459
:1044A00093C7F7FF232291042326110413971701C2
:1044B000930405001384050063160700EFF01FE363
:1044C000631205088357240193C7F7FF1397170159
:1044D000630407069305810013850400EFF01FECC9
:1044E0009305410213050400EFF05FEB8355810053
:1044F00003554102630CB5049307A1001307610241
:104500001306010283D6070093872700639A0608E3
:10451000835607001307270063940608E394C7FE39
:10452000130500008320C104032481048324410473
:10453000130101056780000013050400EFF01FDB85
:10454000E30A05F81305E0FF6FF0DFFD13351500F2
:104550000356A100835661023305A0401307A10052
:1045600093076102137525001305F5FF9305C10339
:104570009387270013072700631ED600E382B7FA4C
:104580000356070083D607001307270093872700E9
:10459000E306D6FEE3E8C6F83305A0406FF09FF8C7
:1045A00013051000E38005F81305F0FF6FF09FF787
:1045B000130101FF23261100EFF05FD38320C10018
:1045C000133515001301010167800000130101FE7E
:1045D000232C8100232A9100232E1100232821015E
:1045E00023263101938405001304050063C4050AE2
:1045F0009307F00013860500130545009306840118
:104600009305F00063D497029307050003D72700B2
:1046100093872700239FE7FEE39AD7FE231C04001D
:10462000130606FFE3C2C5FE93F4F400930770007F
:1046300063D89702130784019305240093070000B1
:10464000835607001307E7FF13968600B3E7C700FA
:104650002311F70093D78600E314B7FE938484FFF9
:10466000638A04009384F4FF13050400EFF09FB7FE
:10467000E39A04FE130500008320C1010324810195
:1046800083244101032901018329C100130101028F
:1046900067800000930710FF3309B04063DCF51218
:1046A0009305850193090000930645001306F00069
:1046B0000357840193870500B3E9E90003D7E7FFB7
:1046C0009387E7FF2391E700E39AD7FE23120400C4
:1046D000130909FFE34E26FD930700FF130710FFA0
:1046E000B38797401309000063C4E40A3309F90053
:1046F0009307700063D627059399090193D909415F
:10470000834784019305A401B3E9F9009399090152
:1047100093D909019307000003D60600938626006B
:104720001357860033E7E700931786009397070136
:10473000239FE6FE93D70701E390B6FE130989FF96
:10474000630C0906835784011309F9FF130504005C
:1047500093F71700B3E93701EFF05FA2E31409FE06
:104760009397090193D707416390070413950901B3
:10477000135505018320C1010324810183244101D4
:10478000032901018329C100130101026780000090
:1047900013F907FF330920413309F900930770002B
:1047A000E3D027FB6FF05FF5930910001395090123
:1047B000135505016FF01FFC13850900639809006C
:1047C00013150501135505016FF01FEB13051000BC
:1047D0006FF01FFF930790FF93090000E3D4F5F6F5
:1047E000930644006FF0DFF183574500130101FF8A
:1047F000232291002326110023248100232021015C
:1048000093040500639C070C035765001304000024
:104810009317070193D7074163C4070A9306A501BD
:104820001306000A63180702938764006F00800074
:1048300003D7070093872700239EE7FEE39AF6FE3F
:10484000239C040013040401630CC40603D7640012
:10485000E30C07FC937707F063900704138584014A
:104860009385240093070000130705008356070073
:104870001307E7FF13968600B3E7C7002311F7007D
:1048800093D78600E394E5FE03D764001304840005
:10489000937707F0E38807FC1309000A6F004001D3
:1048A00013041400EFF01F94634C890003D76400D5
:1048B000131707011357074113850400E35207FE3E
:1048C0008320C100130504000324810083244100D8
:1048D00003290100130101016780000013F707F0AD
:1048E00013040000631007041309F0F66F00400181
:1048F0001304F4FFEFF09F88E30424FD83D7440002
:1049000013850400E39607FE8320C100130504000D
:1049100003248100832441000329010013010101C4
:1049200067800000930645009305A501130700006A
:104930006F00800083D7060013D687003367C70057
:10494000939787002390E60013970701938626002C
:1049500013570701E390B6FE83D74400130480FF8A
:104960006FF09FF8130101FE232C8100232A910090
:10497000232821012326310123244101232251012F
:104980001389060093840700232E110013040500E9
:1049900093890500130A0600930A0700EFF0DFE48D
:1049A000930700093309A94063DCA716B787000005
:1049B0009387E7FF63DA271F63840A1C03A544007B
:1049C00083A70400630AF5061387A40193874403B1
:1049D00013072700231F07FEE31CF7FE930780033E
:1049E000630CF53263D0A71693070004630CF52E11
:1049F000930710076318F534B78700409387F7FFD4
:104A00001307A00023AAF400B787FFFF23A4E40044
:104A1000239CF40023A6E4009307A000378700003E
:104A20009387870093971700B387F4002395E700D7
:104A300023A0A4006358201B83A5840083D74401CE
:104A40001308F008139615003306C4000357060038
:104A5000B376F700634AA8021308B0006346B802B1
:104A6000930706009305840103D72700630407001A
:104A700093E616002391070093872700E396F5FE3F
:104A80000357060083D7440193C7F7FFB3F7E70046
:104A90002310F60083D7640133F7D70063000704BF
:104AA0006384D71A13862403930684019384C40174
:104AB000130700008357060083D506009386E6FFA0
:104AC0001306E6FFB387B700B387E70013D70701E4
:104AD0002391F60013771700E31E96FC6358201904
:104AE00083574400639E0712B7870000231C04000D
:104AF0009387E7FF63C82709231124018320C1019D
:104B00000324810183244101032901018329C10078
:104B1000032A8100832A41001301010267800000FB
:104B20006354090E930700F7635CF90893072400A8
:104B30001304A40193872700239F07FEE39C87FEAD
:104B40006FF0DFFB930780016308F51693075003AE
:104B5000631AF51E37170000B707000493066000BC
:104B60009387F77F1307078023AAF40023A4D400B8
:104B7000239CE40023A6D400930760006FF05FEA53
:104B8000231C0400B787FFFF93C7F7FF2311F4002E
:104B900093074400130484012390070093872700A0
:104BA000E31CF4FE6FF09FF5930724001304A401A7
:104BB00093872700239F07FEE39C87FE6FF01FF477
:104BC0009305090013050400EFF05FA063040500DE
:104BD00093091000638C0A0C03A5440083A704000A
:104BE000E314F5DE930700096304F50A8357840193
:104BF0001305040093F71700B3E9F900EFF00FD89D
:104C000003A544006FF05FE3E3800AEE03A54400D0
:104C100083A70400E31AF5DAE34020E36FF09FFC7A
:104C200013050400EFF08FD5B787000013091900B2
:104C3000231C04009387E7FFE3C627F5E35E09EA38
:104C4000231104006FF09FEB6394090C83A7C40049
:104C500003D7840193971700B307F40083D70700A5
:104C6000B3F7E700E39007E4E34C20E7930700097C
:104C70006306F50013050400EFF0CFD68357440018
:104C8000E39007FA231C0400E34C09FA6FF0DFE617
:104C900003A6840083D74401131616003306C4000C
:104CA00003570600B3F6E7006FF01FDE231C040075
:104CB000231104006FF09FE4B70780009387F70F7C
:104CC0001307400023AAF4009307001023A4E40074
:104CD000239CF40023A6E400930740001307001070
:104CE0006FF01FD49307700023A4F400B70701806E
:104CF0009387F7FF23AAF40093071000239CF40086
:104D00009307600023A6F400130710006FF05FD133
:104D1000E30A0AD86FF09FDCB70780009387F70F8C
:104D20001307600023AAF4009307001023A4E400F3
:104D3000239CF40023A6E4009307600013070010EF
:104D40006FF01FCE9307C00023A4F400B7070180C3
:104D50009387F7FF23AAF40093071000239CF40025
:104D60009307B00023A6F400130710006FF05FCB89
:104D7000130101FD23229102232E310193840500AA
:104D80008359250023261102232481022320210395
:104D9000232C410113090600232A51012328610114
:104DA0002326710123248101232291012320A101C3
:104DB000130A0500EFF05FA303D424009307050056
:104DC00013850400B389F940930A4903EFF0DFA18A
:104DD0003304A4401307E90493870A00938727004C
:104DE000239F07FEE39CE7FE634A3409930B4A00C6
:104DF000138B44009389F9FF930CAA01138C2400B0
:104E000013070B0093870B0003D607008356070098
:104E10009387270013072700631AD60AE39697FFA4
:104E200013068A0113878401930600008357070045
:104E3000835506001307E7FFB387D740B387B74012
:104E400093D607012311F70093F616001306E6FF29
:104E5000E31EECFC130D100013850A00EFF08FB871
:104E60008357C9041304F4FF13850400336DFD0058
:104E70002316A905EFF00FB7E31434F993060400E5
:104E8000032481028320C1028329C101032A8101F5
:104E9000832A4101032B0101832BC100032C8100D4
:104EA000832C4100032D01009307090013850400A2
:104EB00003290102832441021307000013060000A6
:104EC00093050000130101036FF0DFA9130D00002B
:104ED000E3E4C6F86FF0DFF40357050083572500BD
:104EE0006306070037870000B3E7E7002399F50062
:104EF00003572500B78700009387F7FF6304F70285
:104F000093076500938505011305850103D7070005
:104F1000938727009385E5FF2391E500E398A7FE9B
:104F200067800000930765001305A50103D70700FC
:104F300093872700631A0702E39AA7FE13872501C8
:104F40009387050093872700239F07FEE31CF7FE46
:104F500083D72501378700001307F7FFB3E7E70082
:104F60002399F500678000001387050193870500EA
:104F700093872700239F07FEE31CF7FEB7C7FF7F39
:104F800023A8F50067800000130101F723286107BB
:104F9000035B2501B78700009387F7FF232C4107A8
:104FA00033FA6701131A0A01232481082322910886
:104FB00023202109232E310723261108232A5107F4
:104FC000232671072324810723229107135A0A01FC
:104FD0009304050013890500130406009389060055
:104FE0006312FA10EFF08FB0631A0528835A290173
:104FF000B3775A016382472B13850400EFF04FDB30
:10500000630E052EB755018093850513130509001E
:10501000EFF04FC863060536835A2901B7870000B1
:105020009387F7FFB3FA5701939A0A0193DA0A01BB
:105030006394FA2C13050900EFF08FD76310053243
:1050400083D72401B3F7FA006398570B1385040044
:10505000EFF00FD66318050013050900EFF04FD5E8
:10506000630C050813850400EFF04FAF93040500AF
:1050700013050900EFF08FAEB384A440B334900061
:105080009394F40023199400130724019307040058
:1050900093872700239F07FEE31CF7FE8357240115
:1050A000378700001307F7FFB3E7E7002319F40081
:1050B0008320C108032481088324410803290108AF
:1050C0008329C107032A8107832A4107032B01078C
:1050D000832BC106032C8106832C41061301010991
:1050E0006780000083DA250133F7570113170701A2
:1050F00013570701630AF704138504009305C100E1
:10510000EFF0CFA91305090093058102EFF00FA975
:105110008354E1000359A102639C04049307010135
:10512000930641026388D72003D70700938727009F
:10513000E30A07FE1305C100EFF00FEB0357A102CE
:10514000B304A0406F00000313850500EFF00F9A31
:10515000E30605EC130749018357090013092900E9
:1051600013042400231FF4FEE318E9FE6FF05FF43C
:1051700013070900930A09009307C102930601046B
:10518000631207026382F61C03D707009387270088
:10519000E30A07FE13058102EFF00FE50357A102B2
:1051A000B30AA94083578102138C8903239BE90228
:1051B000239AF9021387E90493070C002390070050
:1051C00093872700E31CF7FE138AC904930B0000A2
:1051D00013094102930C0101130B610403550900EB
:1051E0001309E9FF6318050C03D7C90493070A00E4
:1051F000B3EBEB0003D7E7FF9387E7FF2391E700CB
:10520000E39A87FF239C0902E31A99FD1387490358
:105210009307810293052104035607009387270013
:1052200013072700239FC7FEE398F5FEB7C6FFFFCD
:10523000B38454019386260093850B0013058102E5
:105240009387090013070004B386D40013060000F7
:10525000EFF04FF1035781028357C100930504001B
:1052600013058102B387E740B337F000B307F0407E
:105270002314F102EFF05FC66FF09FE31387440140
:1052800083D704009384240013042400231FF4FE16
:10529000E398E4FE6FF0DFE113050900EFF00F85FE
:1052A000E31A05EA13850400EFF08FB0E30805D692
:1052B0006FF05FD51306410493058102EFE09FF97B
:1052C00093050A00130600001307C10503D8050063
:1052D000835707009385E5FF1307E7FFB3870701AF
:1052E000B387C70013D607012391F5001376160084
:1052F000E31E67FD6FF05FEF03DB2401B78700005B
:105300009387F7FF33FB6701131B0B01135B0B0143
:10531000E314FBDE13850400EFF08FA9E31405D43A
:105320008357290193C7F7FF13971701E31607DC8B
:105330006FF09FD29307440113042400231F04FE3F
:10534000E39C87FE6FF0DFD693074401130424002B
:10535000231F04FEE31CF4FE6FF09FD5B7550180B8
:105360009385051313850400EFF0CF92630A0500BF
:1053700083D72401B3F7FA00E38E57F96FF05FFA91
:10538000130704019307040093872700239F07FE58
:10539000E39CE7FEB7C7FF7F2328F4006FF05FD1DF
:1053A00083572501130101F52324810A93C7F7FFD1
:1053B0002322910A2320210B232E31092326110AAF
:1053C000232C4109232A5109232861092326710925
:1053D00023248109232291092320A109232EB10727
:1053E000139717011309050093890500130406009C
:1053F0009384060063160700EFE05FEF631805383B
:1054000083D7290193C7F7FF13971701630E070886
:10541000375A018093050A1313050900EFF08F87AF
:1054200063040510035A290103D72901B787000037
:105430009387F7FF33FA4701B3FAE700631AFA08D4
:1054400013050900EFF0CF966308051063984A0131
:1054500013850900EFF0CF956310050E9307440103
:1054600013042400231F04FEE31CF4FE8320C10A5E
:105470000324810A8324410A0329010A8329C109DB
:10548000032A8109832A4109032B0109832BC108BF
:10549000032C8108832C4108032D0108832DC107AB
:1054A0001301010B6780000013850900EFE01FE482
:1054B000E30005F61387490183D709009389290082
:1054C00013042400231FF4FEE398E9FE6FF01FFA93
:1054D0006386FA08130509009305C101EFE01FEC8C
:1054E0009305810313850900EFE05FEB835BA10364
:1054F0000359E10163920B0C9307C103930D01055E
:10550000638EFD3403D7070093872700E30A07FE65
:1055100013058103EFF04FADB307A0400356E1013F
:105520002326F1006F00C00993050A1313850900B3
:10553000EFE05FF6E31805EE13070401930704009C
:1055400093872700239F07FEE39CE7FEB7C7FF7FF3
:105550002328F4006FF09FF1E39E4AF713850900BA
:10556000EFF00F85E30805F613050900EFE01FDFF4
:105570009304050013850900EFE05FDEB387A440C4
:10558000B337F0009397F7002319F40013072401B1
:105590009307040093872700239F07FEE39CE7FE01
:1055A00083572401378700001307F7FFB3E7E700AD
:1055B0002319F4006FF09FEB2326710113060900F5
:1055C000232421019307010293064103631206027B
:1055D0006380F62A03D7070093872700E30A07FEB4
:1055E0001305C101EFF04FA0B307A9402324F10038
:1055F00003278103138D840393070D0023AAE4027C
:105600001389E40493872700239F07FEE31CF9FE18
:1056100013058103EFE09FB6035C2102370A010006
:10562000930D0105931A0C01B38A8A41130BA10350
:10563000130AFAFF930CE106930961058357C1032E
:105640000357E103930B0A0093970701B387E70021
:1056500063E8FA00B3D78703939B070193DB0B0141
:10566000130641059305C10113850B00EFE09FBEB2
:105670001307C1039307810583D50700035607006D
:1056800093872700130727006390C512E39697FFBF
:10569000930700009305C10613860D00035706000B
:1056A00003D805001306E6FF3307F7403307074129
:1056B000935707012311E60093F717009385E5FF41
:1056C000E31E66FD23107D019307C10303D7270066
:1056D00093872700239FE7FEE39AB7FF231801046F
:1056E000130D2D00E31CA9F5930500009307C103DA
:1056F0009306210503D7070093872700B3E5E5004C
:10570000E39AD7FE9397050193D707416384070077
:10571000930510009395050193D505011387440364
:105720009307810303560700938727001307270079
:10573000239FC7FEE398F6FE8327C100032781005D
:10574000B74600009386F6FFB38BE740130581034D
:105750009387040013070004B386DB0013060000E0
:10576000EFF04FA0035781038357C1019305040055
:1057700013058103B387E740B337F000B307F04068
:10578000231CF102EFF04FF56FF05FCE13074901D4
:10579000835709001309290013042400231FF4FE72
:1057A000E318E9FE6FF09FCCE374B6EE9387FBFF3E
:1057B0009398070193D808019307000093054103CC
:1057C0001306C1060357060003D805001306E6FFBB
:1057D0003307F74033070741935707012311E600CA
:1057E00093F717009385E5FFE31E36FD1307C1030A
:1057F0009307810583D50700035607009387270089
:10580000130727006398C500E39697FF938B080062
:105810006FF01FE8E37CB6FE9387EBFF939B0701D5
:1058200093DB0B0113060000930541031307C10628
:105830008357070003D805001307E7FFB387C74066
:10584000B387074113D607012311F700137616001B
:105850009385E5FFE31E37FD6FF09FE39307440157
:1058600013042400231F04FEE39C87FE6FF01FC077
:105870000357C101835781036304F7003786000093
:105880002319C400130724019307040093872700FA
:10589000239F07FEE31CF7FE835724013787000090
:1058A0001307F7FFB3E7E7002319F4006FF01FBCFD
:1058B000130101FD23248102232611021384050014
:1058C000930741001307E10193872700239F07FEF9
:1058D000E39CE7FE0356E5009317060193D70741C3
:1058E00063CA0706B78700009387F7FF23120100FA
:1058F0003376F600630CF6069307E5002313C10028
:105900001307A10083D6E7FF9387E7FF130727005C
:10591000231FD7FEE318F5FE6312060223140100CD
:105920009305040013054100EFF00FDB8320C10253
:105930000324810213010103678000009307100014
:105940009305F0FF130541002314F100EFE01FC899
:105950006FF01FFD9307F0FF2312F100B7870000DF
:105960009387F7FF3376F600E318F6F89307050000
:105970009306E50003D7070093872700631C0704FD
:10598000E39AD7FE13074401930704009387270087
:10599000239F07FEE31CF7FE13072401930704006F
:1059A00093872700239F07FEE31CF7FE83572401FC
:1059B000378700001307F7FFB3E7E7002319F40068
:1059C0008317E500E3D407F613050400EFE05F94C6
:1059D0006FF0DFF513070401930704009387270096
:1059E000239F07FEE31CF7FEB7C7FF7F2328F400C1
:1059F0006FF0DFF383A8C500130101E183AE05005A
:105A000003AE450003A38500232E1103832505045F
:105A10009308F0FF23201117930800092324811E07
:105A2000232C411D2326111E2322911E2320211FDA
:105A3000232E311D232A511D2328611D2326711D6C
:105A40002324811D2322911D2320A11D232EB11B60
:105A50002328D103232AC103232C610223221117F7
:105A60002324C1002328D100232AE100232E010191
:105A7000130A050013840700638005020327450409
:105A800093071000B397E70023A2E50023A4F500D5
:105A9000EF10905D23200A04930901069385090005
:105AA00013050103EFF0DFE013850900EFE01F8B22
:105AB000032781003335A0002320A4009307300082
:105AC000E302F714930740012326F100E31E076069
:105AD000835721070327411693C7F7FF232CE100C3
:105AE000139717016318070013850900EFE01F8063
:105AF000E3160540930700092322F1161307C10797
:105B0000938709001306410783D607009387270070
:105B100013072700231FD7FEE398C7FE0356E108AB
:105B2000232201009317060193D7074163DE070084
:105B300013161601B7070100135616019387F7FFD6
:105B40002317C1082322F100B75A018093870A1353
:105B5000938B4701930600009307810913870B007D
:105B6000930DC10A6F0080008356070093872700BA
:105B7000239FD7FE13072700E398B7FF630206169B
:105B8000B78700009387F7FFE30CF6588317C10827
:105B9000E3DE075C9305C10713850B00EFE09F8FE1
:105BA000630C0514E34C050C8357E108E392076688
:105BB0008317C108930400001309011663C8070284
:105BC000B757018093870713138487111306C10702
:105BD000930609009305060013050400EFF0CFBA01
:105BE0008317C1089384F4FFE3D207FE1304010D69
:105BF000130B810E130704009307C1071306010955
:105C000083D607009387270013072700231FD7FE9B
:105C1000E398C7FE930600009307810913870B00E2
:105C20006F0080008356070093872700239FD7FECD
:105C300013072700E398B7FFB757018013870713AF
:105C40009387071337FDFFFF930C8702930DC7124D
:105C5000138C87116F00C000938D4D01938C4C0104
:105C60009305040013850B00EFE0DF829307050026
:105C70009305040013850D006356F004EFE09F8147
:105C8000930705009306090013060400930504001A
:105C900013850C0063C00702EFF00FAF13068109F4
:105CA000930609009305060013850C00EFF0CFADB5
:105CB000B384A4019357FD01338DA701135D1D40EB
:105CC000E39C8CF9130681099306090093850B0068
:105CD00013050600EFF0CFEC930C41126F000003A8
:105CE0009307C1079306E10803D7070093872700AE
:105CF000E31207EAE39AD7FE93040000930C4112E3
:105D0000130901161304010D130B810E93050400F2
:105D100013058109EFE08FE8130781099307040059
:105D200083D607009387270013072700231FD7FE7A
:105D3000E39867FF930504001305C1072318010AC0
:105D4000EFE0CFE59307C1070357040013042400D5
:105D500093872700239FE7FEE31864FF130581095B
:105D6000130609009305C107231A0108EFF04F80BD
:105D70000355C11A6314051C130D41091304E107EF
:105D8000930B610B93850A131305C107EFE08FF0A6
:105D90006306051A1307000093060D006F00C0018B
:105DA000131717002390F600131707019386E6FFD9
:105DB000135707016384860483D7060013960701EF
:105DC0001356064193971700635406001367170094
:105DD0009397070193D707011376270093E51700E0
:105DE000E30006FC131717002390B60013170701F2
:105DF0009386E6FF13570701E39086FC1307410BD8
:105E00009307C10783D6070093872700130727004E
:105E1000231FD7FEE398A7FF2316010C13070000EA
:105E20009306C10C6F00C001131717002390F600F2
:105E3000131707019386E6FF13570701638476055E
:105E400083D7060013960701135606419397170050
:105E500063540600136717009397070193D7070150
:105E60001376270093E51700E30006FC13171700CD
:105E70002390B600131707019386E6FF1357070117
:105E8000E39076FD130700009306C10C6F00C0017C
:105E9000131717002390F600131707019386E6FFE8
:105EA000135707016384760583D70600139607010D
:105EB00013560641939717006354060013671700A3
:105EC0009397070193D707011376270093E51700EF
:105ED000E30006FC131717002390B6001317070101
:105EE0009386E6FF13570701E39076FD1306000043
:105EF00093060D001307C10C83D5060083570700D6
:105F00009386E6FF1307E7FFB387B700B387C700A1
:105F100013D607012391F60013761600E31E77FDD2
:105F200013058109130609009305C107EFE05FE43B
:105F30000355C11A9384F4FFE30605E48327410067
:105F40008326810013073000B337F000B307F04019
:105F500093F7D700938707022302F1128327C1002A
:105F60006394E600B38797001307A0021384070029
:105F70006354F7001304A0021307A0006308E54C64
:105F8000130505031307E002A302A1122303E11284
:105F9000E3CE071E930771122322F100930B00003A
:105FA000130D410B130B4109130CE107930D610B0A
:105FB0001306000093050B006F00C00113161600B6
:105FC0002390F500131606019385E5FF135606018D
:105FD0006384850583D70500139507011355054193
:105FE00093971700635405001366160093970701F3
:105FF00093D707011375260093E81700E30005FC0B
:106000001316160023901501131606019385E5FF5C
:1060100013560601E39085FD13060D009307C10793
:1060200083D507009387270013062600231FB6FE9B
:10603000E39867FF2316010C130600009305C10CBB
:106040006F00C001131616002390F5001316060109
:106050009385E5FF135606016384B50583D70500D4
:1060600013950701135505419397170063540500D5
:10607000136616009397070193D70701137526003F
:1060800093E81700E30005FC131616002390150192
:10609000131606019385E5FF13560601E390B5FD3F
:1060A000130600009305C10C6F00C0011316160003
:1060B0002390F500131606019385E5FF135606019C
:1060C0006384B50583D70500139507011355054172
:1060D0009397170063540500136616009397070102
:1060E00093D707011375260093E81700E30005FC1A
:1060F0001316160023901501131606019385E5FF6C
:1061000013560601E390B5FD1305000093050B003F
:106110001306C10C83D80500835706009385E5FF5D
:106120001306E6FFB3871701B387A70013D507014E
:106130002391F50013751500E31EB6FD1306090043
:106140009305C10713058109EFE09FC28357C11A68
:106150000327410093850703330677012300B60028
:10616000938B1B00E35674E51345F4FF1355F5417B
:106170003375A4001309150033092701B30BA700D9
:1061800013074000635EF70413075000E386E7023D
:106190008347E9FF1307E9FF93F7F707634A047A98
:1061A0009306E0021306800393050003638ED70075
:1061B0006358F67A8347F7FF2300B7001307F7FF0A
:1061C00093F7F7076FF09FFE8347F7FF930680036F
:1061D000E3FAF6029307100393841400A30FF7FE6B
:1061E000B7550180138604009385C51213850B00F3
:1061F000EF20D00983572107032781012328911617
:1062000093C7F7FF2322E11613971701631E0700B8
:1062100013850900EFE0CFB963100522138509004B
:10622000EFE0CF8C631A052083264101034741121A
:106230009387140023A0F60093870C00630A0702DB
:106240009306E002630CD71C03C71700938717005F
:10625000E31A07FE9306500463E6FC006F0040015A
:106260006388970103C7F7FF9387F7FFE31AD7FE09
:106270002380070093870C00930600021306D002C8
:1062800003C707006304D7006316C700938717008E
:106290006FF01FFF13840C006F00C00003C70700DE
:1062A000138406002300E40093061400938717006C
:1062B000E31607FE83268100930720000347F4FFBF
:1062C0006386F6128327C1009386070063D4970084
:1062D00093860400930700036316F702B307944103
:1062E00063D2F602130600036F00800063DCE60051
:1062F0008347E4FFA30F04FE1304F4FF3307944124
:10630000E386C7FE03278100930730006302F70A84
:106310008327010123220A049386970093077001C3
:1063200063F2D70C130710009307400093971700F0
:10633000138647019305070013071700E3F8C6FE0D
:106340002322BA0413050A00EF1080472320AA0471
:1063500093850C0093040500EF20D0108327C10122
:1063600063880700330494413384840023A08700AA
:106370008320C11E0324811E0329011E8329C11D00
:10638000032A811D832A411D032B011D832BC11C60
:10639000032C811C832C411C032D011C832DC11B4C
:1063A000138504008324411E1301011F6780000030
:1063B0008327C100B384970063CE04528327410131
:1063C0000327010183A70700B307F7002328F10083
:1063D0008327010123220A04938637009307700163
:1063E000E3E2D7F4930500006FF0DFF593070003B5
:1063F000E310F7F2B307944193061000E3C4F6EEFE
:106400006FF01FF1032C0101232681019307A002E5
:1064100063D087ED2326F1006FF08FEB03C70700F1
:10642000E30A07E203C7170093871700A38FE7FE6D
:10643000E31A07FE6FF01FE203274101B7270000B0
:106440009387F7702320F7006FF0DFE21307100344
:10645000A302E1121307E0022303E1129384140064
:10646000635EF02A93070003A303F11293078112DE
:106470001304F4FF2322F1006FF05FB2130D410B00
:1064800013070D009307C1071306010983D6070000
:106490009387270013072700231FD7FEE398C7FE23
:1064A000B74700009387E7082313F10CB757018023
:1064B00093870713138B870CB78700009387F7FF29
:1064C0002322F102B7C7FFFF93872700130E0001B5
:1064D00093040000930C4112130901161304010DDB
:1064E000130CA10A2324F102930609001306810963
:1064F00093050D0013050B002320C103EFE05FEAB5
:10650000032E01021307C1049307810983D60700F4
:106510009387270013072700231FD7FEE398B7FFB1
:10652000832741028355E10533F6F5008327810275
:106530003305F600635AA03C130600093306A64053
:10654000130704009307C10483D60700938727002D
:1065500013072700231FD7FEE39837FF6358C006B1
:106560009307F0001307040063DCC702130606FF5D
:106570009356460013871600131717003307E400DD
:106580009307040093872700239F07FEE39CE7FE01
:10659000130600083306A640939646003306D640FD
:1065A000B757018093870713131616003386C70069
:1065B0008356062383570700B3F7D7002310F7004D
:1065C0009395050193D5054163C20516930781098B
:1065D0001307040003D6070083560700938727009C
:1065E000130727006314D602E316FCFE13070D0001
:1065F0009307810983D60700938727001307270095
:10660000231FD7FEE398B7FFB384C401B7570180B7
:1066100093870713130B4B019387C712135E1E005A
:10662000E314FBEC8357610C0357E1081306810C5C
:10663000B387E70037C7FFFF130727F7B387E700E4
:106640002313F10C1307C10793070D0083D607002E
:106650009387270013072700231FD7FEE398C7FE61
:1066600013070000930781096F00800003D70B0018
:1066700093872700239FE7FE938B2B00E398B7FFB8
:10668000B75701801387071393870713B71D0000BF
:10669000130B8702938B87116F00000193DD1D00A0
:1066A00063047B2B130B4B0193050D0013850B002B
:1066B000EFD05FDE1307050093050D0013050B00F7
:1066C0006344E028EFD01FDDE34AA0FC93060900F5
:1066D00013060D0093050D0013050B00EFE05FCCD2
:1066E00013068109930609009305060013050B00A4
:1066F000EFE09F89B384B4016FF05FFA930C41120D
:10670000B75501809385851013850C00B7240000D0
:10671000EF20C0379384F4706FF0DFAD930B7112EC
:10672000E39007AC232271016FF05F879307C104E8
:10673000130704006F00C0009306E105E388F6E844
:1067400003D6070083560700938727001307270007
:10675000E304D6FE8357210E03274102B377F700E7
:106760006394E702130504002320C103EFD01FB890
:10677000032E0102E31C05E413050400EFD05FE3E0
:10678000032E0102E31405E49305C10E13850B00EB
:106790002320C103EFD09FC093058110130504008F
:1067A000EFD0DFBF0356C10E0355A110835EE10E8B
:1067B0001346F6FF13160601135606012316C10EE3
:1067C000B385AE40032E010293060500635EB0065A
:1067D00093860C001307811093070112835507005D
:1067E0001307270093862600239FB6FEE318F7FEC3
:1067F000231E0112130781109306C10E6F00800043
:1068000003D6060013072700231FC7FE9386260022
:10681000E318F7FE231001121307C10E93870C0033
:10682000130FC11383D60700938727001307270090
:10683000231FD7FEE398E7FF8356A110B305D54188
:1068400023120110138506006380052E2326D10232
:106850009307F0F663CEF5061305C10E2320C1039E
:10686000EFD0DFD6032E01028326C1029305050077
:1068700093070112130641100355C10E03578110EF
:106880006300E5301305000003D70700835E0600B0
:106890009387E7FF3307A7403307D7411355070115
:1068A0002391E7001307A110137515001306E6FFE7
:1068B000E39CE7FC1306100093070900130700048C
:1068C000130581102320C103EFE0CF89032E0102BD
:1068D00093050400130581102320C103EFE0CFDFEF
:1068E000032E01026FF09FCE83270101138CF7FF67
:1068F0006FF09FB1832741012302011213840C0022
:1069000023A007006FF0DFAC930704001307410ECC
:1069100093872700239F07FEE39CE7FE6FF05FCA83
:1069200083274100930C4112638A0706B755018003
:106930009385051113850C00B7240000EF20001586
:106940009384F4706FF01F8B130B810E6FF00FBCEC
:1069500093071003230FF9FE938414006FF05F88F0
:10696000938717002300F7006FF09F87930C411265
:10697000B75501809385851213850C00B72400005C
:10698000EF20C0109384F4706FF0DF868357C11A34
:10699000930B6112130971126FF08FFEB7550180CE
:1069A0009385C51113850C00B7240000EF20000E5D
:1069B0009384F4706FF01F84930581091305C10758
:1069C000EFE08FD193850A1313058109EFD09FACB7
:1069D000631005FCE34604808347E9FF138727FD26
:1069E000133717001347F7FF3387EB000347070000
:1069F00013771700630607FE1307E9FF93F7F707FE
:106A00006FF00FFA93871700A30FF7FE6FF04FFD9B
:106A10001304010D930504001305C107374D000051
:106A2000EFD0DF9793040000130B810E1309C10C04
:106A3000930C210D130DEDFF130C50FD8357810EA8
:106A400093F777006398070C1307410B9307040033
:106A500083D607009387270013072700231FD7FE3D
:106A6000E39867FF1305410B2316010CEFD00FF1DC
:106A70001305410BEFD08FF01306000093060900B9
:106A800013070B0083D50600835707009386E6FFA4
:106A90001307E7FFB387B700B387C70013D6070113
:106AA0002391F60013761600E31E97FD8357610BC2
:106AB0000357810B93873700231BF10A63000702FA
:106AC0001305410BEFD08FEB8357610B0357810BFD
:106AD00093871700231BF10AE31407FE8357C10CA9
:106AE000639A07028357610B6366FD021307040074
:106AF0009307410B83D607009387270013072700CE
:106B0000231FD7FEE39827FF2314010E9384F4FF7D
:106B1000E39684F39305C10713050400EFE0CFBBB0
:106B2000130901166FF00F8D1307C1109307010FA2
:106B300083DE07000356070093872700130727000B
:106B40006398CE0213066110E394C7FE0357C10E8B
:106B5000835781106302F706930704001307410E61
:106B600093872700239F07FEE39CE7FE6FF01FA695
:106B70006366D60D93070112130641106FF0DFCF45
:106B800013050000130FE10E83DE07000357060014
:106B90009387E7FF1306E6FF3307D7013307A70004
:106BA000135507012391E70013751500E31EE6FD59
:106BB000130600006FF05FD013870600639206068D
:106BC0008317E11063CE0704930601126F000002E1
:106BD0002390F60013171700131707019386E6FF9B
:106BE0009307A11013570701E384F6CE83D706005D
:106BF0001396070113560641939717006354060036
:106C0000136717009397070193D70701137627009F
:106C100093E51700E30E06FA2390B6006FF09FFB92
:106C20001306C11093070112631207086382C70895
:106C300003570600130626006FF01FFF13860C0093
:106C4000130781109307011203550700130727004C
:106C500013062600231FA6FEE318F7FE231E0112CB
:106C6000130581101307C10E13064110835E070040
:106C70001307270013052500231FD5FFE318C7FEC0
:106C8000231001121305C10E13870C00130FC1133B
:106C9000835E07001307270013052500231FD5FF78
:106CA000E318E7FF231201106FF01FBD13851600D4
:106CB0002315A1106FF0DFC1032785008327C500CE
:106CC0000326050083264500130101FC130501007E
:106CD000930541012324E1002326F100232E110214
:106CE0002320C1002322D100EFE09FBC8357610223
:106CF0001305000093C7F7FF13971701631A0700E6
:106D000013054101EFD08FDE133515001305150073
:106D10008320C10313010104678000001305050FE0
:106D20006780000037750180130585926780000039
:106D3000377501801305859267800000130101F902
:106D400023248106138405008395E5002322910600
:106D50002320210723261106930406001389060029
:106D600063CA050413068100EF60404F63440504C5
:106D70000327C100B7F700008320C106B3F7E7007F
:106D800037E7FFFFB387E7000324810693B71700B7
:106D90002320F9009307004023A0F40037150000DA
:106DA0008324410603290106130505801301010709
:106DB000678000008357C4002320090093F7070869
:106DC000638407028320C10603248106930700041D
:106DD00023A0F400032901068324410613050000C3
:106DE00013010107678000008320C1060324810688
:106DF0009307004023A0F4000329010683244106E1
:106E000013050000130101076780000083D7C50048
:106E1000130101FE232C8100232E1100232A91004F
:106E20002328210193F727001384050063880702B4
:106E30009387350423A0F50023A8F50093071000DD
:106E400023AAF5008320C101032481018324410189
:106E50000329010113010102678000009306C100AC
:106E60001306810093040500EFF05FED8325810098
:106E70001309050013850400EF00400B8317C400BD
:106E800063080504374700801307C78623AEE40272
:106E9000032781008326C10093E707082316F40027
:106EA0002320A4002328A400232AE40063980604D6
:106EB000B3E727018320C1012316F40003248101D5
:106EC00083244101032901011301010267800000AD
:106ED00013F70720E31807F693F7C7FF93E7270098
:106EE000130734042316F400930710002320E40052
:106EF0002328E400232AF4006FF0DFF48315E40074
:106F000013850400EF609006631605008317C40024
:106F10006FF01FFA0357C4001377C7FF13671700FA
:106F20009317070193D707416FF09FF8130101FDF5
:106F3000232E3101232611022324810223229102D0
:106F400023202103232C4101232A510123286101FD
:106F50002326710123248101232291019387B50007
:106F600013076001930905006366F70693070001A4
:106F700063E6B71EEF0050049304000113062000DF
:106F8000930780013769018013090943B307F900AA
:106F900003A44700138787FF630AE4208327440084
:106FA0008326C4000326840093F7C7FFB307F400C9
:106FB00003A747002326D60023A4C60013671700A3
:106FC0001385090023A2E700EF00407F130584002A
:106FD0006F00801993F487FF63C2071863E0B41849
:106FE000EF00807D9307701F63F6974693D7940058
:106FF0006386071A13074000636CF73C93D764005D
:10700000138697031385870393163600376901802B
:1070100013090943B306D90003A44600938686FFEB
:10702000638686029305F0006F000001635C0732FF
:107030000324C400638C86008327440093F7C7FFB2
:1070400033879740E3D4E5FE1306050003240901C6
:107050009308890063081417032544009306F00081
:107060001375C5FFB307954063CCF640232A190179
:107070002328190163D6073E9307F01F63EAA72E62
:10708000937785FF9387870083254900B307F9002D
:1070900083A6070013555500130710003317A700E8
:1070A0003367B700938587FF2326B4002324D400D9
:1070B0002322E90023A0870023A6860093572640B9
:1070C00093051000B395F5006368B710B3F7E500BA
:1070D00063940702939515001376C6FFB3F7E50096
:1070E00013064600639A070093951500B3F7E50071
:1070F00013064600E38A07FE1308F0001313360058
:1071000033036900130503008327C500130E06002F
:107110006302F52E03A747001384070083A7C70067
:107120001377C7FFB30697406342D82EE3C206FE2B
:107130003307E400832647000326840013850900F3
:1071400093E616002322D7002326F60023A4C700C7
:10715000EF00C066130584006F0000019307C000B4
:1071600023A0F900130500008320C102032481023B
:1071700083244102032901028329C101032A8101D9
:10718000832A4101032B0101832BC100032C8100C1
:10719000832C410013010103678000009306002047
:1071A000130600041305F0036FF05FE603A4C700A5
:1071B00013062600E39487DE03240901930889005F
:1071C000E31C14E903274900935726409305100058
:1071D000B395F500E37CB7EE03248900832A4400CD
:1071E00013FBCAFF63689B00B3079B401307F000C3
:1071F0006346F714B7770180B77C018083AA879D27
:1072000003A78C9C9307F0FF330A6401B38A5401EF
:10721000630AF734B71700009387F700B38AFA00C0
:10722000B7F7FFFFB3FAFA0093850A001385090048
:10723000EF1000799307F0FF930B0500630CF5281E
:1072400063684529377C0180130CCC9D83250C0095
:10725000B385BA002320BC00938705006304AA3AD3
:1072600083A68C9C1307F0FF638CE63A338A4B416C
:10727000B307FA002320FC0093FC7B0063860C30EC
:10728000B7170000B38B9B4193858700938B8B00CE
:10729000B3859541B38A5B019387F7FFB385554169
:1072A00033FAF50093050A0013850900EF104071C9
:1072B0009307F0FF6300F53C33057541B30A4501C0
:1072C00083250C002324790193EA1A00B305BA0040
:1072D0002320BC0023A25B01630824359306F00041
:1072E00063F866350327440093074BFF93F787FF46
:1072F000137717003367F7002322E40013065000CA
:107300003307F4002322C7002324C70063EEF636B8
:1073100083AA4B0013840B00B777018003A7479D16
:107320006374B70023AAB79CB777018003A7079DB2
:107330006376B71A23A8B79C6F00401A13E71400AE
:107340002322E400B30494002324990093E7170058
:107350001385090023A2F400EF00404613058400C2
:107360006FF09FE08326C400032684006FF01FC4E3
:1073700093579500130740006372F71413074001F9
:10738000636AF7229386C7059385B70593963600FF
:10739000B306D90083A70600938686FF6388F61C90
:1073A00003A747001377C7FF6376E50083A787002D
:1073B000E398F6FE83A6C700032749002326D400DE
:1073C0002324F40023A4860023A687006FF01FCF98
:1073D000130740016376F71213074005636AF71E2F
:1073E00093D7C4001386F7061385E7069316360075
:1073F0006FF0DFC1130E1E0093773E00130585006A
:10740000638E07108327C5006FF09FD0032684008A
:1074100093E514002322B4002326F60023A4C7001A
:10742000B3049400232A99002328990093E71600B7
:1074300023A6140123A4140123A2F4003307E400BB
:10744000138509002320D700EF004037130584007F
:107450006FF09FD113D63400938784006FF09FB2F2
:107460003307A400832747001385090093E717001B
:107470002322F700EF008034130584006FF0DFCE85
:1074800013E714002322E400B3049400232A990094
:107490002328990013E7170023A6140123A414013D
:1074A00023A2E4003305A4002320F500138509007E
:1074B000EF00C030130584006FF01FCB93576500B9
:1074C0009386970393858703939636006FF05FEC5E
:1074D000630E241103248900832A440093FACAFF0F
:1074E000B3879A4063E69A001307F000E348F7E495
:1074F00013850900EF00802C130500006FF0DFC634
:107500001386C7051385B705931636006FF01FB0B5
:10751000832783001306F6FF6392671C9377360078
:10752000130383FFE39607FE0327490093C7F5FF84
:10753000B3F7E7002322F90093951500E3EEB7C8EF
:10754000E38C05C833F7F500631A0700939515001F
:1075500033F7F500130E4E00E30A07FE13060E0084
:107560006FF0DFB9938A0A016FF01FCC0325490041
:1075700093D52540130710003317B7003367A700D2
:107580002322E9006FF09FE3B3855B01B305B040B0
:107590009395450113DA450193050A001385090007
:1075A000EF1000429307F0FFE318F5D0130A000034
:1075B0006FF01FD1130740056362F7089357C500AA
:1075C0009386F7069385E706939636006FF05FDCA7
:1075D000130740156362F70893D7F40013868707F3
:1075E00013857707931636006FF05FA2377C018012
:1075F000130CCC9D83270C00B387FA002320FC00DA
:107600006FF01FC613174A01E31C07C40324890047
:10761000B30A5B0193EA1A00232254016FF0DFCF13
:1076200023A47C9D6FF05FC513840B006FF0DFCE49
:107630009307100023A2FB006FF09FEB1307401588
:107640006362F7069357F50093868707938577075C
:10765000939636006FF0DFD3130740556362F70649
:1076600093D724011386D7071385C70793163600CF
:107670006FF0DF99938C8CFFB38A9A01B38A7A41B9
:10768000130A00006FF0DFC393058400138509001F
:10769000EFC00FE80324890083250C00832A4400EF
:1076A0006FF09FC7130740556364F7029357250196
:1076B0009386D7079385C707939636006FF05FCD03
:1076C0009306803F1306F0071305E0076FF01F9441
:1076D0009306803F9305E0076FF09FCB8327490017
:1076E0006FF09FE59377350093F6F50F638A0702F5
:1076F0009307F6FF630E06021306F0FF6F0080018A
:107700001305150013773500630E07009387F7FF05
:107710006380C70203470500E314D7FE67800000BB
:1077200093070600130730006366F70263960700AD
:107730001305000067800000B307F5006F00C0006C
:1077400013051500E386A7FE03470500E31AD7FEDD
:107750006780000037070100939885001307F7FF43
:10776000B3F8E80093F5F50FB3E5B8009398050179
:10777000B3E8B8003708FFFEB78580801308F8EF3C
:1077800093850508130330000327050033C7E8007D
:10779000330607011347F7FF3377E6003377B70067
:1077A000E31C07F89387C7FF13054500E36EF3FC5E
:1077B000E39407F86FF0DFF7678000006780000050
:1077C0008327C504130101FF232481002322910094
:1077D00023261100232021011304050093840500B2
:1077E000638E070213952400B387A70003A5070043
:1077F000630605040327050023A0E70023280500EE
:10780000232605008320C100032481008324410036
:107810000329010013010101678000001306100213
:1078200093054000EF50805A2326A40493070500D7
:10783000E31A05FA130500006FF0DFFC13091000CE
:1078400033199900130659001316260093051000EA
:1078500013050400EF508057E30E05FC232295002A
:10786000232425016FF09FF96380050203A74500DB
:107870008327C50413172700B387E70003A7070072
:1078800023A0E50023A0B70067800000130101FEDC
:10789000232A910083A4050137030100232C8100D2
:1078A0002328210123263101232E11002324410105
:1078B0001389050093090500138406001388450108
:1078C000930800001303F3FF832708001308480000
:1078D00093881800B3F66700B386C60293D70701F2
:1078E000B387C702B386860013DE060133F766004E
:1078F000B386C701939706013387E700232EE8FE7E
:1079000013D40601E3C298FC6302040283278900B2
:1079100063D0F4049387440093972700B307F900DA
:1079200023A2870093841400232899008320C10197
:1079300003248101832441018329C100032A81009A
:1079400013050900032901011301010267800000EA
:10795000832549001385090093851500EFF05FE644
:10796000130A0500630C0504032609019305C900E9
:107970001305C5001306260013162600EF50107DD0
:107980000327490083A7C90413172700B387E7001B
:1079900003A707002320E90023A0270193874400C1
:1079A00013090A0093972700B307F90023A2870061
:1079B00093841400232899006FF05FF7B756018075
:1079C0003755018093864638130600009305500B07
:1079D00013058539EF50C038130101FE232C8100B7
:1079E000232A910023282101232631012324410148
:1079F0001388860093079000232E11002322510143
:107A00003348F80293890600130905001384050022
:107A1000130A06009304070063D8D70C93071000DD
:107A2000930500009397170093851500E3CC07FF9B
:107A300013050900EFF0DFD893050500630A050A76
:107A4000930710002328F500232A95009307900040
:107A500063D64709930A940093840A0033044401CF
:107A600083C604001306A00013050900938606FDD3
:107A7000EFF0DFE19384140093050500E39284FEA8
:107A800013048AFF33848A0063563A03B389494159
:107A9000B3093401834604001306A000130509004E
:107AA000938606FDEFF09FDE130414009305050096
:107AB000E39289FE8320C1010324810183244101D3
:107AC000032901018329C100032A8100832A41007F
:107AD0001385050013010102678000001304A40050
:107AE000130A90006FF05FFA930500006FF05FF4E7
:107AF000B75601803755018093864638130600003B
:107B00009305E00C13058539EF5080253707FFFFFB
:107B10003377E5009307050013050000631607009F
:107B20009397070113050001370700FF33F7E700BC
:107B3000631607001305850093978700370700F049
:107B400033F7E700631607001305450093974700D6
:107B5000370700C033F7E700631607001305250059
:107B60009397270063C807001397170013051500A4
:107B7000635407006780000013050002678000005F
:107B8000832705001307050093F677006384060238
:107B900093F6170013050000639E060693F6270070
:107BA0006380060893D717002320F7001305100001
:107BB000678000009396070193D606011305000025
:107BC0006396060093D707011305000193F6F70F9C
:107BD000639606001305850093D7870093F6F70098
:107BE000639606001305450093D7470093F63700C8
:107BF000639606001305250093D7270093F6170018
:107C0000639C060093D717001305150063960700C1
:107C100013050002678000002320F7006780000042
:107C200093D727002320F70013052000678000006A
:107C3000130101FF23248100138405009305100024
:107C400023261100EFF0DFB7630005028320C10097
:107C5000232A850003248100130710002328E50050
:107C60001301010167800000B7560180375501807C
:107C700093864638130600009305001413058539D2
:107C8000EF50000E130101FE2328210123263101AC
:107C900003A9050183290601232A91002324410118
:107CA000232E1100232C8100138A05009304060063
:107CB000634C390113870900938405009309090077
:107CC000130A06001309070083A7840083A5440054
:107CD00033842901B3A78700B385F500EFF05FAEC9
:107CE000630C051A1303450193182400B30813010C
:107CF000930703006378130123A0070093874700CD
:107D0000E3EC17FF13084A01131E2900938E440168
:107D100093952900330EC801B385BE00637CC80B60
:107D200093875401130F400063FEF51437060100DA
:107D30001306F6FF6F000001130848001303430009
:107D4000637AC809832F0800B3F4CF006394040C4E
:107D500093DF0F01E3820FFE03270300930203006A
:107D600093860E00930407009303000083A7060088
:107D700093D904013377C700B3F7C700B387F7037C
:107D800083A44200938242009386460033F9C400E4
:107D9000B3873701B38777009393070133E7E30095
:107DA00023AEE2FE03D7E6FF93D707013307F703BD
:107DB000330727013307F70093530701E3E8B6FAC7
:107DC000B307E30123A0E7001308480013034300AF
:107DD000E36AC8F7634880006F0080011304F4FF72
:107DE0006308040083A7C8FF9388C8FFE38807FEE1
:107DF0008320C101232885000324810183244101BC
:107E0000032901018329C100032A81001301010212
:107E1000678000009303030093820E0013090000A3
:107E200003A7020083AF030093834300B376C70028
:107E3000B38696029357070133F7CF0093DF0F0104
:107E400093824200B3879702B386E600B386260189
:107E500013D70601B3F6C600B387F701B387E7006F
:107E600013970701B366D70023AED3FE13D90701DA
:107E7000E3E8B2FAB307E30123A02701832F080048
:107E80006FF01FED338F9540130FBFFE137FCFFFB1
:107E9000130F4F006FF09FE9B756018037550180EF
:107EA00093864638130600009305D01513058539CF
:107EB000EF40106B130101FE232C810023263101BA
:107EC00023244101232E1100232A9100232821017C
:107ED000937736001304060093090500138A050002
:107EE0006394070C1354244013090A006308040622
:107EF00083A48904638E040C9377140013090A0089
:107F00006390070213541440630A040403A5040099
:107F1000630805069304050093771400E38407FEC5
:107F2000138604009305090013850900EFF09FD51F
:107F3000630809060327490083A7C90413541440A2
:107F400013172700B387E70003A707002320E900E2
:107F500023A0270113090500E31A04FA8320C101B5
:107F600003248101832441018329C100032A810064
:107F700013050900032901011301010267800000B4
:107F8000138604009385040013850900EFF09FCF4A
:107F900023A0A40023200500930405006FF0DFF761
:107FA000130905006FF01FF69387F7FF375701801D
:107FB0001307073F93972700B307F70003A60700AF
:107FC00093060000EFF09F8C130A05006FF09FF1FD
:107FD0009305102713850900EFF09FC523A4A9047A
:107FE00093040500232005006FF01FF1130101FE2B
:107FF0002324410103AA050183A78500232631011B
:1080000093595640338A4901232C8100232A910039
:108010002328210123225101232E110013091A00C4
:10802000938405001304060083A54500930A050008
:1080300063D827019397170093851500E3CC27FF9A
:1080400013850A00EFF0CFF7630C05101308450104
:1080500063543003938959009399290033073501FC
:10806000930708009387470023AE07FEE39CE7FED3
:108070009389C9FE3308380103A70401938744019B
:108080001373F401131627003386C7006304030A31
:1080900093050002B385654093080800930600002D
:1080A00003A70700938848009387470033176700AA
:1080B0003367D70023AEE8FE03A7C7FFB356B70068
:1080C000E3E0C7FE1387540193074000636AE600AC
:1080D000B30796409387B7FE93F7C7FF9387470090
:1080E0003308F8002320D80063840600130A09002F
:1080F00003A7440083A7CA048320C10113172700E4
:10810000B387E70003A70700232845010324810163
:1081100023A0E40023A09700032901018324410147
:108120008329C100032A8100832A4100130101022F
:108130006780000003A707009387470013084800E3
:10814000232EE8FEE3F6C7FA03A70700938747004C
:1081500013084800232EE8FEE3EEC7FC6FF05FF93A
:10816000B7560180375501809386463813060000C4
:108170009305901D13058539EF40903E03270501B7
:1081800083A70501130805003305F7406314F704BE
:108190009397270013084801938545013307F8009A
:1081A000B387F5006F0080006376E8028326C7FF7F
:1081B00003A6C7FF1307C7FF9387C7FFE386C6FE63
:1081C000B3B6C6003305D0401375E5FF130515009F
:1081D000678000006780000083A705010327060170
:1081E000130101FF23248100232291002320210178
:1081F0002326110093840500130406003389E74009
:108200006394E71A931627009385450113074601E7
:10821000B387D5003307D7006F00800063FCF518E3
:1082200003A6C7FF8326C7FF9387C7FF1307C7FFB0
:10823000E306D6FE6360D61683A54400EFF04FD860
:108240006302051A03AE040183220401938F4401E3
:10825000931E2E00130844019392220093034501BC
:10826000B708010023262501B38EDF01B3025800B1
:10827000138F030013830F00930700009388F8FF08
:108280000327030083250800130F4F00B37617015F
:10829000B386F600B3F71501B386F64093D5050112
:1082A00093570701B387B74013D70641B387E70059
:1082B00013970701B3F61601B366D70013084800F9
:1082C000232EDFFE1303430093D70741E36A58FAD6
:1082D000B38582409385B5FE1304540193D52500E0
:1082E0001307000063E48200139725003387E3003F
:1082F0001308400063E6820093851500139825005B
:10830000B38F0F01B383030163FEDF05B7080100DC
:108310001388030093850F009388F8FF03A70500D7
:108320001308480093854500337617013306F6009D
:108330009356064193570701B387D70093960701D9
:1083400033761601B3E6C600232ED8FE93D7074135
:10835000E3E6D5FD1387FEFFB30FF74113F7CFFF19
:108360003387E300639A06008327C7FF130EFEFFDF
:108370001307C7FFE38A07FE8320C100032481009F
:108380002328C501832441000329010013010101B1
:108390006780000093870400130910009304040011
:1083A000138407006FF05FE9E34609FE130900003C
:1083B0006FF09FE893050000EFF08FC063020504A3
:1083C0008320C10003248100930710002328F500B7
:1083D000232A050083244100032901001301010120
:1083E00067800000B7560180375501809386463874
:1083F000130600009305002413058539EF4050163D
:10840000B756018037550180938646381306000021
:108410009305202313058539EF409014B707F07FAB
:10842000B3F5B700B707C0FCB385F5006358B000DB
:10843000930700001385070067800000B305B04074
:1084400093D545419307300163C8B700B7070800CB
:10845000B3D5B7406FF0DFFD1387C5FE9306E0018B
:108460009305000093071000E3C6E6FCB707008001
:10847000B3D7E7001385070067800000130101FEF2
:10848000232A910083240501232C81001304450134
:1084900093942400B30494002328210103A9C4FF6A
:1084A0002326310123244101130509009389050086
:1084B000232E1100EFF08FE513070002B307A7404A
:1084C00023A0F9009307A000138AC4FF63D0A70874
:1084D000130555FF6370440583A784FF63000504FB
:1084E000B306A74033D7D7003319A9003369E90091
:1084F000138684FF3707F03F3367E900B397A7007F
:108500006372C40203A644FFB356D600B3E7D70094
:108510006F00400193070000631405063707F03F22
:108520003367E9008320C1010324810183244101D1
:10853000032901018329C100032A81001385070053
:108540009305070013010102678000009306B00045
:10855000B386A640B707F03F3357D9003367F7001B
:10856000930700006376440183A784FFB3D7D70045
:10857000130555013315A900B367F5006FF09FFA95
:108580003315A9003707F03F3367E5009307000074
:108590006FF05FF9130101FD232C4101138A0500DF
:1085A000930510002322910223202103232E310161
:1085B0002326110223248102232A51019304060059
:1085C0009389060013090700EFF08F9F630A0510D7
:1085D00093D74401370710001306F7FF939657010E
:1085E000130405003376960093FAF77F6384060040
:1085F0003366E6002326C10063080A0813058100DC
:1086000023244101EFF0CFD70327C10093070500D2
:108610006302050C0326810093060002B386A64080
:10862000B316D700B3E6C6003357A700232AD400F9
:108630002326E100B334E00093841400232CE400EB
:108640002328940063840A06938ADABCB38AFA006A
:108650001305500323A05901B307F5402320F90067
:108660008320C102130504000324810283244102F4
:10867000032901028329C101032A8101832A4101BF
:1086800013010103678000001305C100EFF04FCF15
:10869000930710002328F4008327C10093041000DF
:1086A000232AF40093070502E3900AFA13972400A3
:1086B0003307E400032507019387E7BC23A0F900F3
:1086C000EFF0CFC493945400B384A44023209900C6
:1086D0006FF01FF983268100232AD4006FF09FF5E5
:1086E000B75601803755018093864638130600003F
:1086F0009305A03013058539EF408066130101FD15
:1087000023202103138905009305810023261102EC
:108710002324810223229102232E31019309050093
:10872000EFF0DFD59304050013840500130509005D
:108730009305C100EFF09FD48327090103A7090126
:108740008326C1003307F7408327810013175700A2
:10875000B387D740B307F70093060500635EF002C6
:10876000939747013384870013860600138504001E
:108770009386050093050400EF7050398320C102F1
:108780000324810283244102032901028329C101B8
:10879000130101036780000013974701B385E5408B
:1087A0006FF09FFC130101FF2320210123261100FC
:1087B00023248100232291009307700113090500EF
:1087C00063DAA704377701808327879A8325C79ABE
:1087D000377701800324079B8324479B1385070079
:1087E0001306040093860400EF80403E1309F9FF4E
:1087F00093070500E31409FE8320C10003248100D0
:10880000832441000329010013850700130101019E
:1088100067800000B7570180131935009387073F21
:1088200033892701832709018320C10003248100A4
:108830008325490183244100032901001385070092
:108840001301010167800000832606019385F5FF6F
:1088500093D55540938515009307460193962600BE
:1088600093952500B386D700B305B50063F8D7020A
:108870001307050003A80700938747001307470065
:10888000232E07FFE3E8D7FEB387C6409387B7FEE2
:1088900093F7C7FF938747003305F5006378B5006A
:1088A00013054500232E05FEE36CB5FE678000002E
:1088B0000327050113D65540930645016352C702AD
:1088C00093172700B387F60063F2F60403A7C7FFE8
:1088D0009387C7FFE30A07FE1305100067800000B7
:1088E00093172600B387F600E350E6FE93F5F501F3
:1088F000E38C05FC03A60700130510003357B600F0
:10890000B315B700E302B6FC678000001305000052
:1089100067800000130101FF23229100B70400804B
:10892000232481002326110093C4F4FF13040600BE
:1089300023200600B3F6B4003706F07F93870500C6
:108940001307050063D0C606B3E8A600638C0804CD
:1089500033F6C50013880500930800006312060271
:10896000B777018083A6C79B03A6879BEF8000266D
:108970001307050013880500B3F6B4009308A0FCA4
:1089800093D64641B70710809387F7FF938626C09A
:108990003378F800B3861601B707E03FB367F800F5
:1089A0002320D4008320C1000324810083244100BC
:1089B000130507009385070013010101678000007C
:1089C000130101FF232481002322910013040500D9
:1089D000B7740180138505002326110023A204A08B
:1089E000EF708FF29307F0FF630CF5008320C10056
:1089F00003248100832441001301010167800000EA
:108A000083A744A0E38407FE8320C1002320F40051
:108A100003248100832441001301010167800000C9
:108A2000130101F6930EC108232AF10837030080D1
:108A3000B707FFFF138E05001343F3FF2326D1086A
:108A4000938787209305810093860E00232E1106BD
:108A5000232AF1002328E108232C0109232E1109E0
:108A60002324C101232CC101232E6100232861008E
:108A70002322D101EF00403D83278100238007009E
:108A80008320C1071301010A67800000130E05004F
:108A900037750180130101F60325459C930E81086B
:108AA000232AF10837030080B707FFFF1343F3FFC2
:108AB0002324C1082326D108938787201386050025
:108AC00093860E0093058100232E1106232AF100C0
:108AD0002328E108232C0109232E11092324C10195
:108AE000232CC101232E6100232861002322D10100
:108AF000EF00803583278100238007008320C10792
:108B00001301010A67800000130101FF2324810083
:108B1000138405008395E50023261100EF50C0065D
:108B200063400502832704058320C100B387A700A3
:108B30002328F4040324810013010101678000004D
:108B40008357C40037F7FFFF1307F7FFB3F7E700BA
:108B50008320C1002316F4000324810013010101C6
:108B60006780000013050000678000008397C50040
:108B7000130101FE232C8100232A910023282101C7
:108B800023263101232E110013F70710138405004B
:108B9000930405008395E5001309060093890600F8
:108BA000631E070237F7FFFF1307F7FFB3F7E7006E
:108BB0002316F400032481018320C1019386090058
:108BC000130609008329C10003290101138504004C
:108BD00083244101130101026F40C011930620005C
:108BE00013060000EF4090488317C4008315E4008B
:108BF0006FF05FFB130101FF232481001384050044
:108C00008395E50023261100EF4050469307F0FFBF
:108C10006304F5028357C400371700008320C100A6
:108C2000B3E7E7002328A4042316F40003248100FB
:108C300013010101678000008357C40037F7FFFF6D
:108C40001307F7FFB3F7E7008320C1002316F400F2
:108C50000324810013010101678000008395E50072
:108C60006F40C021B367B50093F7370063920708E0
:108C700003A70500B7867F7F9386F6F7B377D70003
:108C8000B387D700B3E7E700B3E7D7001306F0FFD9
:108C9000639EC706130605001308F0FF2320E600B5
:108CA00003A745009385450013064600B377D70018
:108CB000B387D700B3E7E700B3E7D700E38007FF48
:108CC00083C7050003C7150083C625002300F600EF
:108CD000638A0700A300E600630607002301D600AD
:108CE0006394060067800000A3010600678000000F
:108CF0009307050003C705009387170093851500A8
:108D0000A38FE7FEE31807FE678000001306050047
:108D10006FF01FFB9377350013070500639C070472
:108D2000B7867F7F9386F6F79305F0FF032607004B
:108D300013074700B377D600B387D700B3E7C70060
:108D4000B3E7D700E384B7FE8346C7FF0346D7FFE8
:108D50008347E7FF3307A74063800604630A0602E0
:108D60003335F0003305E5001305E5FF67800000AB
:108D7000E38806FA83470700130717009376370046
:108D8000E39807FE3307A7401305F7FF678000004D
:108D90001305D7FF678000001305C7FF6780000039
:108DA000B3E7A50093F7370013070500639807069C
:108DB0009307300063F4C7063703FFFEB78880804F
:108DC0001303F3EF93880808130E300083A6050001
:108DD000B387660013C8F6FFB3F70701B3F71701AF
:108DE000639E07022320D7001306C6FF1307470020
:108DF00093854500E36CCEFC93851500930717001F
:108E00006304060283C6F5FF1308F6FFA38FD7FE9F
:108E1000638E06001387070013060800938515006C
:108E200093071700E31006FE678000003306C700B3
:108E3000630A080093871700A38F07FEE39CC7FE11
:108E40006780000067800000130101E12326111EE6
:108E5000232A511D2328611D2320A11D138B0500EA
:108E6000130D06002326D1002324811E2322911EE8
:108E70002320211F232E311D232C411D2326711D4C
:108E80002324811D2322911D232EB11B930A05004B
:108E9000EFD05FE983270500138507002320F10445
:108EA000EFF05FE78357CB002328010E232A010E42
:108EB000232C010E232E010E93F70708232EA10267
:108EC0006388070083270B01639407006F10C05B62
:108ED000B757018093878751232AF10083470D00FC
:108EE000930BC110B75901802322710F2326010E65
:108EF0002324010E23280100232C01002322010436
:108F0000232C01022324010423260104232201002F
:108F100093880B00938949696380072213040D002D
:108F2000930650026382D73C834714001304140055
:108F3000E39A07FEB304A4416300A4218326C10E73
:108F40008327810E23A0A801B3869600938717007C
:108F500023A298002326D10E2324F10E930670003D
:108F60009388880063CAF6380327410083470400CA
:108F7000330797002322E1006380071C8344140019
:108F8000A303010C130414001303F0FF130A0000E1
:108F900013090000130CA005930C9000930DA00280
:108FA00013041400938704FE6364FC040327410147
:108FB00093972700B387E70083A707006780070020
:108FC000130A0000938704FD8344040093162A00CB
:108FD000338A4601131A1A00338A4701938704FD26
:108FE00013041400E3F2FCFE938704FEE370FCFC20
:108FF0006384041423069114A303010C130C1000C2
:10900000930C1000130DC114930D00001303000006
:1090100023260102232A010223280102937F29002B
:1090200063840F00130C2C00137F49088327C10EA3
:1090300063160F0033088A41E34000738346710CC6
:10904000638A06028326810E1306710C23A0C800D2
:1090500093871700130610009386160023A2C800FA
:109060002326F10E2324D10E130670009388880066
:109070006340D660638C0F028326810E1306810C39
:1090800023A0C800938727001306200093861600AC
:1090900023A2C8002326F10E2324D10E130670004C
:1090A000938888006354D6006F00107B93060008F5
:1090B000E302DF4E33039341E34A605A937609108B
:1090C000E39E06380327810EB387970123A0A801EA
:1090D0001307170023A298012326F10E2324E10E83
:1090E0009306700063C0E66E938888001379490088
:1090F00063060900B3048A416346906E63548A0193
:10910000130A0C0003274100330747012322E10023
:10911000E39C07602324010E63880D0093850D00F6
:1091200013850A00EFA0DFBE93880B00130D040027
:1091300083470D00E39407DE8327C10E6384070095
:109140006F1090398357CB0093F7070463840700AF
:109150006F20803F8320C11E0324811E0325410010
:109160008324411E0329011E8329C11D032A811D59
:10917000832A411D032B011D832BC11C032C811C41
:10918000832C411C032D011C832DC11B1301011FC6
:109190006780000013850A00232E1101232461003B
:1091A000EFD05FB883274500138507002326F1041D
:1091B000EFF05FB69307050013850A00938407005C
:1091C0002324F104EFD01FB68327850003238100F9
:1091D0008328C101232CF102638404006F10C015A1
:1091E000834404006FF0DFDB834404001369090249
:1091F0006FF01FDB13690901937709026388076C1D
:109200008327C1009387770093F787FF03A7470061
:1092100083AD0700938787002326F100930C070096
:109220006340076E1307F0FF130C0900E30CE30023
:1092300033E79D01137CF9F7E3160700E31A0300F7
:1092400013090C0013030000930C0000130D011B05
:10925000138C0C0063D46C00130C03008347710C57
:1092600023260102232A010223280102930D000074
:10927000E38607DA130C1C006FF05FDA136909014B
:1092800093770902638C07608327C10013877700F7
:10929000137787FF832D0700832C470093078700F0
:1092A0002326F100137CF9BF13070000A303010C70
:1092B0009306F0FF630AD366B3E69D011379FCF7CA
:1092C000E3980648E31E0312E31E07F6937C1C0096
:1092D000130D011BE38E0CF693070003A307F11A8D
:1092E000130DF11A6FF0DFF6B304A441E318A4C51F
:1092F000834704006FF05FC81306410E93050B000F
:1093000013850A00EF40507EE31E05E293880B00B0
:109310006FF09FC593778900638407006F10800703
:109320008327C1001305010B232E110193877700BA
:1093300093F787FF83A5070003A64700938787005D
:10934000232461002326F100EFB0C0488327010BDE
:109350008328C101032381002328F10E8327410BB9
:10936000232AF10E8327810B232CF10E8327C10BB7
:10937000232EF10E1305010F232E1101232461006A
:10938000EFD09F932326A10C930720000323810095
:109390008328C1016314F5006F10C05E93071000AD
:1093A0006314F5006F109000930710066394F400A7
:1093B0006F204012930710046394F4006F10D0469E
:1093C00093FCF4FD9307F0FF232C91076314F30043
:1093D0006F109015930770046394FC006F20801742
:1093E000032EC10F23242107832E010F032F410FCA
:1093F000832F810F9367091063540E006F20002A9A
:10940000232E010613890700930D000093076004C3
:109410006394FC006F10D0219307500423241103A0
:109420006384FC006F10D029930C1300130C010B04
:109430001308C10D93860C009307010D1307C10C8F
:109440001306200093050C0013850A0023226102F5
:109450002328D10B2320D103232AE10B232EE10162
:10946000232CF10B2328F101232EC10B2324C1014E
:10947000EFC04FD8032E8100832F0101032FC101BC
:10948000832E0102032341028328810233089501C0
:10949000130D0500930C010A93850C0013050C00B5
:1094A000232E010123281101232461002328D10B3D
:1094B000232AE10B232CF10B232EC10B2320010ABD
:1094C0002322010A2324010A2326010AEF70906A4D
:1094D0000328C101032381008328010193070800A9
:1094E000630205028327C10D63FE07011306000313
:1094F00093861700232ED10C2380C7008327C10D2C
:10950000E3E807FF0327C10CB387A7412328F10035
:109510002328E10203278107930770046314F700EF
:109520006F10500203278107930760046314F7004C
:109530006F10502783270103032781079305100429
:109540009387F7FF2326F10C93F6F40F1306000020
:109550006318B7009386F60093F6F60F1306100013
:10956000230AD10C9306B00263DA07000327010334
:10957000930710009306D002B387E740A30AD10CEB
:109580009306900063C4F6006F2000231308310E89
:10959000130508001306A000130E3006B3E6C70239
:1095A00093050500138307001305F5FF9386060353
:1095B000A38FD5FEB3C7C702E3426EFE93870703AE
:1095C00013F6F70FA30FC5FE9387E5FF63E40701CA
:1095D0006F2040339306610D6F00800003C60700C3
:1095E0002380C6009387170093861600E39807FF31
:1095F0009307510EB387B7401307610DB307F70008
:109600009306410DB387D7402322F10403270101BC
:109610008326410493071000B30CD70063C4E7000E
:109620006F20801C8327C103B38CFC008327810635
:1096300013CCFCFF135CFC4113F9F7BF136909104D
:1096400033FC8C0123260102232A01022328010274
:109650008327C107639407006F1000769307D00239
:10966000A303F10C13030000130C1C006FF01F9BED
:109670001306410E93050B0013850A002320610297
:10968000232EE1012324F101EF401046E318050ADF
:109690008327C10E03230102032FC101832F810001
:1096A00093880B006FF01F9D0326810E0327010195
:1096B0009306100023A0A8019387170093041600B7
:1096C000938C8800E3DCE6329306100023A2D800D6
:1096D0002326F10E2324910E93067000E3C6963ED6
:1096E0000327C1038326010493841400B387E70092
:1096F00023A0DC0023A2EC002326F10E2324910EEC
:1097000093067000938C8C00E3C2963E8326010F73
:10971000138814009305010A2328D10A8326410FD8
:109720001305010B232EF100232AD10A8326810F72
:10973000232401012320010A232CD10A8326C10FEF
:109740002322010A2324010A232ED10A2326010AF7
:10975000EF705042832701010328810093888C0019
:109760009386F7FF130608008327C101E30C052A3F
:1097700013071D00B387D70023A0EC0023A2DC0051
:109780002326F10E2324010F13077000E34A077705
:1097900013870C0113862400938C0800930807009C
:1097A000832641041307410D23A0EC00B387F60084
:1097B00023A2DC002326F10E2324C10E1307700020
:1097C000E356C7921306410E93050B0013850A005A
:1097D000EF409031631405768327C10E93880B0008
:1097E0006FF0DF90930600010327810E63C496009B
:1097F0006F10D002B7560180938E4668130900019E
:10980000930C70006F00C000938404FF635A9904A6
:10981000938707011307170023A0D80123A228016B
:109820002326F10E2324E10E93888800E3DEECFC6E
:109830001306410E93050B0013850A002324D10162
:10984000EF40902A631C056E938404FF8327C10EAA
:109850000327810E832E810093880B00E34A99FA37
:10986000B38797001307170023A0D80123A29800FD
:109870002326F10E2324E10E93067000E3D0E68840
:109880001306410E93050B0013850A00EF40D02507
:109890006316056A8327C10E6FF05F868326C100B9
:1098A0009377090113874600E39E072C93770904F9
:1098B000639407006F10C02D8327C100930C000034
:1098C0002326E10083DD07006FF0DF9D8326C100C2
:1098D0009377090113874600E39C072893770904CF
:1098E000639407006F1000278327C1002326E1003F
:1098F000839D070093DCFD4113870C00E35407921E
:109900003337B001B3079041B38CE7401307D0025F
:10991000A303E10C9306F0FFB30DB041130C090053
:1099200013071000E31AD39893061000630CD710A6
:10993000930620006302D72E130D011B1396DC0142
:1099400093F67D0093DD3D0093860603B36DB6016B
:1099500093DC3C00A30FDDFE33E69D0193050D0073
:10996000130DFDFFE31C06FC93771C006380072E9C
:1099700093070003638CF62C9385E5FFA30FFDFE90
:109980009307011BB38CB74013090C00138D05001E
:109990006FF01F8C8327C100A303010C03AD0700E8
:1099A00093864700E3060D309307F0FF6314F3003E
:1099B0006F108010130603009305000013050D00BF
:1099C000232ED1002326110123246100EFD09FD143
:1099D000032381008328C1008326C101930D050064
:1099E000631405006F104056B30CA5418347710CFA
:1099F00013CCFCFF135CFC412326D100232601027B
:109A0000232A01022328010233FC8C01930D00005C
:109A100013030000E39007866FF04FE00327C100B7
:109A2000A303010C130C1000832707001307470042
:109A30002326E1002306F114930C1000130DC1142A
:109A40006FF08FDCE3940C4E13079000E360B74F88
:109A5000938D0D03A307B11B13090C00930C100089
:109A6000130DF11A6FF0CFFE83440400136949000F
:109A70006FF00FD39307B00283440400A303F10CEB
:109A80006FF00FD283440400136909086FF04FD1BF
:109A900083440400930614006394B4016F10D061F2
:109AA000938704FD138406001303000063ECFCCECF
:109AB00083440400931623003383660013131300BA
:109AC0003303F300938704FD13041400E3F2FCFE58
:109AD0006FF04FCD8327C1008344040003AA070021
:109AE000938747002326F100635C0ACA330A40418A
:109AF000136949006FF0CFCA834404001369190049
:109B00006FF00FCA8347710C83440400639A07C83F
:109B100093070002A303F10C6FF08FC8136C0901C7
:109B200093770C02638A07768327C1001387770037
:109B3000137787FF93078700832D0700832C470047
:109B40002326F100130710006FF04FF68327C100A2
:109B50003787FFFF1347078383AD07002314E10C0A
:109B600093874700375701802326F100930787F436
:109B7000930C0000136C2900232CF1001307200024
:109B8000930480076FF08FF2834404001369890007
:109B90006FF00FC1834404009307C006E386F40C02
:109BA000136909016FF0CFBF834404009307800657
:109BB000E384F408136909046FF08FBE8326C100A3
:109BC0009377090203A70600938646002326D10057
:109BD0006398077493770901E39A076293770904FE
:109BE000638407006F10C00813790920E30009623D
:109BF00083274100130D04002300F7006FF04FD3BB
:109C0000930610006314D7006F1090139306200082
:109C1000130C0900E312D7D2130D011B8327810116
:109C200093F6FD0093DD4D00B386D70003C6060012
:109C30009396CC01B3EDB60193DC4C00A30FCDFE9F
:109C4000B3E69D01130DFDFFE39A06FC9307011B8C
:109C5000B38CA74113090C006FF08FDF93065006F9
:109C6000E3D496A48326010F9305010A1305010B83
:109C70002328D10A8326410F232EF100232411012A
:109C8000232AD10A8326810F2320010A2322010AD5
:109C9000232CD10A8326C10F2324010A2326010A7B
:109CA000232ED10AEF70006D832881008327C10124
:109CB000631C053C0327810EB7560180938686F707
:109CC00023A0D800938717009306100013071700EE
:109CD00023A2D8002326F10E2324E10E9306700060
:109CE00093888800E3C4E6420327C10C8326010160
:109CF0006350D762032701048326C1039388880039
:109D000023ACE8FE0327810EB387D70023AED8FE2D
:109D1000130717002326F10E2324E10E930670008B
:109D200063C4E672032701019304F7FF635090BCFC
:109D3000930600010327810EE3DA963E930C00019F
:109D4000130D70006F00C000938404FFE3D09C3EAD
:109D5000938707011307170023A0380123A2980156
:109D60002326F10E2324E10E93888800E35EEDFCA8
:109D70001306410E93050B0013850A00EF40C056F1
:109D8000631E051A8327C10E0327810E93880B00DB
:109D90006FF09FFB33088A41635E00B11306000138
:109DA0008326810E635C0607130E0001930E70007C
:109DB0006F00C000130808FF63520E079387070166
:109DC0009386160023A0380123A2C8012326F10E92
:109DD0002324D10E93888800E3DEDEFC1306410EB7
:109DE00093050B0013850A00232E01012324610033
:109DF000EF40804F631405140328C101130E0001C6
:109E00008327C10E130808FF8326810E03238100D8
:109E100093880B00930E7000E3420EFBB38707019B
:109E20009386160023A0380123A208012326F10EF1
:109E30002324D10E1306700093888800635CD6A695
:109E40001306410E93050B0013850A0023246100BD
:109E5000EF4080496314050E032381008327C10E60
:109E600093880B0033039341635A60A413060001E7
:109E70008326810E6358660613080001130E7000D6
:109E80006F00C000130303FF635E6804938707013C
:109E90009386160023A0380123A208012326F10E81
:109EA0002324D10E93888800E35EDEFC1306410E66
:109EB00093050B0013850A0023246100EF40C04284
:109EC000631E050603238100130800018327C10ECA
:109ED000130303FF8326810E93880B00130E70007B
:109EE000E34668FAB38767009386160023A038011B
:109EF00023A268002326F10E2324D10E130670003E
:109F000093888800635CD69A1306410E93050B0074
:109F100013850A00EF40403D631205028327C10EFE
:109F200093880B006FF08F991306410E93050B0079
:109F300013850A00EF40403B630E059C63840DA02F
:109F400093850D0013850A00EF909FDC6FF08F9FC3
:109F5000130C09006FF05F9D375701801306000155
:109F60008326810E930E4768130E00019302700042
:109F7000634806016F004008130808FF635E0E0780
:109F8000938707019386160023A0D80123A2C80156
:109F90002326F10E2324D10E93888800E3DED2FC21
:109FA0001306410E93050B0013850A002324D103E9
:109FB0002322010323206102232EE1012324F10146
:109FC000EF408032E31C05F603284102130E000126
:109FD0008327C10E130808FF8326810E832E81027A
:109FE00003230102032FC101832F810093880B00FB
:109FF00093027000E3460EF9B387070193861600BB
:10A0000023A0D80123A208012326F10E2324D10E78
:10A0100013067000938888006344D6006FF00F82A7
:10A020001306410E93050B0013850A0023206102DD
:10A03000232EE1012324F101EF40002BE31005F072
:10A040008327C10E03230102032FC101832F810047
:10A0500093880B006FE09FFE1306410E93050B00E3
:10A0600013850A00232E61002324E101EF40C0275D
:10A07000E31605EC8327C10E0323C101032F8100E2
:10A0800093880B006FF08F828325C10C635CB078DE
:10A0900003270103832601019304070063C6E63208
:10A0A000635690028326810EB387970023A0A801F0
:10A0B0009386160023A298002326F10E2324D10EA6
:10A0C0001306700093888800E340D63693C6F4FFE9
:10A0D0000327010393D6F641B3F4D400B3049740A9
:10A0E0006348903E0327010393760940B304ED00D3
:10A0F000639406448325C10C0327010163C6E50070
:10A1000093761900E3860634832601040327C103EE
:10A110001306700023A0D8008326810EB387E700C2
:10A1200023A2E800938616002326F10E2324D10EE5
:10A1300093888800E34CD64C832601013307DD0069
:10A140003386B64033079740930C06006354C7002C
:10A15000930C0700635690030327810EB387970182
:10A1600023A098001307170023A298012326F10EBD
:10A170002324E10E9306700093888800E3CCE65E0A
:10A1800013C7FCFF1357F74133F7EC00B304E64065
:10A19000634490006FE09FF5930600010327810E52
:10A1A00063D69678930C0001130D70006F00C00009
:10A1B000938404FF63DC9C769387070113071700E1
:10A1C00023A0380123A298012326F10E2324E10EB7
:10A1D00093888800E35EEDFC1306410E93050B00A7
:10A1E00013850A00EF404010E31A05D48327C10EFF
:10A1F0000327810E93880B006FF09FFB9375190066
:10A20000639405CC23A2D8002326F10E2324910EBB
:10A21000130770006346974E1306260093880801C3
:10A220006FF00FD8635ED0D6130700016344D700E8
:10A230006F100068130D70006F000001938606FF19
:10A24000E350D70C138814009387070123A03C0127
:10A2500023A2EC002326F10E2324010F930408000F
:10A26000938C8C00E35C0DFD1306410E93050B00EF
:10A2700013850A002324D100EF400007E31005CC2A
:10A280008327C10E8324810E83268100938C0B00CB
:10A29000130700016FF09FFA8326C10093770C012A
:10A2A00013874600639C070A93770C04E38407082E
:10A2B0008327C100930C00002326E10083DD070003
:10A2C000130710006FE09FFE1306410E93050B006D
:10A2D00013850A00EF404001E31205C68327C10E33
:10A2E0008324810E938C0B006FF08FBF1306410EF9
:10A2F00093050B0013850A00EF30107FE31005C4AF
:10A300008327C10E8324810E938C0B006FF00FC046
:10A3100013771900631407006FE05FDD6FF09F9DF6
:10A3200083264100130D040093D7F6412320D70064
:10A330002322F7006FE0DFDF8327810383440400DB
:10A34000639407006FE0DFC583C7070063940700CD
:10A350006FE01FC5136909406FE09FC42326E10029
:10A3600083AD0600930C0000130710006FE01FF48C
:10A3700083AD06002326E10093DCFD4113870C002A
:10A380006FE01FEA83AD0600930C00002326E10076
:10A390006FE05FF10327C100832707001307470021
:10A3A0002326E10083A5070003A6470083A68700B4
:10A3B00083A7C7002328B10E232AC10E232CD10E58
:10A3C000232EF10E6FE01FFB93840600E34C90CC2C
:10A3D0006FF0DFCF130C09006FF08FF4B7570180D7
:10A3E000938787F4232CF100937709026386072C67
:10A3F0008327C10013877700137787FF832D07001A
:10A40000832C4700930787002326F1001377190058
:10A41000630E070033E79D01630A0700130700037B
:10A420002304E10CA304910C13692900137CF9BFE8
:10A43000130720006FE09FE783441400136909208D
:10A44000130414006FE0DFB51306410E93050B00F3
:10A4500013850A00EF305069E31205AE8327C10E61
:10A4600093880B006FF01F8C83441400136909025A
:10A47000130414006FE0DFB2B75701809387C7F56C
:10A48000232CF1006FF05FF69305000413850A009A
:10A49000EFC0DFA92320AB002328AB006314050025
:10A4A0006F10C04393070004232AFB006FE05FA2F4
:10A4B00093076000930C030063E8677837570180C7
:10A4C000138C0C002326D100130D07F76FE0DFB3C8
:10A4D000130600018326810E635A966E930C0001C9
:10A4E000130870006F00C000938404FF63D09C6E5B
:10A4F000938707019386160023A0380123A29801B1
:10A500002326F10E2324D10E93888800E35ED8FC25
:10A510001306410E93050B0013850A00EF30D05C43
:10A52000E31E05A08327C10E8326810E93880B00AE
:10A53000130870006FF05FFB03270101130E70001A
:10A54000130800013307ED002324E1000327410332
:10A55000630E070A0327C102631E070A032781034C
:10A560001307F7FF232CE102032741031307F7FF2B
:10A57000232AE1028326C1040327810493888800EB
:10A5800023ACD8FE8326810EB387E70023AEE8FE16
:10A59000938616002326F10E2324D10E634EDE127D
:10A5A000032781038346070003278100938C06005D
:10A5B000330697406354D600930C0600635890030B
:10A5C0008326810EB387970123A0980093861600F7
:10A5D00023A298012326F10E2324D10E634CDE36EC
:10A5E00003278103938888008346070013C6FCFF76
:10A5F0001356F641B3FCCC00B38C964163449003F0
:10A60000B384D40003274103E31607F40327C102F0
:10A61000630007720327C1021307F7FF2326E10235
:10A620006FF05FF58326810E634898016F00C005C7
:10A63000938C0CFF635A9805938707019386160045
:10A6400023A0380123A208012326F10E2324D10ED2
:10A6500093888800E35EDEFC1306410E93050B0031
:10A6600013850A00EF305048E31A058C13080001E7
:10A67000938C0CFF8327C10E8326810E93880B00D9
:10A68000130E7000E34A98FBB38797019386160078
:10A6900023A0380123A298012326F10E2324D10EF2
:10A6A0006346DE7203278103938888008346070090
:10A6B000B384D4006FF01FF58326C100937709019E
:10A6C000138746006386072283AD0600930C0000C3
:10A6D0002326E1006FF09FD31306410E93050B0074
:10A6E00013850A00EF305040E31A05848327C10E1A
:10A6F00093880B0013080001130E70006FF05FEADF
:10A700001306410E93050B0013850A00EF30D03D70
:10A71000E31605820326810E8327C10E930841119B
:10A7200013061600938C0B006FF08F8713790C4083
:10A7300023280100130D011B6F0040031306A00026
:10A740009306000013850D0093850C00232E110144
:10A7500023246100EF504037032381008328C10187
:10A7600063880C4A930D0500938C05001306A00026
:10A770009306000013850D0093850C00232E110114
:10A7800023246100EF50807783270101130505031F
:10A79000A30FADFE938717002328F1000323810048
:10A7A0008328C101130DFDFFE30A09F80327810384
:10A7B00083460700E394D7F81307F00FE380E7F828
:10A7C00063960C009307900063F2B7C98327810456
:10A7D0008325C104232E1101330DFD40138607008C
:10A7E00013050D0023246100EFE08FDB8327810335
:10A7F0001306A0009306000003CE170013850D007A
:10A8000093850C00333EC001B387C701232CF102AE
:10A81000EF50802B032381008328C10123280100EE
:10A820006FF05FF48326810E37560180130686F79A
:10A8300023A0C80093871700130610009386160004
:10A8400023A2C8002326F10E2324D10E1306700084
:10A8500093888800634CD6066392051C0327010188
:10A8600093761900B3E6E600639406006FE01F8854
:10A87000832601040327C1031306700023A0D80018
:10A880008326810EB387E70023A2E8009386160093
:10A890002326F10E2324D10E6342D64693888800E6
:10A8A000032701019386160023A0A801B387E700C0
:10A8B00023A2E8002326F10E2324D10E13077000F3
:10A8C0006344D7006FE05F826FE0DFEF1306410E55
:10A8D00093050B0013850A00EF301021631005E685
:10A8E0008325C10C8327C10E93880B006FF0DFF620
:10A8F00093770904638007288327C100930C000025
:10A900002326E10083DD07006FF05FB01306410EE0
:10A9100093050B0013850A00EF30101D631005E24C
:10A920008327C10E93880B006FF00FBC23A0380162
:10A9300023A29800B3879700130717002326F10E70
:10A940002324E10E9306700063C4E6006FE0CFF9A4
:10A950006FE05FE71306410E93050B0013850A00B5
:10A96000EF309018631C05DC8327810393880B006C
:10A970001308000183C60700130E70008327C10E61
:10A980006FF0DFC68327010F9305010A1305010B42
:10A990002328F10A8327410F232411012320010AD0
:10A9A000232AF10A8327810F2322010A2324010A83
:10A9B000232CF10A8327C10F2326010A232EF10A33
:10A9C000EF60D04283288100634C05428347710CBD
:10A9D000130770046354972437570180130DC7F38E
:10A9E00023260102232A0102232801021379F9F701
:10A9F000130C3000930D0000930C30001303000083
:10AA0000638407006FE01F876FE04FE183274100F9
:10AA1000130D04002320F7006FE08FF1832601045B
:10AA20000327C1031306700023A0D8008326810EDC
:10AA3000B387E70023A2E800938616002326F10ED1
:10AA40002324D10E93888800634AD62AE3DA05E4EA
:10AA5000130600FFB304B040E3D6C528930C0001F1
:10AA6000130870006F00C000938404FFE3DC9C2691
:10AA7000938707019386160023A0380123A298012B
:10AA80002326F10E2324D10E93888800E35ED8FCA0
:10AA90001306410E93050B0013850A00EF30D00416
:10AAA000631E05C88327C10E8326810E93880B0081
:10AAB000130870006FF05FFB13050D0023241101D4
:10AAC0002326D100EFE00FA58347710C134CF5FF4F
:10AAD000135CFC4123260102232A010223280102E0
:10AAE00083288100930C0500337C8501930D0000C1
:10AAF00013030000638407006FE0CFF76FE00FD20D
:10AB00001386140013878C00B387D70023A2DC00C0
:10AB100023A03C012326F10E2324C10E93067000CE
:10AB2000E3C0C6BE1306160093088700930C070007
:10AB30006FE01FC793770C20638407188327C10039
:10AB4000930C00002326E10083CD070013071000BB
:10AB50006FE0CFF593770920638807148327C1003E
:10AB60002326E100838D070093DCFD4113870C0051
:10AB70006FE00FEB93770920638E07108327C100E6
:10AB8000930C00002326E10083CD07006FF01F889F
:10AB9000937709206386070E8327C100930C00007A
:10ABA0002326E10083CD07006FE0CFEF8327C10F9D
:10ABB00063C007148347710C1307700463529742F4
:10ABC00037570180130D47F46FF09FE1B38797006B
:10ABD0009386160023A0380123A298002326F10EA5
:10ABE0002324D10E1306700093888800635CD6CEB0
:10ABF0001306410E93050B0013850A00EF30C06E5B
:10AC0000631E05B28327C10E93880B006FF08FCDB2
:10AC100093079000E3E8B7B56FF04F833757018093
:10AC2000130D87F36FF0DFDB1306410E93050B0066
:10AC300013850A00EF30406B631205B08327C10E05
:10AC400093880B006FF08FC8930C60006FF01F8724
:10AC5000832601013307DD003386B6403303974076
:10AC6000930C0600635EC3D0930C03006FF04FD1CA
:10AC700083274100130D04002310F7006FE04FCB32
:10AC80008327C100930C00002326E10083AD070059
:10AC90006FE04FE18327C100930C00002326E10001
:10ACA00083AD07006FF08FF68327C1002326E100F4
:10ACB00083AD070093DCFD4113870C006FE04FD696
:10ACC0008327C100930C00002326E10083AD070019
:10ACD000130710006FE08FDD1306410E93050B0084
:10ACE00013850A00EF3040608357CB006FE0CFC57B
:10ACF0009307D002A303F10C6FF01FEC1306410E73
:10AD000093050B0013850A00EF30005E631805A25F
:10AD10008325C10C8327C10E8326810E93880B00E7
:10AD2000E3D005B86FF0DFD2130360006FE04FEBA4
:10AD300003270101B306ED0063FE96BA9384060073
:10AD40006FF04FBB032701039307D0FF6344F70065
:10AD5000635AE3009384E4FF93F7F4FD232CF10698
:10AD60006FE04FFD83270101032701036340F728AC
:10AD700083278106930C070093F71700638607006B
:10AD80008327C103B30CF7008327810693F707409D
:10AD90006386070083270103E340F00613CCFCFF22
:10ADA000135CFC4133FC8C019304700623260102E2
:10ADB000232A01026FE0DF898347710C130300002F
:10ADC000638407006FE00FCB6FE04FA51306410EC1
:10ADD00093050B0013850A00EF30005163100596B0
:10ADE0008327810393880B001308000183C60700A3
:10ADF000130E70008327C10EB384D4006FF09F80C0
:10AE00009307D002A303F10C6FF09FBC1306410E11
:10AE100093050B0013850A00EF30004D6310059277
:10AE20008325C10C8327C10E93880B006FF0CFB030
:10AE3000130C010B930603001308C10D9307010DBA
:10AE40001307C10C1306300093050C0013850A008C
:10AE500023241103232261022328D10B2320D103B1
:10AE6000232AE10B232EE101232CF10B2328F101EE
:10AE7000232EC10B2324C101EFA0DFB7032E8100D5
:10AE8000832F0101032FC101832E010203234102FD
:10AE900083288102130D05009307600433086D00B9
:10AEA000639CFC6883460D0093070003E388F61457
:10AEB000930C010A8327C10C3308F8006FE0CFDD43
:10AEC000130C010B9307010D930603001308C10D2A
:10AED0001307C10C1306200093050C0013850A000C
:10AEE000232261022328D10B2320D103232AE10B43
:10AEF000232EE101232CF10B2328F101232EC10B7A
:10AF00002324C101EFA01FAF93077004032E81001B
:10AF1000832F0101032FC101832E0102032341026C
:10AF200083288102130D0500E398FCF68327810630
:10AF300093F71700639C075E130770048327C10D06
:10AF4000232CE1066FE00FDC8347710C2326D10030
:10AF500023260102232A010223280102130C0300E5
:10AF6000930C030013030000638407006FE08FB0AD
:10AF70006FE0CF8A1306410E93050B0013850A007C
:10AF8000EF308036630405006FE05FFB8324C10C63
:10AF9000032701018327C10E93880B0033069740D6
:10AFA0006FF00F9E832781060327010393F7170095
:10AFB000B3E76700E354E00C6398076C832C01034C
:10AFC000930460068327810693F70740639807621E
:10AFD00013CCFCFF135CFC4133FC8C016FF01FDDD4
:10AFE00037570180130D07F46FF09F9F83270101EE
:10AFF0000327C10393047006B38CE7008327010382
:10B00000E342F0FCB38CFC40938C1C0013CCFCFF9F
:10B01000135CFC4133FC8C016FF05FD9B7560180A3
:10B02000938E46686FE0DF83930700032304F10CDF
:10B030009307800513672900A304F10C2324E1067C
:10B0400093073006930D0000130DC11463CE6744BF
:10B05000032EC10F93FCF4FD232C9107232E010630
:10B06000832E010F032F410F832F810F13692910A6
:10B0700063420E3C930710066388F4629307100442
:10B080006384F4006FE08FB8130C010B13050C0000
:10B0900023261103232461022328D10B232AE10B49
:10B0A000232CF10B232EC10BEF9050151306C10C6E
:10B0B000EFD05F86138605009305050013050C008D
:10B0C000EF90407193070109938507002324F10055
:10B0D0008327010B930C010A130601082328F108AA
:10B0E0008327410B13850C002326C106232AF10870
:10B0F0008327810B2320010823220108232CF10838
:10B100008327C10B23240108232EF108B707FC3F36
:10B110002326F108EF6040620328010A032E410A4A
:10B12000832E810A032FC10A93850C0013050C009E
:10B130002328010B23220103232AC10B2320C1034F
:10B14000232CD10B232ED101232EE10B2328E10147
:10B150002320010A2322010A2324010A2326010AAB
:10B16000EF604021032F0101832EC101032E010254
:10B1700003284102032381028328C10263160500CC
:10B18000930710002326F10CB75701809387C7F56A
:10B190002322F1069306F3FF93070D006F00400989
:10B1A00093850C0013050C002320C106232EF10506
:10B1B000232C5104232A71042328F104232A110388
:10B1C000232861022328710A23267102232A510AA7
:10B1D00023245102232CF10B2322F103232EC10A35
:10B1E0002320C1022320010A2322010A2324010A69
:10B1F0002326010AEF6000188326C101032F0102F4
:10B20000832E4102032E81020328C102032301037E
:10B210008328410383270105832341058322810578
:10B22000832FC105032601069386F6FF630E0510E2
:10B230000326810093850C00232AF10213050C00DC
:10B24000B70703402328D1042328110323266102D2
:10B25000232EF1082326E10B2320010B2322C10B0F
:10B260002324D10B23280108232A0108232C0108B9
:10B27000EF60804C832E010B032E410B0328810BC2
:10B280000326C10B13050C002324D1032322C10381
:10B2900023200103232EC100EF9000249305050015
:10B2A0002328A10013050C00EF90C03D0326C10127
:10B2B000832E8102032E4102232EC1080326010B97
:10B2C00003280102832581002320C1080326410BA6
:10B2D00013850C002328D1092322C1080326810BE2
:10B2E000232AC109232C01092324C1080326C10BE9
:10B2F0002326C1080326C106EF708071032741068B
:10B3000083270101832601058323010A3306F70001
:10B3100083450600832741038322410A832F810A44
:10B320000326C10A232AF1062380B7002328D10669
:10B330001307F0FF232ED1000323C102832801034A
:10B3400093871700E39EE6E4B706FE3F93850C0063
:10B3500013050C002320F102232E11012324610088
:10B360002328710A23287102232A510A2326510215
:10B37000232CF10B2324F103232EC10A2322C10223
:10B380002320010A2322010A2324010A2326D10AA9
:10B39000EF600011032381008328C101832701028C
:10B3A0006344A00A832301038322C102832F810205
:10B3B00003264102B706FE3F93850C0013050C00DF
:10B3C0002328710A232A510A232CF10B232EC10AA8
:10B3D0002320010A2322010A2324010A2326D10A59
:10B3E000EF505079032381008328C1018327010294
:10B3F000631805000327010193761700639606047E
:10B40000032701071306000393061700B386D7002E
:10B41000635407006FE00F8F93871700A38FC7FE59
:10B42000E39CD7FE6FE00F8E23242107930D0000CD
:10B4300013890200B707008033CEC7019307D002FB
:10B44000232EF1066FF01FC30327410793860700E1
:10B45000232EE10C0327410603C6F7FF8345F700BF
:10B460006310B60213050003A38FA6FE8326C10D49
:10B470001386F6FF232EC10C03C6F6FFE386C5FE36
:10B48000930516001305900393F5F50F6306A600C8
:10B49000A38FB6FE6FE00F87032741068345A70001
:10B4A000A38FB6FE6FE00F869305130013850A0085
:10B4B0002328110123246100EFB05FA7032381003B
:10B4C00083280101130D050063040542930D050057
:10B4D0006FF01FB8930700032304F10C9307800754
:10B4E0006FF05FB5B38797009386160023A03801ED
:10B4F00023A298002326F10E2324D10E13067000F8
:10B50000635ED6B81306410E93050B0013850A003F
:10B51000EF20905D630405006FE05FA28327C10EFA
:10B520008326810E93880B006FF08FB7930770040A
:10B5300033086D00232CF106930C010A6FD0DFF560
:10B54000130C09006FE0CFD09307F0FF2322F10026
:10B550006FD05FC06314030013031000032EC10FEC
:10B56000832E010F032F410F832F810F9362091048
:10B57000E34C0EEA130C010B930603001308C10DF4
:10B580009307010D1307C10C1306200093050C004F
:10B5900013850A002326510223241103232261026A
:10B5A0002328D10B2320D103232AE10B232EE101F1
:10B5B000232CF10B2328F101232EC10B2324C101DD
:10B5C000EFA04FC38322C10223242107032E810051
:10B5D000832F0101032FC101832E010203234102A6
:10B5E00083288102130D050013890200930D0000CA
:10B5F000232E01066FF09F93930470068327810327
:10B600009306F00F2326010283C70700232A0102B5
:10B610006388D7040327010363D4E704B307F74023
:10B62000032781032328F10283471700638E070055
:10B630000326410313071700232CE102130616000B
:10B64000232AC1026FF0DFFC0327C1028327810395
:10B650001307170083C707002326E1026FF05FFB83
:10B660000327C10283274103B387E700032781042F
:10B67000B387E702B38C970113CCFCFF135CFC414A
:10B6800033FC8C016FD0DFFC8327C1039304600679
:10B69000B30CF700B38C6C006FF0DF92930D0000D9
:10B6A000138907006FF01FD9130C010B13050C0051
:10B6B00023261103232461022328D10B232AE10B23
:10B6C000232CF10B232EC10BEF9040331306C10C3A
:10B6D000EFD04FA4138605009305050013050C0059
:10B6E000EF90400F93070109938507002324F10091
:10B6F0008327010B930C010A130601082328F10884
:10B700008327410B13850C002326C106232AF10849
:10B710008327810B2320010823220108232CF10811
:10B720008327C10B23240108232EF108B707FC3F10
:10B730002326F108EF6040000328010A032E410A86
:10B74000832E810A032FC10A93850C0013050C0078
:10B750002328010B23220103232AC10B2320C10329
:10B76000232CD10B232ED101232EE10B2328E10121
:10B770002320010A2322010A2324010A2326010A85
:10B78000EF50503F032F0101832EC101032E010210
:10B7900003284102032381028328C10263160500A6
:10B7A000930710002326F10CB7570180938787F485
:10B7B0002322F1066FF01F9E9306610D63180600A9
:10B7C00093060003230BD10C9306710D1307011B85
:10B7D000938707033386E6402380F6009307D60D50
:10B7E0002322F1046FD09FE28327810693F717008D
:10B7F000639407006FD09FE36FD0DFE2930C010AE0
:10B8000093850C0013050C00232601032324110348
:10B81000232261022328D10B2320D103232AE10B09
:10B82000232EE101232CF10B2328F101232EC10B40
:10B830002324C1012320010A2322010A2324010A0F
:10B840002326010AEF501033032E8100832F0101BC
:10B85000032FC101832E01020323410283288102A9
:10B860000328C102630805E493071000B38767400B
:10B870002326F10C3308F8006FD01FC2639A07002B
:10B88000130C100093046006930C10006FF00FD29D
:10B890008327C10393046006938C1700B38C6C005C
:10B8A00013CCFCFF135CFC4133FC8C016FF00FD018
:10B8B000138708006FF04FA58327C10003A307007B
:10B8C00093874700635403001303F0FF834414007D
:10B8D0002326F100138406006FD08FEC9307C0007D
:10B8E00023A0FA009307F0FF2322F1006FD09F8678
:10B8F0008357CB0013E70704930707002316EB00D9
:10B900006FD09F84930720002322F1046FD01FD0B3
:10B9100083A74506130101FD232861012326110297
:10B92000232481022322910223202103232E31018B
:10B93000232C4101232A5101232671012324810153
:10B9400013972701130B06006358070A8327860005
:10B95000832B06001389050093090500930AF0FF65
:10B960006388070803AC4B0003A40B00135A2C0098
:10B9700063060A06930400006F00C000130444002D
:10B98000630C9A048325040013060900138509003B
:10B99000EF10100293841400E31255FF1305F0FF1B
:10B9A0008320C1020324810223240B0023220B00E5
:10B9B00083244102032901028329C101032A810151
:10B9C000832A4101032B0101832BC100032C810039
:10B9D000130101036780000083278B00137CCCFFD9
:10B9E000B38787412324FB00938B8B00E39C07F6EE
:10B9F000130500006FF0DFFAEF10D00C6FF05FFA64
:10BA000003278600630407006FF09FF023220600DF
:10BA10001305000067800000130101ED232E311192
:10BA2000232A51112320A11123261112232481122C
:10BA30002322911223202113232C41112328611149
:10BA4000232671112324811123229111232EB10F5A
:10BA50002326D100930A050093890500130D0600E3
:10BA600063060500832785036388076A0397C90077
:10BA7000931707019316270193D7070163CA06029C
:10BA8000B727000083A64906B367F700939707011D
:10BA900037E7FFFF93D707411307F7FF33F7E600B8
:10BAA0002396F9009397070123A2E90693D707018C
:10BAB00013F787006304073E03A709016300073EED
:10BAC00093F7A7011307A000638AE73EB7570180E9
:10BAD0009304C1049387476AB76B0180376901807B
:10BAE000232091042324010423220104138704004A
:10BAF000232801002322010223240102232601021C
:10BB000023240100232AF100938B0B81130909825E
:10BB100083470D00638E072413040D009306500223
:10BB20006386D7428347140013041400E39A07FE88
:10BB3000330AA441630EA42383268104832741048E
:10BB40002320A701B306DA009387170023224701B9
:10BB50002324D1042322F104130670001307870065
:10BB60006350F602E3840636130601049385090048
:10BB700013850A00EFF0DFD9631005201387040056
:10BB80008326810083470400B38646012324D10025
:10BB90006380071E83461400130D1400A30D0102D9
:10BBA000930CF0FF13040000930D0000130AA0058E
:10BBB000130C9000130BA002130D1D00938706FEBB
:10BBC0006364FA040326410193972700B387C700F3
:10BBD00083A707006780070013040000938706FD12
:10BBE00083460D009315240033848500131414003C
:10BBF00033848700938706FD130D1D00E372FCFE5E
:10BC0000938706FEE370FAFC638406162306D108C8
:10BC1000A30D0102130A1000130C1000130BC1082E
:10BC2000930C000093FF2D0063840F00130A2A0079
:10BC30008326410413FF4D088327810413861600D1
:10BC40009305060063160F0033084441E3440017D0
:10BC50000345B10313068700630C05029306B10385
:10BC60002320D70093871700930610002322D700C4
:10BC70002324F1042322B10413077000E342B70C1C
:10BC800093860500130706009385150013068600AA
:10BC9000638E0F049306C1032320D70093872700E8
:10BCA000930620002322D7002324F1042322B10489
:10BCB00013077000E352B70EE3840726130601044E
:10BCC0009385090013850A00232CE101EFF05FC47E
:10BCD0006314050A8326410483278104032F81010D
:10BCE0001306410593851600138704001305000809
:10BCF0006306AF68B38C8C4163429077B307FC0056
:10BD000023206701232287012324F1042322B10485
:10BD1000130770006352B7026382072413060104FD
:10BD20009385090013850A00EFF09FBE6316050492
:10BD3000832781041386040093FE4D0063860E0062
:10BD4000330C4441634880236354440113040A00C4
:10BD500003278100330787002324E100639E077ACD
:10BD600083470D002322010413870400E39607DABA
:10BD700083278104E396076283D7C90093F70704FA
:10BD8000E39E07648320C1120324811203258100EE
:10BD900083244112032901128329C111032A81112D
:10BDA000832A4111032B0111832BC110032C811015
:10BDB000832C4110032D0110832DC10F130101139A
:10BDC0006780000013850A00232CE100EFA09FF597
:10BDD00083274500138507002326F102EFC09FF358
:10BDE0009307050013850A002324F102EFA09FF3B7
:10BDF00003278500832781022322E1020327810193
:10BE0000E398072A83460D006FF01FDB83460D0081
:10BE100093ED0D026FF05FDA93ED0D0193F70D02D4
:10BE2000638A07228327C100138B7700137B8BFF64
:10BE300083264B00032C0B0093078B002326F10075
:10BE40001388060063C006249306F0FF138A0D00D2
:10BE50006388DC00B3660C0113FAFDF7E38E060677
:10BE6000E318081293069000E3E4861393070C038B
:10BE7000A307F10E930D0A00130C1000130BF10E23
:10BE8000138A0C0063D48C01130A0C008347B1039E
:10BE9000B337F000330AFA006FF0DFD8938509005A
:10BEA00013850A00EF70CFBBE31A055283D7C90090
:10BEB0001307A00093F7A701E39AE7C08397E9006F
:10BEC000E3C607C08326C10013060D009385090051
:10BED00013850A00EF0010562324A1006FF09FEA9B
:10BEE00093ED0D0193F70D02638007148327C100C2
:10BEF000138B7700137B8BFF032C0B0003284B0065
:10BF000093078B002326F10013FAFDBF9306000070
:10BF1000A30D01021306F0FF638ACC1833660C01EF
:10BF2000937DFAF76314066863960C3E639A067A6B
:10BF3000137C1A00130B010FE3040CF493070003A6
:10BF4000A307F10E130BF10E6FF09FF3330AA44118
:10BF5000E314A4BF834704006FF09FC323220104AE
:10BF600093FE4D0063800E72330C4441635C80711C
:10BF7000138604001307000183264104E358874514
:10BF8000930C0001130B70006F0080019385260055
:10BF90001306860093060700130C0CFF63D88C056C
:10BFA0009387070113871600232076012322960129
:10BFB0002324F1042322E104E35AEBFC6388073ACB
:10BFC000130601049385090013850A00EFF05F94BE
:10BFD000E31405DA83264104130C0CFF8327810444
:10BFE0001386040093851600E3CC8CFBB38787018E
:10BFF00023207601232286012324F1042322B10485
:10C0000013077000E352B7D4638E0766130601046A
:10C010009385090013850A00EFF09F8FE31E05D476
:10C02000832781046FF05FD20326C10093F70D01CF
:10C0300093064600E390070C93F70D04E38E072464
:10C040008327C100130800002326D10003DC07006A
:10C050006FF09FEB0326C10093F70D019306460096
:10C06000E390070893F70D04E38807208327C100B6
:10C070002326D100039C07001358FC4193060800B7
:10C08000E3D406DCB3368001330800413308D840DE
:10C090009306D002A30DD1021306F0FF330C8041AA
:10C0A000138A0D0093061000E39ACCE613061000E5
:10C0B000E388C6DA130620006388C626130B010F37
:10C0C0001316D80193767C0093573C0093860603A1
:10C0D000336CF60013583800A30FDBFE33660C01F7
:10C0E00093050B00130BFBFFE31C06FC93771A0070
:10C0F00063860726930700036382F6269385E5FF90
:10C10000A30FFBFE9307010F338CB740930D0A007A
:10C11000138B05006FF0DFD6EF701FA76FF01F9530
:10C120008327C100A30D010203AB070093864700DC
:10C13000E3040B129307F0FFE38CFC0613860C005C
:10C140009305000013050B00232CD1002326E100EA
:10C15000EFB04FD90327C10083268101E30C0524EA
:10C16000330C65412326D100930C00006FF05FD1A2
:10C170008326C100A30D0102130A100083A7060045
:10C18000938646002326D1002306F108130C1000E5
:10C19000130BC1086FF0DFA883460D009307C0069C
:10C1A000E38EF60893ED0D016FF01FA183460D009D
:10C1B00093078006E38CF60693ED0D046FF0DF9F86
:10C1C00013EA0D0193770A02638407528327C100A3
:10C1D00093061000138B7700137B8BFF93078B0064
:10C1E000032C0B0003284B002326F1006FF05FD2D5
:10C1F00083460D0093ED0D086FF01F9C8327C1004F
:10C2000013EA2D00B786FFFF03AC0700B75D01807E
:10C210009387470093C606832326F10093878DF406
:10C22000231ED102130800002328F10093062000EA
:10C230006FF01FCE0326C10093F70D028326060080
:10C24000130646002326C1006392076893F70D0189
:10C25000639E077E93F70D04E392070E93FE0D2075
:10C2600063860E7E832781002380F6006FF05F8A4D
:10C270008327C10083460D0003A40700938747006E
:10C280002326F100E35A04923304804093ED4D00DD
:10C290006FF09F9283460D0093ED1D006FF0DF91CC
:10C2A0008347B10383460D00E3980790930700028C
:10C2B000A30DF1026FF05F9083460D0093ED4D00EA
:10C2C0006FF09F8F9307B00283460D00A30DF1021C
:10C2D0006FF09F8E83460D0093051D00E38C661161
:10C2E000938706FD138D0500930C0000E368FC8C1A
:10C2F00083460D0013982C0033089801131818007A
:10C30000B30CF800938706FD130D1D00E372FCFECD
:10C310006FF0DF8A13061000E38EC60A13062000B2
:10C32000138A0D00E39CC6D8130B010F832701016C
:10C330009376FC00130BFBFFB386D70003C6060001
:10C3400093574C009316C80133ECF600135848007D
:10C350002300CB00B3660C01E39A06FC9307010FA0
:10C36000338C6741930D0A006FF09FB19305100065
:10C3700093060000138604006FF01FC23308444187
:10C38000E35A009713050001E3500507130F00015E
:10C39000930F70006F00800113852600130787003C
:10C3A00093060600130808FF63500F0793870701E1
:10C3B00013861600232027012322E7012324F104FA
:10C3C0002322C104E3DACFFC6384071613060104B9
:10C3D0009385090013850A00232C0101EFF04FD348
:10C3E000E31C05980328810183264104130F0001F3
:10C3F000130808FF832781041387040013851600A0
:10C40000930F7000E3440FFB130F8700B3870701FE
:10C4100023202701232207012324F1042322A1043E
:10C42000130770006352A746638E076C130601045E
:10C430009385090013850A00EFF08FCDE31E059266
:10C4400083264104B38C8C41832781041306410564
:10C450009385160013870400E352908B13050001A7
:10C460006358956913030001130F70006F0080017A
:10C47000938526001307870093060600938C0CFF14
:10C48000635C930593870701138616002320270119
:10C49000232267002324F1042322C104E35ACFFCA2
:10C4A00063840706130601049385090013850A00B7
:10C4B000EFF00FC6E312058C83264104130300013D
:10C4C000938C0CFF83278104138704009385160047
:10C4D000130F7000E34893FB93068700B38797011F
:10C4E00023202701232297012324F1042322B104CE
:10C4F000130770006344B71A9385150013868600EE
:10C50000138706006FF08FFF93051000930600005D
:10C51000138704006FF09FF613060104938509004A
:10C5200013850A00EFF0CFBEE30C05826FF0DF84C5
:10C530001305100093060000138704006FF09FE6B8
:10C54000638A071E130601049385090013850A00F8
:10C55000232EE101232CF101EFF08FBBE31E0580B8
:10C560008326410483278104032FC101832F810186
:10C570001306410593851600138704006FF04FF1F1
:10C580009307C1032326F104930720002328F10415
:10C590009305100013064105938605001307060056
:10C5A00093851600130687006FF04FF4138A0D0071
:10C5B0006FF0DFAF9305000163D6056193020001C0
:10C5C000930370006F00C0011385260013078700D6
:10C5D00093060600130808FF63D8020713861600A7
:10C5E0009387070123207701232257002324F10496
:10C5F0002322C104E3DAC3FC638E07061306010499
:10C600009385090013850A0023200103232EE101ED
:10C61000232CF101EFF0CFAF631005F603280102E0
:10C620008326410493020001130808FF8327810435
:10C63000032FC101832F8101138704001385160086
:10C6400093037000E3CC02F9B3870701232077013D
:10C65000232207012324F1042322A104930670005E
:10C6600063CAA60E130787009305150093060500FD
:10C670006FF00FDE9306000013051000138704000F
:10C680006FF05FF56354440113040A0083278100AF
:10C69000B38787002324F1006FF08FEC638A07349F
:10C6A000130601049385090013850A00EFF04FA6D5
:10C6B000631405EC83254104832781041306410597
:10C6C00093851500138704006FF04FE323220104C4
:10C6D000138704006FF0CFCA639A0CF8930D0A0019
:10C6E000930C0000130C0000130B010F6FF04FF9B7
:10C6F0000326C10093770A01930646006390071A48
:10C7000093770A046386073C8327C100130800005F
:10C710002326D10003DC0700930610006FF04FFFC3
:10C7200013064105930510009306000013870400CB
:10C730006FF0CFDB63880F1C9307C1032326F1043E
:10C74000930720002328F1049306100013074105E6
:10C750006FF01FE5638E0726130601049385090019
:10C7600013850A00232EE101232CF101EFF04F9AEB
:10C77000631405E08326410483278104032FC1014C
:10C78000832F810113870400938516006FF04FCC2F
:10C7900093770A402320F102930D0000130B010F41
:10C7A0006F004003930508001306A00093060000E5
:10C7B00013050C00232EE100232C0101EF30C030C3
:10C7C000032881010327C10163080832130C050007
:10C7D00013880500930508001306A00093060000C7
:10C7E00013050C00232EE100232C0101EF30007112
:10C7F0008327010213050503A30FABFE0328810164
:10C800000327C101130BFBFF938D1D00E38C07F879
:10C810008327410283C60700E396B6F99307F00F1A
:10C82000E382FDF86316080093079000E3F887B3EE
:10C83000832781028325C102232E0101330BFB4094
:10C840001386070013050B00232CE100EFC04FD522
:10C85000032741020328C1011306A00083451700E6
:10C860009306000013050C00B337B000B307F700C0
:10C87000930508002322F102EF30002503278101F0
:10C88000930D00006FF09FF49305150013068F00C1
:10C890009306050013070F006FF0CFC52326D100C4
:10C8A000032C060013080000930610006FF04FE6FB
:10C8B0008327410283460D00638007B083C70700CA
:10C8C000638C07AE93ED0D406FF00FAF0326810030
:10C8D0009357F64123A0C60023A2F6006FF04FA3A2
:10C8E000032C06002326D1001358FC4193060800B0
:10C8F0006FF04FD5032C0600130800002326D1004B
:10C900006FF08FE0930600001306410593051000B9
:10C91000138704006FF08FBDB75701809387C7F569
:10C920002328F10093F70D02638407068327C100D3
:10C93000138B7700137B8BFF032C0B0003284B001A
:10C9400093078B002326F10013F61D00630E0600EB
:10C9500033660C01630A060013060003230EC102AE
:10C96000A30ED10293ED2D0013FAFDBF9306200014
:10C970006FF00FDA138A0D006FF0DF84B757018074
:10C98000938787F42328F10093F70D02E39007FAC9
:10C990008325C10093F70D0113864500638A0706BE
:10C9A00003AC0500130800002326C1006FF0DFF977
:10C9B00013050B00232CE1002326D100EFC08FB517
:10C9C00003278101130C0500930C00006FF04FCB7F
:10C9D0000347B10363160714E3940FBA93060000EC
:10C9E0009305100013064105138704006FF00FB084
:10C9F0001307100093070C002326610523288105E7
:10CA0000232481052322E104130641056FF0CFB2F0
:10CA100093F70D046380070A8327C1001308000001
:10CA20002326C10003DC07006FF01FF283461D00C0
:10CA300093ED0D20130D1D006FF00F9883461D0020
:10CA400093ED0D02130D1D006FF00F9783278100EA
:10CA500023A0F6006FF0CF8B93076000138C0C00BF
:10CA600063EC970BB7580180130A0C002326D10002
:10CA7000138B08F76FF0CF9A93F70D20638607109A
:10CA80008327C1002326D100038C07001358FC41E3
:10CA9000930608006FF00FBB93F70D20638C070C13
:10CAA0008327C100130800002326D10003CC070010
:10CAB0006FF08FC593F70D206384070A8327C100A9
:10CAC000130800002326C10003CC07006FF0DFE746
:10CAD00093770A20638A07068327C10013080000A2
:10CAE0002326D10003CC0700930610006FF04FC23D
:10CAF000930606006FF09F9E93079000E3E887CDB2
:10CB00006FF0DF85130641059305100093060000C2
:10CB1000138704006FF00F9E130C60006FF09FF4FA
:10CB20009307B1032326F104930710002328F1048F
:10CB300093051000130641056FF08F948327810041
:10CB40002390F6006FE0DFFC8327C100130800008C
:10CB50002326D10003AC0700930610006FF04FBBF3
:10CB60008327C100130800002326C10003AC07007F
:10CB70006FF09FDD8327C100130800002326D1003A
:10CB800003AC07006FF04FB88327C1002326D10004
:10CB900003AC07001358FC41930608006FF08FAAFE
:10CBA000130601049385090013850A00EFE05FD6A0
:10CBB0006FF08F9C138C0C002326D100930C000087
:10CBC0006FF00FAC130506006FF01FA893851600D9
:10CBD0006FF0CFC1138A0D006FF04FA99307F0FFDC
:10CBE0002324F1006FF00F9A130F06001385050040
:10CBF0006FF0DF818327C10083AC07009387470074
:10CC000063D40C00930CF0FF83461D002326F10033
:10CC1000138D05006FE05FFA3777018093070500F9
:10CC20000325479C9306060013860500938507009D
:10CC30006FE09FDE83D7C50003AE450603D3E50052
:10CC400083A8C50103A84502130101B893F7D7FFD4
:10CC500013070040232C8146231AF100138405009A
:10CC60009307010793058100232A91462328214732
:10CC7000232E1146130905002326C107231B61003B
:10CC800023221103232601032324F100232CF10086
:10CC90002328E100232EE10023200102EFE0DFD76B
:10CCA00093040500635C05028357410193F7070471
:10CCB000638807008357C40093E707042316F40032
:10CCC0008320C147032481470329014713850400BA
:10CCD00083244147130101486780000093058100C8
:10CCE00013050900EF609FAFE30005FC9304F0FF1C
:10CCF0006FF09FFB130101FF1387050023248100C0
:10CD0000232291009305060013040500B7740180E7
:10CD100013860600130507002326110023A204A092
:10CD2000EF300FBF9307F0FF630CF5008320C100C5
:10CD30000324810083244100130101016780000066
:10CD400083A744A0E38407FE8320C1002320F400CE
:10CD50000324810083244100130101016780000046
:10CD6000B777018003A7479C130101FF9387060053
:10CD700013080600232611008328C7009306050028
:10CD8000138705001386070063000802B767018058
:10CD900093870783B7650180938505841385080011
:10CDA000EF004029EF20D01C376801809307C8832B
:10CDB0001308C8836FF01FFE130101FF93060600DE
:10CDC0001306000023261100EFF09FF9B385C5027A
:10CDD000130101FF2324810023261100EFA00F95EA
:10CDE00013040500630805020326C5FF130740026C
:10CDF0001376C6FF1306C6FF6360C70693063001AD
:10CE00009307050063E2C60223A0070023A20700E0
:10CE100023A407008320C10013050400032481001C
:10CE20001301010167800000232005002322050073
:10CE30009307B00163F0C7042324050023260500EF
:10CE400093070501E312E6FC2328050093078501FB
:10CE5000232A05006FF05FFB93050000EF300FE819
:10CE60008320C10013050400032481001301010184
:10CE700067800000930785006FF01FF9130101FF21
:10CE8000232481002322910013040500B77401803C
:10CE9000138505002326110023A204A0EF304FA420
:10CEA0009307F0FF630CF5008320C1000324810089
:10CEB00083244100130101016780000083A744A07F
:10CEC000E38407FE8320C1002320F40003248100B3
:10CED000832441001301010167800000130101FF59
:10CEE00023261100232481002322910023202101E5
:10CEF00063800502138405009304050063060500A2
:10CF000083278503638C070A8317C4006392070293
:10CF10008320C10003248100130900008324410001
:10CF200013050900032901001301010167800000B6
:10CF30009305040013850400EF608FE48327C40287
:10CF400013090500638A07008325C40113850400C3
:10CF5000E7800700634C05068357C40093F7070872
:10CF6000639E070683250403638C0500930704046E
:10CF70006386F50013850400EF609FD9232804021F
:10CF8000832544046388050013850400EF605FD89F
:10CF900023220404EF605FC023160400EF601FC06B
:10CFA0008320C1000324810083244100130509006C
:10CFB000032901001301010167800000EF60DFBC5D
:10CFC0008317C400E38607F46FF09FF68357C4000D
:10CFD0001309F0FF93F70708E38607F88325040198
:10CFE00013850400EF60DFD26FF0DFF7B7770180C1
:10CFF0009305050003A5479C6FF05FEE130101FC4C
:10D000001303C1022326D10293060300232E11002D
:10D010002328E102232AF102232C0103232E1103EA
:10D0200023266100EFE05F9F8320C101130101040B
:10D0300067800000130E050037750180130101FCA5
:10D040000325459C130381022324C1022326D10218
:10D05000138605009306030093050E00232E11008E
:10D060002328E102232AF102232C0103232E11039A
:10D0700023266100EFE05F9A8320C10113010104C0
:10D0800067800000130101FD23248102232E31015A
:10D090002328610123261102232291022320210348
:10D0A000232C4101232A5101130B0500938905000C
:10D0B00013040600EF004079930710006310F50297
:10D0C0009387F9FF1307E00F636AF70013F7F90F6F
:10D0D0002306E100130910006F00C0029306C40587
:10D0E000138609009305C10013050B00EF20C05300
:10D0F0009307F0FF130905006304F50A630E0508A2
:10D100000347C10093040000130AF0FF930AA00034
:10D110006F00800283270400938617002320D40029
:10D120002380E700938414009307C100B38797001E
:10D1300063F4240703C70700832784009387F7FF5E
:10D140002324F400E3D807FC832684019305070019
:10D150001306040013050B0063C4D700E31C57FB40
:10D16000EF20C032E31045FD1309F0FF8320C10218
:10D1700003248102832441028329C101032A8101FE
:10D18000832A4101032B0101130509000329010230
:10D190001301010367800000138909006FF01FFD70
:10D1A0008357C40093E707042316F4006FF01FFCB5
:10D1B0008317C6001397270163400702032746061B
:10D1C000B7260000B3E7D700B72600003367D700C3
:10D1D0002316F6002322E6066FF0DFEA130101FEB4
:10D1E000B7770180232C810003A4479C232E1100D4
:10D1F0001386050093050500630604008327840356
:10D20000638007048317C600139727016340070252
:10D2100003274606B7260000B3E7D700B72600006D
:10D220003367D7002316F6002322E6061305040011
:10D23000032481018320C101130101026FF09FE4E7
:10D240002324A100130504002326C100EF60DF930F
:10D250000326C100832581006FF0DFFA130101FF6F
:10D260001387050023248100232291001304050065
:10D27000B7740180930506001305070023261100EB
:10D2800023A204A0EF205FE69307F0FF630CF500F4
:10D290008320C10003248100832441001301010184
:10D2A0006780000083A744A0E38407FE8320C100B9
:10D2B0002320F40003248100832441001301010191
:10D2C0006780000083278600638E073283D7C500FE
:10D2D000130101FD23248102232C4101232A510142
:10D2E000232611022322910223202103232E310120
:10D2F0002328610123267101232481012322910126
:10D300002320A10113F78700130A0600930A0500E2
:10D31000138405006306070803A7050163020708D5
:10D3200013F7270083240A00630C070883274402AD
:10D330008325C401370B0080930900001309000006
:10D34000134B0BC01386090013850A0063020904FE
:10D350009306090063742B0193060B00E780070016
:10D360006358A02883278A00B389A9003309A940FC
:10D370003385A7402324AA00630A0520832744029B
:10D380008325C4011386090013850A00E31209FCF2
:10D3900083A9040003A94400938484006FF09FFADA
:10D3A0009305040013850A00EF509FEB631C053AB8
:10D3B0008357C40083240A0013F72700E31807F6F5
:10D3C00013F7170063140724832C8400032504003B
:10D3D000370B0080934BEBFF130C00001309000088
:10D3E000134BFBFF630E090E13F70720630C072492
:10D3F000138D0C006362992F13F70748630A07081F
:10D400008329440183250401130719009396190009
:10D41000B386360193D9F601330DB540B389D900EF
:10D4200093D919403307A7011386090063F6E90071
:10D43000930907001306070093F707406384072E3C
:10D440009305060013850A00EF905FAE930C05006C
:10D45000630205308325040113060D00EF00004F21
:10D460008357C40093F7F7B793E707082316F40030
:10D470003385AC01B387A941232894012320A4005C
:10D48000232A3401930C09002324F400130D09000E
:10D4900013060D0093050C00EF00005D03278400C8
:10D4A0008327040093090900B30C9741B387A701B0
:10D4B000232494012320F4001309000003268A008A
:10D4C000330C3C01B309364123243A016380090C33
:10D4D000832C8400032504008357C400E31609F05D
:10D4E00003AC040003A94400938484006FF09FEF11
:10D4F00083A9440003AC040093848400E38A09FEFA
:10D50000138609009305A00013050C00EFA08F9D62
:10D510006304051213051500330B854193070B00B7
:10D52000938B090063F43701938B070003250400F4
:10D53000832704018326440163F8A700032984009C
:10D54000338926016342790963C8DB1A83274402C1
:10D550008325C40113060C0013850A00E780070029
:10D56000130905006356A008330B2B411305100067
:10D57000630A0B1603268A00330C2C01B389294158
:10D580003309264123242A01631A090813050000E0
:10D590008320C10203248102832441020329010262
:10D5A0008329C101032A8101832A4101032B01013F
:10D5B000832BC100032C8100832C4100032D01002B
:10D5C000130101036780000093050C001306090096
:10D5D000EF008049832704009305040013850A00A7
:10D5E000B38727012320F400EF604F9FE30E05F679
:10D5F0008317C40093E707042316F4001305F0FF14
:10D600006FF01FF91305000067800000130B000086
:10D6100013050000130C000093090000E38A09ECD5
:10D62000E31E05EE138609009305A00013050C0008
:10D63000EFA04F8BE31005EE93871900138B0700C3
:10D640006FF01FEE8327040163E2A70483274401E0
:10D65000636EF9029306090063F42B0193060B0035
:10D66000B3C6F602032744028325C40113060C0047
:10D6700013850A00B386F602E70007009309050048
:10D68000E358A0F6330939416FF05FE393890C004A
:10D6900063749901930909001386090093050C002E
:10D6A000EF00803C8327840003270400B3873741C1
:10D6B000330737012324F4002320E400E39407FC1C
:10D6C0009305040013850A00EF604F91E31205F201
:10D6D000330939416FF09FDE930C0900130D0900E7
:10D6E0006FF01FDB9305040013850A00EF600F8FB6
:10D6F000E30205E86FF0DFEF13860B0093050C00E3
:10D70000EF008036832784000326040013890B0072
:10D71000B3877741330676012324F4002320C40025
:10D720006FF09FE413850A00EF00C04C930C0500D6
:10D73000E31005D48325040113850A00EF604FDD53
:10D740008317C4001307C00023A0EA0093F7F7F77C
:10D750006FF05FEA1307C0008317C40023A0EA003C
:10D760006FF05FE91305F0FF6FF09FE2130101FF17
:10D77000232481002322910013040500B774018043
:10D78000138505002326110023A204A0EF205F9635
:10D790009307F0FF630CF5008320C1000324810090
:10D7A00083244100130101016780000083A744A086
:10D7B000E38407FE8320C1002320F40003248100BA
:10D7C000832441001301010167800000130101FF60
:10D7D000232611002324810023229100630C0602DA
:10D7E000B76501809385458713050600130406007D
:10D7F000EF00D017B7640180631205021385048718
:10D800008320C1000324810083244100130101010E
:10D8100067800000B76401806FF05FFE9385048726
:10D8200013050400EF009014E30A05FCB7650180BE
:10D830009385C58313050400EF005013E30005FC36
:10D84000130500006FF0DFFBB777018003C5079673
:10D850006780000037770180930705000325479C08
:10D8600013860500938507006FF05FF6130101FF33
:10D8700013870500232481002322910093050600CD
:10D8800013040500B7740180138606001305070012
:10D890002326110023A204A0EF201F869307F0FF88
:10D8A000630CF5008320C100032481008324410020
:10D8B000130101016780000083A744A0E38407FEF1
:10D8C0008320C1002320F40003248100832441002D
:10D8D0001301010167800000B777018003A3C7919E
:10D8E0006700030063800502630206046388060480
:10D8F0008347060023A0F500034506003335A0004A
:10D9000067800000130101FF9305C1006304060254
:10D91000638A06028347060023A0F500034506003C
:10D920003335A000130101016780000013050000DA
:10D9300067800000130500006FF0DFFE1305E0FFB5
:10D94000678000001305E0FF6FF0DFFDB3C7A5009F
:10D9500093F73700B308C5006392070693073000BA
:10D9600063FEC70493773500130705006398070625
:10D9700013F6C8FF930706FE636CF708637CC702C3
:10D98000938605009307070003A8060093874700C6
:10D990009386460023AE07FFE3E8C7FE9307F6FF32
:10D9A000B387E74093F7C7FF938747003307F70034
:10D9B000B385F50063681701678000001307050051
:10D9C000E37C15FF83C70500130717009385150037
:10D9D000A30FF7FEE36817FF6780000083C605000A
:10D9E0001307170093773700A30FD7FE9385150011
:10D9F000E38007F883C60500130717009377370005
:10DA0000A30FD7FE93851500E39A07FC6FF05FF62E
:10DA100083A6450083A2050083AF850003AFC50040
:10DA200083AE050103AE450103A3850103A8C5012B
:10DA30002322D70083A60502232057002324F701C1
:10DA40002326E7012328D701232AC701232C6700B7
:10DA5000232E07012320D70213074702938545028F
:10DA6000E368F7FA6FF09FF163F6A502B387C5008C
:10DA70006372F5023307C500630A060E83C6F7FF1B
:10DA80009387F7FF1307F7FF2300D700E398F5FE0E
:10DA9000678000009307F00063E8C7029307050062
:10DAA0009306F6FF630C060C93861600B386D70028
:10DAB00003C705009387170093851500A38FE7FE22
:10DAC000E398D7FE67800000B3E7A50093F737001F
:10DAD0006390070A930806FF93F808FF93880801EC
:10DAE00033081501138705009307050083260700F7
:10DAF000130707019387070123A8D7FE832647FF53
:10DB000023AAD7FE832687FF23ACD7FE8326C7FF31
:10DB100023AED7FEE31CF8FC1377C600B3851501CE
:10DB20001378F600630E0704138705009388070037
:10DB3000130E30000323070013074700B306E84025
:10DB400023A06800B386D50093884800E364DEFE16
:10DB50001307C8FF1377C7FF130747001376360074
:10DB6000B387E700B385E5006FF09FF3678000009F
:10DB70009306F6FF930705006FF01FF36780000020
:10DB8000130608006FF0DFF1130101FF1387050092
:10DB9000232481002322910093050600130405002D
:10DBA000B7740180138606001305070023261100B1
:10DBB00023A204A0EF20CFD49307F0FF630CF5005D
:10DBC0008320C1000324810083244100130101014B
:10DBD0006780000083A744A0E38407FE8320C10080
:10DBE0002320F40003248100832441001301010158
:10DBF00067800000130101FD232021032326110269
:10DC00002324810223229102232E3101232C41015E
:10DC1000232A510123286101232671012324810134
:10DC20001309060063840522138405009309050087
:10DC3000EF909FB89304B9009307600163FE970EBD
:10DC400093F484FF1387040063CE040E63EC240F67
:10DC50008327C4FF930A84FF13FAC7FF338B4A015B
:10DC6000635CEA18B7660180938B064303A68B00BA
:10DC700083264B00630E662313F6E6FF3306CB00C4
:10DC800003264600137616006314061A93F6C6FFA1
:10DC90003306DA00635EE63293F7170063940702F7
:10DCA000032C84FF338C8A4183274C0093F7C7FFF2
:10DCB000B386D700B38B460163DAEB34B30BFA00BB
:10DCC00063D2EB0C9305090013850900EF900FA6B2
:10DCD00013090500630C05048327C4FF130785FFA0
:10DCE00093F7E7FFB387FA006382E7301306CAFFB2
:10DCF0009307400263E6C730130730018326040010
:10DD0000636CC726930705001307040023A0D70000
:10DD10008326470023A2D7000327870023A4E70018
:10DD20009305040013850900EF509FFE1385090039
:10DD3000EF90DFA86F00C0019304000113070001FA
:10DD4000E3F824F19307C00023A0F90013090000B1
:10DD50008320C10203248102832441028329C1015B
:10DD6000032A8101832A4101032B0101832BC10076
:10DD7000032C81001305090003290102130101038B
:10DD8000678000008327CC0003278C001306CAFF9E
:10DD9000930640022326F70023A4E70013098C0012
:10DDA000330B7C0163E4C62E930530010327040086
:10DDB0009307090063F2C5022324EC000327440003
:10DDC0009307B0012326EC0063E2C73003278400E9
:10DDD00093070C011304840023A0E70003274400E9
:10DDE000138A0B00930A0C0023A2E7000327840088
:10DDF0001304090023A4E70083A74A0033079A40CD
:10DE00009306F00093F7170063ECE606B367FA0099
:10DE100023A2FA0083274B0093E717002322FB007D
:10DE200013850900EF909F99130904006FF05FF2CA
:10DE300093F71700E39807E8032C84FF338C8A419B
:10DE400083274C0093F7C7FF6FF05FE7032481023D
:10DE50008320C10283244102032901028329C101D5
:10DE6000032A8101832A4101032B0101832BC10075
:10DE7000032C810093050600130101036F900F8BA3
:10DE8000B3E7970023A2FA00B3859A00136717003F
:10DE900023A2E50083274B009385850013850900A5
:10DEA00093E717002322FB00EF509FE66FF05FF728
:10DEB00093F6C6FF3306DA00938504016350B60E6D
:10DEC00093F71700E39007E0032C84FF338C8A411B
:10DED00083274C0093F7C7FFB386D700338B4601E7
:10DEE000E34EBBDC8327CC0003278C001306CAFF5C
:10DEF000930640022326F70023A4E70013098C00B1
:10DF000063EEC62093053001032704009307090040
:10DF100063F2C5022324EC00032744009307B001F9
:10DF20002326EC0063E4C7200327840093070C0139
:10DF30001304840023A0E7000327440023A2E70082
:10DF40000327840023A4E70033079C00B3079B400A
:10DF500023A4EB0093E717002322F70083274C004C
:10DF60001385090093F71700B3E4970023229C0060
:10DF7000EF90DF846FF0DFDD2320D500832644009F
:10DF80001307B0012322D5006360C71283268400E3
:10DF900013078400930785006FF05FD7B38A9A0058
:10DFA000B307964023A45B0193E7170023A2FA006E
:10DFB0008327C4FF138509001309040093F7170092
:10DFC000B3E49700232E94FEEF904FFF6FF05FD8DD
:10DFD0008327CB0003278B00130A0600338BCA006C
:10DFE0002326F70023A4E7006FF01FE18327C5FF76
:10DFF00093F7C7FF330AFA00338B4A016FF0DFDF74
:10E0000093050400EFF05FA66FF09FD18327CB004C
:10E0100003278B001306CAFF930640022326F7004E
:10E0200023A4E70003278C008327CC0013098C006E
:10E03000330B7C012326F70023A4E70063E8C60422
:10E04000930630010327040093070900E3F6C6D8BE
:10E050002324EC00032744009307B0012326EC009F
:10E0600003278400E3F6C7D62328EC000327C40067
:10E0700093074002232AEC00032704016304F606F9
:10E0800093078C01130404016FF01FD5930504005E
:10E0900013050900EFF05F9D13040900138A0B00BC
:10E0A000930A0C006FF05FD5032784002324E5005A
:10E0B0000327C4002326E500832604016302F60437
:10E0C00013070401930705016FF05FC483278400E1
:10E0D0002328FC008327C400232AFC000327040113
:10E0E000E310D6FA232CEC000327440193070C021B
:10E0F00013048401232EEC00032704006FF0DFCD0E
:10E100002328D50083264401130784019307850142
:10E11000232AD500832684016FF05FBF9305040096
:10E1200013050900EFF05F946FF01FE2832784006E
:10E130002328FC008327C400232AFC0003270401B2
:10E140006308D60093078C01130404016FF09FDE6F
:10E15000232CEC000327440193070C0213048401D1
:10E16000232EEC00032704006FF0DFDC3367B500DB
:10E170009303F0FF1377370063100710B7877F7F93
:10E180009387F7F70326050083A60500B372F60010
:10E190003363F600B382F200B3E26200639272105E
:10E1A0006316D6080326450083A64500B372F60021
:10E1B0003363F600B382F200B3E26200639E720C36
:10E1C0006316D6060326850083A68500B372F60083
:10E1D0003363F600B382F200B3E262006398720C1C
:10E1E0006316D6040326C50083A6C500B372F600E5
:10E1F0003363F600B382F200B3E262006392720C02
:10E200006316D6020326050183A60501B372F60044
:10E210003363F600B382F200B3E26200639C720AD9
:10E220001305450193854501E30ED6F41317060146
:10E2300093970601631EF7001357060193D7060153
:10E240003305F7409375F50F639005026780000072
:10E250001357070193D707013305F7409375F50F5F
:10E2600063940500678000001377F70F93F7F70FAB
:10E270003305F740678000000346050083C60500AC
:10E2800013051500938515006314D600E31606FEEA
:10E290003305D6406780000013054500938545008F
:10E2A000E31CD6FC13050000678000001305850001
:10E2B00093858500E312D6FC1305000067800000FB
:10E2C0001305C5009385C500E318D6FA13050000B1
:10E2D000678000001305050193850501E31ED6F84C
:10E2E000130500006780000083278600130101FDED
:10E2F000232A510123261102232481022322910281
:10E3000023202103232E3101232C410123286101E5
:10E310002326710123248101930A060063880714D0
:10E32000130B05008329060003A5050083A48500BF
:10E33000138405006F00400D8357C40013F707488E
:10E34000630A070883264401832504011307190083
:10E3500093941600B386D40093D4F601330AB540E3
:10E36000B384D40093D414403307470113860400C8
:10E3700063F6E400930407001306070093F70740D1
:10E380006386070A9305060013050B00EF801FBA8A
:10E39000130C0500630A050A8325040113060A000D
:10E3A000EFF0CFDA8357C40093F7F7B793E7070886
:10E3B0002316F40033054C01338A4441232A940088
:10E3C00023244401232884012320A400930409006A
:10E3D000130A090013060A0093850B00EFF0CFE83B
:10E3E000032784000325040083A78A00B304974011
:10E3F00033054501232494002320A40033892741B9
:10E4000023A42A016304090603A9490083AB090078
:10E41000138A040093898900E30809FEE37E99F0DA
:10E4200093040900130A09006FF0DFFA13050B00CB
:10E43000EFF04FFC130C0500E31E05F683250401E5
:10E4400013050B00EF50DF8C9307C0002320FB0067
:10E450008357C4001305F0FF93E707042316F40065
:10E4600023A40A0023A20A006F00C00023A20A000E
:10E47000130500008320C10203248102832441028A
:10E48000032901028329C101032A8101832A410151
:10E49000032B0101832BC100032C81001301010315
:10E4A0006780000083D7C500130101ED232C4111C3
:10E4B000232861112320A111232611122324811264
:10E4C0002322911223202113232E3111232A5111AB
:10E4D000232671112324811123229111232EB10FA0
:10E4E00093F707082326D100138A0500130B0500B4
:10E4F000130D06006386070083A70501E386075610
:10E50000B7670180930AC10493870788B76B0180BE
:10E51000B764018023205105232401042322010430
:10E5200013870A0023280100232201022324010269
:10E530002326010223240100232AF100938BCB9E82
:10E540009384C49F83470D006380072013040D004C
:10E55000930650026386D7388347140013041400CF
:10E56000E39A07FE3309A4416300A41F83268104B4
:10E57000832741042320A701B38626019387170030
:10E58000232227012324D1042322F10493067000BF
:10E590001307870063CEF634832681008347040087
:10E5A000B38626012324D1006380071A8346140012
:10E5B000130D1400A30D0102930CF0FF13040000CF
:10E5C000930D00001309A005130C90009309A002FD
:10E5D000130D1D00938706FE6364F90403264101B1
:10E5E00093972700B387C70083A7070067800700BA
:10E5F00013040000938706FD83460D009315240045
:10E60000338485001314140033848700938706FD38
:10E61000130D1D00E372FCFE938706FEE370F9FC08
:10E62000638406122306D108A30D0102130910000A
:10E63000130C10009309C108930C000013FF2D0068
:10E6400063040F001309290013FE4D08832781047A
:10E650000326410463160E00B3062441E34AD002A8
:10E660008346B103130516009305870063800604F3
:10E670009306B103938717002320D7009306100059
:10E680002322D7002324F1042322A104930670003F
:10E69000E3CEA60C930F2600930607011306050090
:10E6A0001387050013850F0093850600630C0F0286
:10E6B0009306C1032320D7009387270093062000E9
:10E6C0002322D7002324F1042322A104130770007E
:10E6D000E34CA70C1306050013870500130515006E
:10E6E00093858500930600086302DE60B38C8C413D
:10E6F0006346906BB307FC00232037012322870178
:10E700002324F1042322A104130770006342A77499
:10E7100093F84D0063860800330C24416348801F42
:10E720006354240113040900032781003307870081
:10E730002324E100639E077283470D002322010416
:10E7400013870A00E39407E083278104E392074CD0
:10E750008357CA0093F70704E398074E8320C1123A
:10E76000032481120325810083244112032901120D
:10E770008329C111032A8111832A4111032B01111D
:10E78000832BC110032C8110832C4110032D011009
:10E79000832DC10F130101136780000013050B00C7
:10E7A000232CE100EF800FD8832745001385070055
:10E7B0002326F102EFA00FD69307050013050B00E7
:10E7C0002324F102EF800FD60327850083278102DF
:10E7D0002322E10203278101E398071683460D00F7
:10E7E0006FF01FDF83460D0093ED0D026FF05FDECB
:10E7F00093ED0D0193F70D026382071E8327C1007D
:10E800009389770093F989FF83A6490003AC090037
:10E81000938789002326F100138E060063C8061E25
:10E820009306F0FF13890D006388DC00B366CC010A
:10E8300013F9FDF76384067AE31C0E00930690003B
:10E84000E3E8860193070C03A307F10E930D09007B
:10E85000130C10009309F10E6F00C00693ED0D012B
:10E8600093F70D02638607148327C100938977000D
:10E8700093F989FF03AC090003AE4900938789002F
:10E880002326F10013F9FDBF93060000A30D01023A
:10E890001306F0FF6380CC1A3366CC01937DF9F741
:10E8A0006314065E63980C3E639E0672137C190027
:10E8B0009309010F63080C0093070003A307F10EEF
:10E8C0009309F10E13890C0063D48C0113090C0019
:10E8D0008347B103B337F0003309F9006FF01FD657
:10E8E0003309A441E314A4C9834704006FF0DFCBCC
:10E8F0001306010493050A0013050B00EFF0DF9ED9
:10E90000E31805E413870A006FF01FC9930600019E
:10E910000327410463D08607930C0001930970001C
:10E920006F00C000130C0CFF63D68C0593870701A2
:10E930001307170023A0750123A295012324F104D6
:10E940002322E10493858500E3DEE9FC130601043C
:10E9500093050A0013050B00EFF01F99E31A05DE7B
:10E96000130C0CFF832781040327410493850A00BD
:10E97000E3CE8CFBB38787011307170023A0750133
:10E9800023A285012324F1042322E10493067000CD
:10E99000E3D8E6D81306010493050A0013050B001B
:10E9A000EFF09F94E31605DA832781046FF05FD7B9
:10E9B0000326C10093F70D01930646006392077E7C
:10E9C00093F70D04E38C07188327C100130E000092
:10E9D0002326D10003DC07006FF0DFEA0326C10025
:10E9E00093F70D01930646006398077893F70D049B
:10E9F000E38607148327C1002326D100039C070068
:10EA0000135EFC4193060E00E3DC06E0B3368001A2
:10EA1000330EC041330EDE409306D002A30DD10267
:10EA20001306F0FF330C804113890D00930610008C
:10EA3000E394CCE613061000E380C6E01306200042
:10EA40006384C6269309010F1316DE0193767C00BA
:10EA500093573C0093860603336CF600135E3E002A
:10EA6000A38FD9FE3366CC01938509009389F9FF02
:10EA7000E31C06FC937719006382072693070003C3
:10EA8000638EF6249385E5FFA38FF9FE9307010FAC
:10EA9000338CB740930D0900938905006FF09FE216
:10EAA0008327C100A30D010283A9070093864700B5
:10EAB000E38609049307F0FF6388FC7813860C0053
:10EAC0009305000013850900232CD1002326E100C3
:10EAD000EF805FC10327C10083268101E304051491
:10EAE000330C35412326D100930C00006FF09FDDDD
:10EAF0008326C100A30D01021309100083A706009D
:10EB0000938646002326D1002306F108130C10003B
:10EB10009309C1086FF05FB28327C10013E92D008C
:10EB2000B786FFFF03AC0700B75D018093874700FE
:10EB300093C606832326F10093878DF4231ED1020A
:10EB4000130E00002328F100930620006FF01FD45D
:10EB50000326C10093F70D02832606001306460024
:10EB60002326C1006390076093F70D016392077835
:10EB700093F70D04E398070893F80D20638A08764D
:10EB8000832781002380F6006FF0DF9B83460D0012
:10EB900093ED0D086FF0DFA383460D0093051D0074
:10EBA000E38A360B938706FD138D0500930C000056
:10EBB000E362FCA283460D0093952C0033839501FC
:10EBC00013131300B30CF300938706FD130D1D0000
:10EBD000E372FCFE6FF01FA083460D0093ED4D0025
:10EBE0006FF01F9F9307B00283460D00A30DF10243
:10EBF0006FF01F9E8327C10083460D0003A407000A
:10EC0000938747002326F100E354049C330480409B
:10EC100093ED4D006FF0DF9B83460D0093ED1D00DB
:10EC20006FF01F9B8347B10383460D00E392079A61
:10EC300093070002A30DF1026FF09F9983460D0028
:10EC40009307C0066388F66693ED0D016FF05F9839
:10EC500083460D00930780066386F66493ED0D04EA
:10EC60006FF01F9713E90D0193770902638407384A
:10EC70008327C100930610009389770093F989FFD9
:10EC80009387890003AC090003AE49002326F100F5
:10EC90006FF0DFBF13061000638EC67813062000E6
:10ECA00013890D00E390C6DA9309010F8327010150
:10ECB0009376FC009389F9FFB386D70003C606005C
:10ECC00093574C009316CE0133ECF600135E4E00C2
:10ECD0002380C900B366CC01E39A06FC9307010FB9
:10ECE000338C3741930D09006FF0DFBDB30624412B
:10ECF000E35ED09E130E00016352DE74130F7000AA
:10ED00006F00C000938606FF635EDE0493870701F1
:10ED100013061600232097002322C7012324F104A1
:10ED20002322C10413078700E35ECFFC130601040E
:10ED300093050A0013050B00232CD100EFF0CFDA66
:10ED4000E31805A083268101130E000183278104A7
:10ED5000938606FF0326410413870A00130F7000F1
:10ED6000E346DEFA13061600130E8700B387D700BA
:10ED7000232097002322D7002324F1042322C10457
:10ED8000130770006340C754B38C8C411305160001
:10ED900093058E0013070E00E35E909513030001A8
:10EDA000635C935F130E70006F00C000938C0CFFC8
:10EDB000635A9305938707011306160023209700D3
:10EDC000232267002324F1042322C10413078700B0
:10EDD000E35ECEFC1306010493050A0013050B0045
:10EDE000EFF08FD0E316059613030001938C0CFF10
:10EDF000832781040326410413870A00130E700041
:10EE0000E34A93FB1305160013068700B3879701A7
:10EE100023209700232297012324F1042322A10415
:10EE2000130770006340A7201307060013051500A1
:10EE3000B307FC0023203701232287012324F10498
:10EE40002322A1041307700093058600E352A78CC8
:10EE50001306010493050A0013050B00EFF0CFC859
:10EE6000E318058E8327810493850A006FF05F8A7B
:10EE70001306010493050A0013050B00EFF0CFC63B
:10EE8000E30C058A6FF0DF8C13890D006FF09FBAD9
:10EE90009305000163D0D508930F00019302700021
:10EEA0006F00C000938606FF63D6DF0693870701D5
:10EEB00013061600232077012322F7012324F104EF
:10EEC0002322C10413078700E3DEC2FC13060104FA
:10EED00093050A0013050B002320D102232EC10144
:10EEE000232CE101EFF04FC0E314058683260102D5
:10EEF000930F000183278104938606FF03264104B4
:10EF0000032EC101032F810113870A0093027000B1
:10EF1000E3CEDFF8B387D700130616002322D7000D
:10EF2000232077012324F1042322C10493067000D7
:10EF30001307870063D6C6F21306010493050A007F
:10EF400013050B00232EC101232CE101EFF0CFB9F3
:10EF5000E31005808327810403264104032EC101A9
:10EF6000032F810113870A006FF08FEF130601044E
:10EF700093050A0013050B00232EC101232CE10188
:10EF8000EFF08FB6631605FC032641048327810446
:10EF9000032EC101032F81019305410513051600BE
:10EFA00013870A006FF08FF01306010493050A001F
:10EFB00013050B00232CC101EFF00FB3631A05F802
:10EFC0000326410483278104032E81019305410513
:10EFD0001305160013870A006FF0CFF0E3940C8638
:10EFE000930D0900930C0000130C00009309010F0E
:10EFF0006FF05F8D0326C1009377090193064600E9
:10F000006396071893770904638807368327C1003E
:10F01000130E00002326D10003DC07009306100026
:10F020006FF0DF861306010493050A0013050B0039
:10F03000EFF08FAB631E05F00325410483278104A5
:10F04000930541051305150013870A006FF08FEA39
:10F05000937709402320F102930D00009309010FDB
:10F060006F00400393050E001306A00093060000F6
:10F0700013050C00232EE100232CC101EF00D02446
:10F08000032E81010327C101630C0E30130C050010
:10F09000138E050093050E001306A00093060000D2
:10F0A00013050C00232EE100232CC101EF00106595
:10F0B0008327010213050503A38FA9FE032E8101F7
:10F0C0000327C1019389F9FF938D1D00E38C07F895
:10F0D0008327410283C60700E396B6F99307F00F32
:10F0E000E382FDF863160E0093079000E3F887BFF4
:10F0F000832781028325C102232EC101B389F940F0
:10F100001386070013850900232CE100EF905FC9E7
:10F1100003274102032EC1011306A00083451700F7
:10F120009306000013050C00B337B000B307F700D7
:10F1300093050E002322F102EF001019032781012D
:10F14000930D00006FF09FF48327410283460D006A
:10F15000638007C883C70700638C07C693ED0D4023
:10F160006FF00FC7032681009357F64123A0C60016
:10F1700023A2F6006FF00FBD032C06002326D1005A
:10F18000135EFC4193060E006FF04FE92326D10079
:10F19000032C0600130E0000930610006FF00FEF13
:10F1A000032C0600130E00002326D1006FF08FED14
:10F1B00013890D006FF05FABB75701809387C7F5D8
:10F1C0002328F10093F70D02638007068327C1000F
:10F1D0009389770093F989FF03AC090003AE4900D6
:10F1E000938789002326F10013F61D00630E0600A5
:10F1F0003366CC01630A060013060003230EC10226
:10F20000A30ED10293ED2D0013F9FDBF930620004C
:10F210006FF0CFE7B7570180938787F42328F10079
:10F2200093F70D02E39407FA8325C10093F70D01CC
:10F2300013864500638A070403AC0500130E000023
:10F240002326C1006FF05FFA13850900232CE1002B
:10F250002326D100EF901FAC03278101130C05007A
:10F26000930C00006FF00FE693050004EF701FCCC5
:10F270002320AA002328AA00630005209307000486
:10F28000232AFA006FF0CFA793F70D04638A0708CB
:10F290008327C100130E00002326C10003DC0700F2
:10F2A0006FF09FF483461D0093ED0D20130D1D009C
:10F2B0006FF00FB283461D0093ED0D02130D1D007C
:10F2C0006FF00FB11306010493050A0013050B003C
:10F2D000EFF08F81631E05C6032641048327810456
:10F2E000930541051305160013870A006FF00FC040
:10F2F0008327810023A0F6006FF0CFA4930760005E
:10F30000138C0C0063F49701130C6000B75E01804E
:10F3100013090C002326D10093890EF76FF0CFB1AB
:10F3200093F70D206386070C8327C100130E00009E
:10F330002326C10003CC07006FF01FEB93F70D20CD
:10F34000638C07088327C1002326D100038C0700A4
:10F35000135EFC4193060E006FF04FCC93F70D2027
:10F36000638207068327C100130E00002326D10005
:10F3700003CC07006FF00FD1937709206388070251
:10F380008327C100130E00002326D10003CC070001
:10F39000930610006FF08FCF138605006FF01FA744
:10F3A00093079000E3E487CF6FF05F938327C1005A
:10F3B000130E00002326D10003AC070093061000B3
:10F3C0006FF0CFCC8327C100130E00002326D1009D
:10F3D00003AC07006FF00FCB8327C1002326D100B9
:10F3E00003AC0700135EFC4193060E006FF00FC3E1
:10F3F0008327C100130E00002326C10003AC0700C1
:10F400006FF09FDE832781002390F6006FF08F93CB
:10F410001306010493050A0013050B00EFE0DFEC6F
:10F420006FF00FB3138C0C002326D100930C000057
:10F430006FF04FC913890D006FF0CFC0138E050018
:10F44000130605006FF09F929307F0FF2324F1004D
:10F450006FF0CFB08327C10083AC070093874700CC
:10F4600063D40C00930CF0FF83461D002326F100AB
:10F47000138D05006FF0CF959307C0002320FB008C
:10F480009307F0FF2324F1006FF04FAD130101FE4D
:10F49000232C8100232A910023282101232E1100EF
:10F4A0002326310113090500938405001304060087
:10F4B0006306050083278503638807140317C400C8
:10F4C00083268401937787002324D40093160701B1
:10F4D00093D606016382070883270401638E07061B
:10F4E0001396260193F9F40F93F4F40F635E060864
:10F4F0000327040083264401B307F74063DED70ADD
:10F5000083268400130617002320C4009386F6FF89
:10F510002324D400230037010327440193871700D5
:10F520006308F70C8357C40093F71700638607003E
:10F530009307A000638EF40A8320C1010324810194
:10F54000032901018329C10013850400832441019B
:10F5500013010102678000009305040013050900F0
:10F56000EF301FD0631E05080317C40093F9F40F92
:10F57000832704019316070193D6060113962601EB
:10F5800093F4F40FE34606F683264406372600007C
:10F590003367C70037E6FFFF1306F6FFB3F6C60072
:10F5A0002316E400032704002322D4068326440103
:10F5B000B307F740E3C6D7F4930504001305090029
:10F5C000EF40CFA1631E05020327040083268400B9
:10F5D00093071000130617009386F6FF2320C4003C
:10F5E0002324D4002300370103274401E31CF7F24E
:10F5F0009305040013050900EF404F9EE30E05F24A
:10F600009304F0FF6FF05FF3EF400FD86FF01FEB44
:10F6100037770180930705000325479C1386050073
:10F62000938507006FF09FE6130101FE232C8100F4
:10F63000232A9100B7770180232E110083A7879199
:10F64000130405009384060063820502E780070027
:10F650009307F0FF6306F5028320C10103248101B3
:10F66000832441011301010267800000130600009A
:10F6700093054100E78007009307F0FFE31EF5FCC8
:10F6800023A004009307A0088320C1012320F400D5
:10F6900003248101832441011301010267800000DA
:10F6A000130101FEB7770180232C8100232A9100EA
:10F6B000232E110083A4479CB777018083A78791ED
:10F6C00013040600630A050213860500930604006E
:10F6D0009305050013850400E78007009307F0FFFA
:10F6E000630AF5028320C1010324810183244101BF
:10F6F0001301010267800000930606009305410094
:10F700001306000013850400E78007009307F0FF4D
:10F71000E31AF5FC232004008320C10103248101A6
:10F720009307A00823A0F4008324410113010102E0
:10F7300067800000B777018003A38791670003000B
:10F74000638405029307F00F63E8C7002380C500B8
:10F7500013051000678000009307A0082320F50020
:10F760001305F0FF678000001305000067800000AC
:10F77000130101FF1305600023261100EF00C028CC
:10F7800013051000EF009F90130101FF930500087F
:10F79000232481002326110013040500EF700FF9C4
:10F7A000232EA42C630405029307050823200500DB
:10F7B00013054500E31CF5FE130500008320C1007E
:10F7C0000324810013010101678000001305F0FF8D
:10F7D0006FF0DFFE8327C52D638607001305000049
:10F7E000678000006FF05FFA130101FE232A910089
:10F7F000232E1100232C81009307F00193040500B0
:10F8000063EAB702138405008325C52D63840504CC
:10F810001314240033848500032504002320C4002E
:10F820008320C101032481018324410113010102CA
:10F83000678000008320C1010324810193076001D8
:10F840002320F500832441011305F0FF1301010279
:10F85000678000002326C100EFF01FF39307050027
:10F860001305F0FFE39E07FA83A5C42D0326C1000C
:10F870006FF01FFA130101FF2322910023261100CC
:10F88000232481009307F0019304050063EAB70A7B
:10F890008327C52D1384050063840704139725006F
:10F8A000B387E70003A70700630C07029306100065
:10F8B000630CD7069306F0FF6308D7041385050091
:10F8C00023A00700E7000700130500008320C10004
:10F8D000032481008324410013010101678000009B
:10F8E00013850400EF00001E1306040003248100AA
:10F8F0008320C10093050500138504008324410083
:10F90000130101016F0080158320C10003248100D1
:10F91000930760012320F5008324410013051000A4
:10F9200013010101678000008320C10003248100CE
:10F9300083244100130500001301010167800000CA
:10F94000930760012320F5001305F0FF6FF01FF807
:10F950009307F00163E6B70A8327C52D130101FE63
:10F96000232C9100232E110093040500638C0704BF
:10F9700013972500B387E70003A70700630A070270
:10F980009306F0FF6306D706930610006308D704BA
:10F990001385050023A00700E700070013050000FA
:10F9A0008320C101832481011301010267800000CB
:10F9B0008320C1018324810113051000130101027A
:10F9C000678000002326B100EFF01FDC63160502FC
:10F9D00083A7C42D8325C1006FF09FF98320C10147
:10F9E00083248101130530001301010267800000A8
:10F9F000130520006FF0DFFA1305F0FF6FF05FFAD8
:10FA00001305F0FF67800000B777018093050500BC
:10FA100003A5479C6FF01FE6377701809307050029
:10FA20000325479C13860500938507006FF0DFDBF5
:10FA3000B777018003A5479C8327C52D6386070000
:10FA400013050000678000006FF01FD4B7770180B6
:10FA50009305050003A5479C6FF09FEF130101FF7D
:10FA6000138705002324810023229100130405003D
:10FA7000B7740180930506001305070023261100C3
:10FA800023A204A0EF00CFED9307F0FF630CF50075
:10FA90008320C1000324810083244100130101015C
:10FAA0006780000083A744A0E38407FE8320C10091
:10FAB0002320F40003248100832441001301010169
:10FAC000678000006F004FEA9308050093870500E8
:10FAD00013080600138506001383080063940628A4
:10FAE000B7660180938646BC63F6C50E37070100F2
:10FAF0006378E60C1307F00F3337C700131737008E
:10FB00003355E600B386A60083C60600130500023F
:10FB10003387E600B306E540630CE500B397D700F2
:10FB200033D7E8003318D600B365F7003393D80015
:10FB300093580801B3D7150313160801135606018D
:10FB400013570301B3F6150313850700B305F60237
:10FB50009396060133E7E600637EB700330707019B
:10FB60001385F7FF636807016376B7001385E7FF26
:10FB7000330707013307B740B377170313130301A4
:10FB800013530301335717039397070133E36700B8
:10FB9000B306E60213060700637CD3003303680054
:10FBA0001306F7FF636603016374D3001306E7FFD0
:10FBB000131505013365C500930500006F00400E65
:10FBC0003705000113070001E36CA6F2130780015B
:10FBD0006FF01FF363160600130710003358C702B7
:10FBE000370701006370E80C1307F00F6374070117
:10FBF000130580003357A800B386E60003C706004C
:10FC0000130600023307A700B306E6406316E60AB0
:10FC1000B387074193051000935808011316080194
:10FC20001356060113570301B3F61703B3D717038F
:10FC30009396060133E7E600330EF60213850700BC
:10FC4000637EC701330707011385F7FF6368070168
:10FC50006376C7011385E7FF330707013307C74101
:10FC6000B377170313130301135303013357170318
:10FC70009397070133E36700B306E6021306070014
:10FC8000637CD300330368001306F7FF6366030148
:10FC90006374D3001306E7FF131505013365C50030
:10FCA000678000003707000113050001E364E8F4F2
:10FCB000130580016FF01FF43318D800B3D5E700A7
:10FCC0003393D800B397D70033D7E800935808018F
:10FCD0003366F70033F715039317080193D707012D
:10FCE00013550601B3D51503131707013367A70092
:10FCF000B386B70213850500637ED700330707017B
:10FD00001385F5FF636807016376D7001385E5FF68
:10FD100033070701B306D74033F71603131606015E
:10FD200013560601B3D6160313170701B388D7027B
:10FD3000B367C7001387060063FE1701B387070187
:10FD40001387F6FF63E8070163F617011387E6FFE1
:10FD5000B387070193150501B3871741B3E5E500A4
:10FD60006FF09FEB63E6D5183707010063F4E604F4
:10FD70001307F00FB335D70093953500376701802F
:10FD800033D5B600130747BC3307A7000347070066
:10FD9000130500023307B700B305E5406316E5021B
:10FDA00013051000E3EEF6EE33B5C8001345150059
:10FDB0006FF01FEF3707000193050001E3E0E6FC59
:10FDC000930580016FF09FFB3353E600B396B600B6
:10FDD0003363D30013550301B31EB60033D6E700D7
:10FDE000B376A602B397B70033D7E8003368F700BD
:10FDF0009317030193D70701135708013356A6023F
:10FE00009396060133E7E600338FC702130E060010
:10FE1000637EE70133076700130EF6FF6368670030
:10FE20006376E701130EE6FF330767003307E74108
:10FE3000B376A7023357A702939606013386E702EB
:10FE40009317080193D70701B3E7F600930607005D
:10FE500063FEC700B38767009306F7FF63E8670098
:10FE600063F6C7009306E7FFB387670013150E011B
:10FE7000370E01003365D5009306FEFF3378D500B9
:10FE8000B387C740B3F6DE001356050193DE0E01BB
:10FE90003303D802B306D602135703013308D8033D
:10FEA0003308D800330707013306D6036374D7003D
:10FEB0003306C601935607013386C60063E6C702C0
:10FEC000E39CC7CEB70701009387F7FF3377F700AE
:10FED000131707013373F300B398B80033076700B3
:10FEE00093050000E3FEE8DA1305F5FF6FF0DFCCC1
:10FEF00093050000130500006FF09FDA93080600D9
:10FF0000138706009307050013880500639C0622EB
:10FF1000B7660180938646BC63FCC50C37030100BD
:10FF2000637E660A1303F00F6374C3001307800037
:10FF30003353E600B386660003CE0600330EEE00B0
:10FF4000130700023303C741630CC701B395650073
:10FF5000335EC501B31866003368BE00B317650091
:10FF600013D608013377C80213950801135505010C
:10FF700093D607013358C80213170701B366D70099
:10FF80003308050363FA0601B386160163E616011A
:10FF900063F40601B3861601B386064133F7C60241
:10FFA0009397070193D70701B3D6C602B306D502CC
:10FFB00013150701B367F50063FAD700B38717017C
:10FFC00063E6170163F4D700B3871701B387D740FF
:10FFD00033D56700930500006780000037030001F8
:10FFE00013070001E36666F4130780016FF05FF406
:10FFF0006316060013061000B358160337060100F7
:02000004800179
:1000000063F2C80A1306F00F637416011307800029
:1000100033D6E800B386C60003CE0600330EEE00EA
:10002000130700023303C7416318C709B38515419D
:1000300013D70801139508011355050113D60701BD
:10004000B3F6E502B3D5E50293960601B3E6C60022
:10005000B305B50263FAB600B386160163E616016E
:1000600063F4B600B3861601B385B640B3F6E50275
:100070009397070193D70701B3D5E502B305B502FE
:1000800013950601B367F50063FAB700B38717014C
:1000900063E6170163F4B700B3871701B387B7406E
:1000A0006FF01FF33706000113070001E3E2C8F603
:1000B000130780016FF0DFF5B398680033D7C501EF
:1000C000B3176500335EC50113D50801B376A702E7
:1000D000B3956500336EBE009395080193D5050175
:1000E00013560E013357A70293960601B3E6C600D6
:1000F0003387E50263FAE600B386160163E616016C
:1001000063F4E600B38616013386E640B376A602B2
:10011000131E0E01135E0E013356A60293960601BE
:100120003386C502B3E5C60163FAC500B385150180
:1001300063E6150163F4C500B3851501B385C540B9
:100140006FF01FEFE3EAD5E83707010063FCE60430
:10015000130EF00F3337DE0013173700B768018036
:1001600033D3E600938848BCB388680003CE080008
:10017000330EEE00130700023303C741631EC703AB
:1001800063E4B600636AC500B307C540B385D540D4
:100190003335F5003388A540138507009305080023
:1001A0006FF09FE3B708000113070001E3E816FBB7
:1001B000130780016FF09FFA3357C601B3966600AC
:1001C000336FD700B3D7C50113570F01B3F8E70258
:1001D000B39565003358C5013368B80093150F0116
:1001E00093D5050193560801331666003315650053
:1001F000B3D7E70293980801B3E6D800B38EF502AF
:100200009388070063FED601B386E6019388F7FF63
:1002100063E8E60163F6D6019388E7FFB386E6015B
:10022000B386D641B3FEE60213180801135808013D
:10023000B3D6E602939E0E01B3EE0E01B385D5024E
:100240009387060063FEBE00B38EEE019387F6FF30
:1002500063E8EE0163F6BE009387E6FFB38EEE011E
:10026000B385BE4093980801B70E0100B3E8F800CB
:100270009387FEFF33F8F8009356060193D80801E0
:10028000B377F6003307F802B387F8023308D802D1
:10029000B388D8023308F80093560701B3860601E5
:1002A00063F4F600B388D801B70701009387F7FF1E
:1002B00013D80601B3F6F600939606013377F700DC
:1002C000B30818013387E60063E61501639E150144
:1002D000637CE5003306C7403337C7003307E701C7
:1002E000B388E840130706003307E5403335E500DF
:1002F000B3851541B385A540B397C5013357670052
:1003000033E5E700B3D565006FF01FCD130101FDA4
:1003100023248102232A510123248101232611024F
:100320002322910223202103232E3101232C41017A
:100330002328610123267101232291011304050062
:10034000130C0600938A06007329200093D74501F9
:10035000939BC5001397570193DBCB0013DAF5018C
:10036000630C070213FBF77F9307F07F6308FB081A
:100370001357D501939B3B00B36B7701B707800000
:10038000B3EBFB0093193500130B1BC0930C00005B
:10039000930400006F008008B3E7AB00638E070E84
:1003A00063800B0413850B00EF401033130755FFD8
:1003B0009307C00163CCE7029306D001930985FF40
:1003C000B386E640B39B3B01B356D400B3EB760152
:1003D000B31934019305D0C0338BA5406FF01FFBD8
:1003E000EF40902F130505026FF05FFC930B85FD26
:1003F000B31B7401930900006FF0DFFD33E4AB0021
:100400006306040A9397CB0093090500130BF07F52
:10041000930C300093040001E3CC07F613D74A0194
:100420001395CA009316570193070C001354C50087
:100430009375F77F93DAFA01638406081307F07F58
:100440006386E50E9357DC011315340033E5A700EE
:10045000370480003364850093173C00138515C072
:100460001307000093962C00B3E6E600B305AB40FB
:100470009386F6FF1305E00033465A016360D510FA
:100480003765018093962600130505B1B386A60053
:1004900083A6060067800600930B00009309000006
:1004A000130B0000930C10006FF09FEE930B0000F5
:1004B00093090000130BF07F930C20006FF05FEDA9
:1004C000B36784016384070863020404130504000E
:1004D000EF40902093050500938655FF9307C001D8
:1004E00063CED7021307D001938785FF3307D74028
:1004F0003315F4003357EC003364A700B317FC0046
:100500001307D0C03305B7406FF09FF513050C00FB
:10051000EF40901C930505026FF01FFC138585FDCD
:100520003314AC00930700006FF09FFD3366840125
:10053000630806021317C4001305F07F634C07021B
:1005400013073000930400016FF0DFF11304000083
:100550009307000013050000130710006FF09FF0D1
:1005600013040000930700001305F07F1307200019
:100570006FF05FEF130730006FF0DFEE636674011A
:1005800063968B2E63E4F92E1395FB0113D71900A4
:100590009396F90193DB1B00B369E5001315840002
:1005A00013D887013368A8001355050133D3AB0274
:1005B000131E0801135E0E019398870093D709015B
:1005C000B3FBAB02930F030033076E02939B0B0147
:1005D000B3E7770163FEE700B3870701930FF3FFEB
:1005E00063E8070163F6E700930FE3FFB3870701B2
:1005F000B387E740B3DEA7029399090193D90901B4
:10060000B3F7A70213830E003307DE0393970701A6
:10061000B3E7F90063FEE700B38707011383FEFF2A
:1006200063E8070163F6E7001383EEFFB387070172
:100630003387E740939F0F01B7070100B3EF6F00C7
:100640001383F7FF33FF6F0093D20F0193DE08018E
:1006500033F3680033046F02B3896202338FEE0311
:10066000B3033F01135F0401330F7F00B382D20352
:1006700063743F01B382F200B703010093570F0187
:100680009383F3FFB3825700B3777F0093970701FB
:1006900033747400B38787006368570013840F00B6
:1006A0006314570463F2F604B386160133BF1601D0
:1006B000330F0F013307E7011384FFFF6366E80080
:1006C0006314E80263E2160363665700639EE20068
:1006D00063FCF600B386160133BF1601330F0F011A
:1006E0001384EFFF3307E701338FF640330757409A
:1006F000B3B6E6013307D7409307F0FF6304E8126F
:10070000B352A70293570F013377A70293860200D3
:10071000B30F5E021317070133E7E700637EF701AB
:10072000330707019386F2FF636807016376F701D9
:100730009386E2FF330707013307F741B35FA70250
:1007400093170F0193D707013377A702330EFE03E8
:100750001317070133E7E70093870F00637EC70194
:10076000330707019387FFFF636807016376C701BB
:100770009387EFFF3307070193960601B3E6F60070
:100780009397060193D707013307C74113DE06018C
:10079000330FF30233036E02338ECE03B38EFE02A9
:1007A00093570F01B38E6E00B387D70163F66700CE
:1007B00037050100330EAE0013D307013303C30125
:1007C000370E0100130EFEFF33F5C70113150501A7
:1007D000337FCF013305E501636867006314673E2B
:1007E00093870600630005043307E8009387F6FF4C
:1007F00063640703636667006314673C63F0A802E1
:100800009387E6FF93961800B3B816013388080162
:100810003307070193880600631467006384A80008
:1008200093E717001388F53F635A001913F7770011
:10083000630A070A1307200093E414006302E90A1D
:10084000130730006308E908631E090813F7F7006F
:10085000930640006308D70813874700B337F700B3
:100860003304F400930707006F00C0079385F5FF7A
:10087000930600006FF09FD213060A0013840B004A
:100880009387090013870C00930630006300D7326A
:10089000930610006306D73093062000E314D7F8C0
:1008A0006F00000113860A006FF01FFE93E48400BE
:1008B00013050000930700001307F07F6F00C005C9
:1008C00037040800930700001306000013073000E8
:1008D0006FF09FFB63180600138787006FF01FF807
:1008E000E31C06FE13177400635A0700370700FF66
:1008F0001307F7FF3374E400138805401307E07F04
:10090000634E070713D737009317D401B3E7E70007
:10091000135534001307080013174701B706F07F7B
:100920001315C5003377D7001355C5003365A700ED
:100930001316F6013367C5009305070013850700FA
:100940006384040073A014008320C1020324810285
:1009500083244102032901028329C101032A810161
:10096000832A4101032B0101832BC100032C810049
:10097000832C4100130101036780000093072000CE
:10098000630AF90293073000630AF900631A090049
:10099000930700001307F07F6F000001E30A06FED3
:1009A0009307F0FF1307E07F93E4540013850700DB
:1009B0006FF09FF6E31E06FC6FF09FFE130710001A
:1009C0006316080693F6770013070400638A06048B
:1009D0001307200093E414006300E90413073000B8
:1009E0006304E90213070400631C090293F6F7008D
:1009F000130540006386A60213B7C7FF134717000D
:100A0000330787006F00C00113070400631A060054
:100A100013B787FF6FF09FFE13070400E31A06FE6B
:100A2000135787011347170013771700130510009A
:100A3000330505419306800363CCA60E9306F001AF
:100A400063C2A6069385E54133D8A700B316B40068
:100A5000B397B700B3E60601B337F000B3E7F6008B
:100A60003355A40093F677006380060893062000B0
:100A700093E414006308D90693063000630ED9048A
:100A80006314090693F6F70093054000638EB604DD
:100A900093864700B3B7F6003305F5009387060049
:100AA0006F008004930610FEB3860641930800028F
:100AB000B356D40013080000630615019385E5437F
:100AC0003318B400B367F800B337F000B3E7F600AB
:100AD000130500006FF01FF9631806009386870066
:100AE0006FF05FFBE31C06FE9316850063DE0600D5
:100AF00093E4140013050000930700006316070237
:100B0000130710006FF05FE193D637009317D501FC
:100B1000B3E7D70013553500E30007E013F71400DF
:100B2000E30C07DE1307000093E424006FF0DFDE20
:100B3000B3E78700638407029307200093E414005F
:100B4000630EF902930730006302F9029307100065
:100B5000631409009307500093D7370093E42400EF
:100B600013050000130700006FF01FDB93079000D0
:100B7000E30406FE930710006FF01FFE930790003A
:100B8000E31C06FC6FF01FFF370508009307000009
:100B90001307F07F13060000930400016FF0DFD706
:100BA00013050000930700006FF0DFFB3705080016
:100BB000930700001307F07F130600006FF0DFD5E6
:100BC00093860700938706006FF09FC5130101FD10
:100BD000232481022328610123229101232611026B
:100BE0002322910223202103232E3101232C4101B2
:100BF000232A5101232671012324810113040500B6
:100C0000930C0600138B06007329200093D745012F
:100C10009399C5001397570193D9C90093DAF50149
:100C2000630C070293FBF77F9307F07F6388FB0851
:100C30009357D50193993900B3E93701B70780007D
:100C4000B3E9F900131A3500938B1BC0130C000095
:100C5000930400006F008008B3E7A90063800710C9
:100C60006380090413850900EF400027130755FF2F
:100C70009307C00163CCE7029307D001130A85FFF5
:100C8000B387E740B3994901B357F400B3E937019B
:100C9000331A4401930BD0C0B38BAB406FF01FFBF2
:100CA000EF408023130505026FF05FFC930985FD7B
:100CB000B3193401130A00006FF0DFFD33E4A9001B
:100CC0006308040A9397C900130A0500930BF07F89
:100CD000130C300093040001E3CC07F613574B01CB
:100CE0001314CB009316570193870C001354C400C0
:100CF0001375F77F135BFB01638606081307F07F0C
:100D00006306E50E93D7DC011314340033E4870047
:100D1000B70780003364F400130515C093973C00B7
:100D20001307000093162C00B3E6E600B38BAB006C
:100D30009386F6FF1306E000B3C56A0113851B0016
:100D4000636AD61637660180939626001306C6B4EA
:100D5000B386C60083A606006780060093090000DC
:100D6000130A0000930B0000130C10006FF05FEEED
:100D700093090000130A0000930BF07F130C20006E
:100D80006FF01FEDB36794016382070863000404EA
:100D900013050400EF404014930655FF9307C0016C
:100DA00063CED7021307D001930785FF3307D740DF
:100DB0003314F40033D7EC0033648700B397FC009E
:100DC0001307D0C03305A7406FF09FF513850C00C3
:100DD000EF408010130505026FF01FFC130485FD22
:100DE00033948C00930700006FF09FFD33669401ED
:100DF000630806021317C4001305F07F634C070253
:100E000013073000930400016FF0DFF113040000BA
:100E10009307000013050000130710006FF09FF008
:100E200013040000930700001305F07F1307200050
:100E30006FF05FEF130730006FF0DFEE370408004C
:100E4000930700001307F07F93050000930400014F
:100E500013174701B706F07F1314C4003377D70088
:100E60001354C4009395F501336487003367B400CD
:100E700013850700930507006384040073A0140022
:100E80008320C10203248102832441020329010239
:100E90008329C101032A8101832A4101032B010116
:100EA000832BC100032C8100832C4100130101031B
:100EB00067800000370601001307F6FF93560A010A
:100EC00013DE0701337AEA00B3F7E70033034E037A
:100ED000B38E4703338FF6023308E30113D30E01B9
:100EE00033030301B388C6036374E301B388C80006
:100EF0003378E300B3FEEE00135603011318080124
:100F0000135304013374E4003308D801330F8A0209
:100F1000B38E8602330A43033307DA01135A0F01F3
:100F2000330AEA00B38666026376DA013707010006
:100F3000B386E600935E0A01B38EDE00B7060100B9
:100F40009382F6FF337A5A00337F5F0013D709018B
:100F5000131A0A01B3F95900330AEA01B302EE0287
:100F6000B30F4601338F3703330E3E0313560F0181
:100F7000B307F702330EFE003306C6016374F600B2
:100F8000B382D200B70601009387F6FF135E060115
:100F90003376F600337FFF0013160601B38789020C
:100FA0003306E601330E5E0033048702330FE3029B
:100FB00013D707013303330333038300330367007D
:100FC00063748300330FDF00370701001307F7FF57
:100FD000B376E300B3F7E70093960601B388F80110
:100FE000B386F60033BA4801B386D601338746018B
:100FF000B388C80033B6C800B30FC701B382CF00AF
:10100000B3B6D6013337470133E7E60033B6C20043
:101010001353030133BECF01330767003366CE009D
:10102000939798003307C7003307E701B3E7070139
:1010300013179700B337F00093D8780113D47201D7
:10104000B3E71701939292009316770033648700F9
:10105000B3E7570063D0060A13D7170093F71700BA
:10106000B367F7001317F401B3E7E7001354140054
:101070001308F53F6358001113F77700630807085A
:101080001307200093E414006300E90813073000FD
:101090006306E906631C090613F7F7009306400090
:1010A0006306D70613874700B337F7003304F4000D
:1010B000930707006F00800593850A0013840900D9
:1010C00093070A0013070C00930620006302D72839
:1010D000930630006306D72893061000E31AD7F86A
:1010E00013040000930700006F00402493050B00D9
:1010F0006FF09FFD13850B006FF09FF7639805005D
:10110000138787006FF05FFAE39C05FE13177400E6
:10111000635A0700370700FF1307F7FF3374E40033
:10112000130805401307E07F634E070113D737000C
:101130009317D401B3E7E7001354340013070800F2
:101140006FF01FD193072000630AF9029307300064
:10115000630AF900631A0900930700001307F07F80
:101160006F000001E38A05FE9307F0FF1307E07F9D
:1011700093E45400138407006FF09FCDE39E05FCB9
:101180006FF09FFE130710006316080693F67700B2
:1011900013070400638A06041307200093E4140075
:1011A0006300E904130730006304E9021307040035
:1011B000631C090293F6F700130640006386C6021B
:1011C00013B7C7FF13471700330787006F00C0012D
:1011D00013070400639A050013B787FF6FF09FFEA3
:1011E00013070400E39A05FE1357870113471700FE
:1011F0001377170093061000B38606411306800389
:10120000634CD60E1306F0016342D6061305E54182
:101210003316A40033D8D700B397A700336606016E
:10122000B337F000B367F6003354D40093F6770079
:10123000638006089306200093E414006308D9062F
:1012400093063000630ED9046314090693F6F70081
:1012500013064000638EC60493864700B3B7F600BA
:101260003304F400938706006F008004130610FE19
:1012700033060641930800023356C40013080000E9
:10128000638616011305E5433318A400B367F8001D
:10129000B337F000B367F600130400006FF01FF9D6
:1012A00063980500938687006FF05FFBE39C05FE63
:1012B0009316840063DE060093E414001304000018
:1012C0009307000063160702130710006FF05FB862
:1012D00093D637009317D401B3E7D70013543400E3
:1012E000E30807B613F71400E30407B6130700007A
:1012F00093E424006FF0DFB5B3E78700638407024F
:101300009307200093E41400630EF9029307300062
:101310006302F90293071000631409009307500059
:1013200093D7370093E42400130400001307000050
:101330006FF01FB293079000E38405FE930710003F
:101340006FF01FFE93079000E39C05FC6FF01FFFFA
:1013500013040000930700001307F07F6FF05FAFE6
:1013600037040800930700001307F07F930500007F
:101370006FF01FAE83270500832E4500032F8500E5
:101380008326C50003A7050083A2450083AF85001F
:1013900003A3C500130101FF732620003788000056
:1013A00013D606011308F8FF139E060193150301D7
:1013B00093D8F6013376060193560301135E0E01AE
:1013C00093D50501B3F606011353F301631E06011D
:1013D00033E8D7013368E8013368C80163120808AD
:1013E000639CC60A6F008000639A06013368570049
:1013F0003368F8013368B800631608041305100059
:101400006396C6026394E70263925E026310FF0371
:10141000631EBE0063846802639A060033E5D70149
:101420003365E5013365C5013335A00013010101C2
:1014300067800000736018006F000006130500004D
:101440006FF0DFFE378500001305F5FF6310A6047B
:10145000B3E7D701B3E7E701B3E7C7016388070242
:1014600013150E0113550541E35605FCB78700001F
:101470009387F7FF13051000E39AF6FA33675700D6
:101480003367F7013367B700E30207FA9395050165
:1014900093D50541E3D005FA130510006FF01FF94D
:1014A000832F050003284500032E850083A2050035
:1014B0000325C50083A8450083AE850083A6C5002B
:1014C000130101FFF3272000B78700001356050121
:1014D0009387F7FF931505011393060113D70601B0
:1014E0003376F60093D505011355F5011353030127
:1014F0003377F70093D6F6016310F602B3E70F01D6
:10150000B3E7C701B3E7B7006384070C7360180043
:101510001305E0FF6F000005631AF700B3E712013F
:10152000B3E7D701B3E76700E39207FE6314060A47
:10153000B3E70F01B3E7C701B3E7B70093B71700ED
:10154000631A070033EF1201336FDF01336F6F004F
:1015500063040F06638207081305F0FF6384060027
:101560001385060013010101678000009307000046
:101570006FF05FFD6356E600E31605FE6F00800620
:101580006360B306639E650263ECCE05631EDE03F3
:1015900063E808056314180163E4F205E36E18FDBF
:1015A00063141801E3EA5FFC130500006FF09FFB72
:1015B000130510006FF01FFBE39807FE6F00400259
:1015C000E3EC65FA6FF05FFEE368DEFB6FF0DFFDD2
:1015D000E306C7F4E30C07F86394A600E35CC7F8DE
:1015E000E30805FC1305F0FF6FF0DFF7832F05001C
:1015F00003284500032E850083A205000325C500AE
:1016000083A8450083AE850083A6C500130101FFB2
:10161000F3272000B7870000135605019387F7FFD3
:10162000931505011393060113D706013376F600CF
:1016300093D505011355F501135303013377F700D3
:1016400093D6F6016310F602B3E70F01B3E7C701C3
:10165000B3E7B7006384070C73601800130520001C
:101660006F000005631AF700B3E71201B3E7D70173
:10167000B3E76700E39207FE6314060AB3E70F01BE
:10168000B3E7C701B3E7B70093B71700631A0700C2
:1016900033EF1201336FDF01336F6F0063040F0606
:1016A000638207081305F0FF6384060013850600B4
:1016B0001301010167800000930700006FF05FFDD8
:1016C0006356E600E31605FE6F0080066360B3060E
:1016D000639E650263ECCE05631EDE0363E80805C6
:1016E0006314180163E4F205E36E18FD6314180136
:1016F000E3EA5FFC130500006FF09FFB1305100089
:101700006FF01FFBE39807FE6F004002E3EC65FA01
:101710006FF05FFEE368DEFB6FF0DFFDE306C7F40A
:10172000E30C07F86394A600E35CC7F8E30805FC44
:101730001305F0FF6FF0DFF7130101F42328210BED
:101740002324410B2322510B2320610B232C8109DD
:10175000232A91091309050083A6050083A74500E4
:1017600003A5850083AAC500832C0600032B460031
:10177000032C8600032AC600232E110A232C810A7B
:10178000232A910A2326310B232E71092328A1092C
:101790002326B109F32420003786000013970A019D
:1017A00093D90A01135707011306F6FF23265107A1
:1017B0002320D1062322F1062324A1062328D102C7
:1017C000232AF102232CA102232EE102B3F9C9003E
:1017D00093DAFA0163800906638EC91637050100A2
:1017E0003367A700232EE102130601039307C10309
:1017F00003A7070083A6C7FF9387C7FF1317370008
:1018000093D6D6013367D70023A2E700E312F6FE92
:101810008327010337C5FFFF130515009397370092
:101820002328F102B389A900930B000013040000E0
:101830006F00801433E6D7003366A6003366E600F7
:10184000630606206300070613050700EF30C06833
:10185000930645FF93D7564093F6F601638E06062E
:101860001307C0FF3387E7021303010313080002C5
:10187000939527003308D8401307C7003307E300C8
:101880006314E30813070108B305B7000327010336
:101890009387F7FFB316D70023A8D5FA9306F0FF76
:1018A0006F00000A63080500EF30006313050502AE
:1018B0006FF01FFA638A070013850700EF30C061DD
:1018C000130505046FF0DFF813850600EF30C060E4
:1018D000130505066FF0DFF71306C0FF3386C70256
:1018E0001307C10393063000B305C70083A50500A5
:1018F0009386F6FF1307C7FF2322B700E3D6F6FE51
:101900009387F7FF6FF09FF90326C7FF832807002F
:10191000330EB70033560601B398D800336616016C
:101920002320CE001307C7FF6FF09FF51397270002
:10193000130601033307E600232007009387F7FF10
:10194000E396D7FEB7C9FFFF93891901B389A94070
:101950006FF09FEDB3E7D700B3E7A700B3E7E70069
:10196000638C070E1317070113570741930B3000C1
:1019700013040001E34C07EA13150A01378700003E
:1019800093570A01135505011307F7FF2326410753
:101990002320910723226107232481072320910517
:1019A00023226105232481052326A104B3F7E70040
:1019B000135AFA016386070A6384E71C370701009C
:1019C0003365E5002326A104930501041307C10430
:1019D000832607000326C7FF1307C7FF9396360029
:1019E0001356D601B3E6C6002322D700E392E5FEE4
:1019F0000327010437C5FFFF130515001317370030
:101A00002320E1043385A700930600003307350146
:101A10002324E100130717002322E10013972B0072
:101A20003367D7001307F7FF1306E000B3C74A0177
:101A30006362E61C3766018013172700130686B819
:101A40003307C7000327070067000700930900005A
:101A5000930B10006FF09FDD930B20006FF01FDDE4
:101A6000B3679B01B3E78701B3E7A700638007145F
:101A7000630E0504EF304046930645FF93D756406A
:101A800093F6F601638006081307C0FF3387E70269
:101A90001303010413080002939527003308D8406C
:101AA0001307C7003307E3006316E30813070108B1
:101AB000B305B700032701049387F7FFB316D700D8
:101AC00023A0D5FC9306F0FF6F00400A630A0C00C8
:101AD00013050C00EF304040130505026FF0DFF9ED
:101AE000630A0B0013050B00EF30003F13050504DC
:101AF0006FF09FF813850C00EF30003E13050506CC
:101B00006FF09FF71306C0FF3386C7021307C104A7
:101B100093063000B305C70083A505009386F6FF42
:101B20001307C7FF2322B700E3D6F6FE9387F7FF1C
:101B30006FF05FF90326C7FF83280700330EB70055
:101B400033560601B398D800336616012320CE0021
:101B50001307C7FF6FF05FF5139727001306010403
:101B60003307E600232007009387F7FFE396D7FEAD
:101B7000B7C7FFFF938717013385A7406FF0DFE8F2
:101B8000336B9B01336B8B01336BAB0063060B0232
:101B9000131505011355054163460502138507001A
:101BA00093063000130400016FF05FE61305000098
:101BB000930610006FF09FE5138507009306200041
:101BC0006FF0DFE413850700930630006FF01FE429
:101BD0001304000137870000232EE104232C0104A5
:101BE000232A0104232801041307F7FF93070000A9
:101BF0006F00D0198325010303250104B7080100F4
